:020000040800F2
:10000000D80900207531000851310008533100082B
:100010005531000857310008593100080000000030
:100020000000000000000000000000005B3100083C
:100030005D310008000000005F31000861310008F8
:100040009131000895310008993100089D31000870
:10005000A1310008A5310008A9310008AD31000820
:10006000B1310008B5310008B9310008BD310008D0
:10007000C1310008C5310008C9310008CD31000880
:10008000D1310008D5310008D9310008DD31000830
:10009000E1310008E5310008E9310008ED310008E0
:1000A000F1310008F5310008F9310008FD31000890
:1000B0000132000805320008093200080D3200083C
:1000C0001132000815320008193200081D320008EC
:1000D0002132000825320008293200082D3200089C
:1000E0003132000835320008393200083D3200084C
:1000F0004132000845320008493200084D320008FC
:100100005132000855320008593200085D320008AB
:100110006132000865320008693200086D3200085B
:100120007132000875320008793200087D3200080B
:100130008132000885320008893200088D320008BB
:100140009132000895320008993200089D3200086B
:10015000A1320008A5320008A9320008AD3200081B
:10016000B1320008B5320008B9320008BD320008CB
:10017000C1320008C5320008C9320008CD3200087B
:10018000D1320008D5320008D9320008DD3200082B
:10019000E1320008E5320008E9320008ED320008DB
:1001A000F1320008F5320008F9320008FD3200088B
:1001B0000133000805330008093300080D33000837
:1001C00011330008153300087CB5044600F0EEFA40
:1001D00006460CB9012076BD04F1400529780129B5
:1001E00001D1022076BD01202870687838B900213D
:1001F0002046297000F0D9FA41F28831A9602068C0
:1002000033460168A26821F4F851521E41EA0221E6
:100210000022016000F0C7F9010022D122681249D2
:10022000136866680B40E16843EA06630B43E169C3
:100230000B43216A0B430D491360226853682669FA
:100240000B40616943EA06430B43A1690B435360CA
:1002500021680A6842F001020A60002169600121F8
:1002600069700021297076BD2FFFFF00FEF8E0FFC6
:1002700010B508B9012010BD00F140042178012912
:1002800001D1022010BD0122227001680A685208C3
:1002900052000A6000F090FA0020606060702070E8
:1002A00010BD2DE9F84304460E46154604F14007FB
:1002B00000F07CFA80463878012808BF022026D05A
:1002C00001213970797801291CD1002043467860DA
:1002D000022078700022009500F067F9814698B9F5
:1002E00000F017F8706A50B90095434601220221C8
:1002F00000F05CF9814638B921680220C86001200D
:10030000787001E04FF00209002038704846BDE8DF
:10031000F28300223146204600F0AAB92DE9FC41C3
:10032000074607F140060C46154600F03FFA3968CB
:100330008046327801F12000012A08BF022043D014
:10034000012333707378012B3BD10022726094B388
:10035000122272700A69521CFA620B695B1CBB6242
:100360007C624A69044622F040624A610EE0012242
:100370000421384600F058F9010019D1786A411C6F
:10038000796200782070F96A491EF962F86A00956E
:1003900043460028EBD101220221384600F044F9FF
:1003A000010005D139680220C860384600F000F924
:1003B0000122727006E0706840F008007060012051
:1003C00000E0022000213170BDE8F6812DE9F843FC
:1003D00006460C46914606F1400700F0E7F9316801
:1003E00080468A693878012801F1200508BF02207B
:1003F00047D001233B707B78012B3FD100207860F0
:10040000B4B3222078700B695B1CB3630869401C8D
:10041000706334634B6923F0406343F080634B6146
:1004200031688A610EE001220621304600F0FCF8B6
:1004300001001AD1306B411C316329780170B16B16
:10044000491EB163B06BCDF8009043460028EAD155
:1004500001220221304600F0E7F8010005D13168A1
:100460000220C860304600F0A3F801227A7006E04E
:10047000786840F008007860012000E00220002148
:100480003970BDE8F2832DE9F843044689461546E4
:100490001F4600F08BF9804604F1400630780128B1
:1004A00008BF022038D000F039F832D1002043468E
:1004B0007060422070700022009700F076F8010012
:1004C00028D121682868886222686868506221689B
:1004D000A868C86221680A68286922F440020243B9
:1004E00042F480020A60E968C9F828104FF00062FF
:1004F0004946FFF710FF009743460122082100F00C
:1005000055F8010006D122680821D16001217170DF
:1005100000E0022000213170BDE8F283012131703A
:100520007178012970472DE9FC4104468846174639
:1005300004F1400600F03AF903463078012808BF7C
:1005400002202AD0FFF7EAFF23D1002000227060AA
:1005500082207070B06800F027F80546D0B9216895
:100560000A68786822F0080202430A60786808285E
:1005700009D12268396811632068102100F00FF852
:1005800041F4801101604FF040624146FFF7C3FE25
:1005900000E00225002030702846BDE8F681C160E9
:1005A000206801687047A8680090202120463BE041
:1005B000F8B5044604F1400600F0F8F805467078F6
:1005C000002781072AD5377000F02AF80BD502687A
:1005D00022F004020260E06B00F0F0F818B17068DD
:1005E00040F00400706020682B460122016841F051
:1005F00002010160B06800900221FFF7D7FF0700F9
:1006000008D1216802202B460022C860B068FFF79D
:10061000CBFF0746380004BF012070703846F2BD9A
:10062000206801684A0770472DE9F04105460E46EB
:1006300090461F46069C2868816816EA010018BF8C
:100640000120404511D014F1010FF4D024B100F085
:10065000ADF8C01B8442EED2042085F84100686CDE
:1006600040F001006864012000E00020BDE8F08156
:10067000F8B54B6A002B18BFB2F1406F03D08C6AFB
:100680000368641E1C618C69002C42D00B6A0668EA
:1006900013B38C68F461CD6A0B6B4C698F69D1F828
:1006A00000C01D434B6B1D434B6A1D430B6945EA5C
:1006B00084451D430B6A1D43CB6943B1CC68254378
:1006C0001D433D434CEA0505154375613DE03D433F
:1006D0004CEA05052A431AE0CF6A0B6BD1F800C03B
:1006E0001F434B6B1F434B6A1F434B6947EA8347CA
:1006F000CB6943B1CD682F431F433C434CEA04040C
:100700001443746121E03C434CEA040422437261C7
:10071000F1BD0B6A0BB305688C68EC61CE6A0B6B9C
:100720004C698F691E434B6B1E434B6A1E430B691A
:1007300046EA84461E430B6A1E43CB694BB1CC6824
:1007400026431E433E4316436E61B2F1406F19D1FA
:10075000F1BD3E4332436A61F1BDCB69B3B1CD6AAD
:100760000C6B4E6925434C6B25434C6A2543CC6882
:1007700045EA864525432B4304681343B2F1406F95
:10078000636111D0006849688161F1BD4B6A5BB15A
:10079000CD6A0C6B006825434C6B496925432B439C
:1007A00043EA81431A434261F1BD70470148406802
:1007B000704700BF3000002070470000F8B50646C3
:1007C00006F13404656AFFF7F1FF074660780228F6
:1007D00005D080210120216200212170F2BD306806
:1007E000016821F0160101603068426922F0800240
:1007F0004261E168002904BF6069002804D03068C4
:10080000016821F008010160306802685208520056
:10081000026030680168CB070BD5FFF7C7FFC01B2C
:100820000628F6D32020206200202070032060706C
:10083000F2BDA06A3F2181400020A9602070012004
:1008400060700020F2BD000038B5040001D1012025
:1008500032BD04F14005687820B900212046297096
:1008600000F0D8FA2421697000F05AF86068226814
:1008700020F0706010612068816821F4004181607F
:10088000E068012805D1A168226841F40041916027
:1008900004E0A068216840F404408860E268022A0D
:1008A00003D121684FF4006048602068426842F03C
:1008B000007242F4004242602068C16821F40041A5
:1008C000C1602269606921680243A06942EA00228E
:1008D000CA60E269206A02432068026020680168F9
:1008E00041F0010101600020686020206870002054
:1008F0002063A87032BD38B5040001D1012032BD9B
:1009000004F140052420687000F00AF8204600F049
:1009100082FA0020686068702063A870287032BD79
:10092000206801684908490001607047CDF80090CF
:100930003B4600228021304600F0B7B9728D4FF05F
:1009400000733285D2B2009070472DE9FE4F00F05F
:100950000FF959D10C9D002D1CBF0D9F002F4CD0BD
:100960002078012850D001212170FFF71FFF00F0EF
:1009700065F8002843D1212000F003F900F022F9A6
:1009800040B16068042802D10021217035E00021C7
:10099000217034E0708DFF25B0F5807F1BD300F00F
:1009A00001F900F047F80E9F4A463946304600F0FC
:1009B0009CF900281ED100F02EF815D1708D00286A
:1009C00012D0FFF7B3FF002819D100F020F807D3A9
:1009D00000F0E8F806E0728D0020FFF7B0FFE0E7D6
:1009E00000F045F800F026F8708D0028DCD100F00A
:1009F000ADF830B16168042901D1012005E0032080
:100A000003E000F025F800E00220BDE8FE8F708DC5
:100A1000B0F5807F7047706A411C71623168007860
:100A20008862708D421E7285318D481E308580B27D
:100A3000002870474146304600F0D5B98146192359
:100A4000CDF8009001224FF40041304600F02DB95E
:100A500032682020D0613168DFF814024B6803400F
:100A600020204B6060700020A07020707047728D55
:100A700000214FF000733285D2B2009170472DE90A
:100A8000FE4F00F075F85ED10C9D002D1CBF0D9F30
:100A9000002F51D02078012855D001212170FFF777
:100AA00085FEFFF7CBFF002848D1222000F069F82F
:100AB00000F0AEF840B16068042802D10021217036
:100AC0003AE00021217039E0718DFF25DFF8F00058
:100AD000B1F5807F20D335854FF080730090FF22E1
:100AE000FFF7A8FF0E9FCDF800903B46002204219F
:100AF000FFF721FF002821D100F02DF8728590B971
:100B0000708D80B1FFF712FF002817D1FFF77FFF2C
:100B100005D300F047F804E0FFF710FFE0E7FFF728
:100B2000A6FFFFF787FF708D0028DCD100F00EF8DC
:100B300030B16168042901D1012005E0032003E000
:100B4000FFF786FF00E00220BDE8FE8F4A463946E7
:100B5000304600F0E3B8706A411C716231684A6A3D
:100B60000270308D401E3085718D80B24A1E7047F4
:100B7000064606F140046078884692469B46202847
:100B800070475B4660704020A07000206060524655
:100B900075624146778570630E9800903046CDF8B7
:100BA000049070473585002100914FF08073FF223B
:100BB00070473146204600F016B990F84100704762
:100BC000002400802DE9FC4100F047F84FF08073CD
:100BD000EAB2FFF7EFFF324600F054F818B1606C4C
:100BE000042812D107E0012D07D000F047F820B10A
:100BF000616C042909D1012008E02068FFB2434656
:100C00000022802100F036F800B10320BDE8F68113
:100C10002DE9FC4100F021F80023EAB2FFF7CAFFFA
:100C2000324600F02FF818B1606C042812D107E0AA
:100C3000012D07D000F022F820B1616C042909D100
:100C4000012008E02068FFB243460022402100F066
:100C500011F800B10320BDE8F6810446DFF8A801D1
:100C600017461D460090DDF82080099E7047000061
:100C700000E800FE87622046009616E02068390AE8
:100C800032468162414620462FE081B0006881698A
:100C90008A0744BF002282628169CA0703D482693D
:100CA00042F00102826101B070472DE9F041054632
:100CB0000E4690461C46069F286881693140B14225
:100CC0000CBF0120002040450CD114F1010FF3D0DE
:100CD00024B1FFF76BFDC01B8442EDD200F07BF81E
:100CE000032000E00020BDE8F08170B505460C4609
:100CF0001646286881698A070ED400F025F808B1E5
:100D0000012070BD14F1010FF3D024B1FFF74EFDA7
:100D1000801B8442EDD21BE0002070BD70B50546FB
:100D20000C461646286881698A060BD400F00CF838
:100D300030B924B1FFF73AFD801B8442F2D207E0BC
:100D4000012070BD002070BD3246214628460FE0CC
:100D500000F004F882700270032070BD05F14000BD
:100D60002022416841F0200141604270002270471A
:100D700070B505460C46286816468169CA0610D526
:100D80002868826991060ED414F1010FF8D024B1BD
:100D9000FFF70CFD801B8442F2D200F01CF8032008
:100DA00070BD002070BD1021C16129682020C8617C
:100DB0002846FFF76AFF2968144800F006F8042166
:100DC000416000F00AF8012070BD4A68024005F158
:100DD00040004A60704705F1400020214170002129
:100DE00081700170704770B50068049C084EC1F3B3
:100DF000090146EA54564568B543294341EA024190
:100E000019432143416070BD0020008000E800FECE
:100E1000FF63FF03704770472DE9FC41044600253E
:100E2000C4B12078DFF86864C10751D5B16801F01A
:100E30000C01042907D0B06800F00C0008280BD181
:100E40007168480208D53268900341D5606800286F
:100E500040F0CF8001206CE16068B0F5803F04D1A4
:100E6000306840F4803030601DE040B9316821F4D2
:100E700080313160326822F48022326013E0B0F5B4
:100E8000A02F08D1306840F480203060316841F4F0
:100E90008031316007E0326822F48032326033689A
:100EA00023F480233360606868B1FFF77FFC074656
:100EB00031688A0300F19D80FFF778FCC01B65282C
:100EC000F6D3032035E1FFF771FC07463068810354
:100ED00040F18F80FFF76AFCC01B6528F6D3F0E76E
:100EE000FFF764FCC01B022840F2B080E9E7E0682D
:100EF00080B1316841F001013160FFF757FC0746CE
:100F00003268900700F1CC80FFF750FCC01B02282C
:100F1000F6D9D6E73068400840003060FFF746FC5D
:100F2000074631688A0766D5FFF740FCC01B0228D8
:100F3000F7D9C6E7706F400840007067FFF736FCCE
:100F40000746716F880775D5FFF730FCC01B022874
:100F5000F7D9B6E708B9306F09E00528306F06D138
:100F600040F004003067316F41F0010105E04008B6
:100F700040003067316F21F004013167A06841F211
:100F8000893768B1FFF712FC8046316F880700F19E
:100F90009880FFF70BFCA0EB0800B842F5D390E770
:100FA000FFF704FC8046306F810740F18A80FFF72D
:100FB000FDFBA0EB0800B842F5D382E7FFF7F6FB94
:100FC000401B022840F294807BE7FFF7EFFB001BF9
:100FD000022840F2A98074E7FFF7E8FB0446316875
:100FE0008A0140F1A580FFF7E1FB001B0228F6D93A
:100FF00067E7207881071BD5B16811F00C0F09D085
:10100000B06800F00C0008287FF471AF71684802E6
:101010003FF56DAF3068820703D5E16801297FF4A1
:1010200019AF3068226920F0F80040EAC200306051
:10103000217808070ED5606900283FF47BAF716FF7
:1010400041F001017167FFF7B1FB0746706F81073F
:101050007FF546AF21784A0738D5306CC10009D4F6
:10106000316C012541F080513164306C00F08050CA
:1010700000900099DFF824723868C20518D43968E6
:1010800041F480713960FFF791FB80463868C205F2
:101090000ED4FFF78BFBA0EB08006528F6D310E712
:1010A0003168206921F0F80141EAC0013160BFE7F1
:1010B000A06801287FF44EAF306F40F00100306728
:1010C0005CE71DB1316C21F080513164A06978B3C7
:1010D000B16801F00C0108293FF4BCAE0228306869
:1010E00020F0807030607FF477AFFFF75FFB05463C
:1010F00031688A013FF562AFE269206AA16A024362
:10110000606A42EA8012E06A4908491E42EA0142E6
:1011100042EA006242F000527260316841F0807130
:101120003160FFF743FB0446306882017FF54DAF25
:101130000020BDE8F6812DE9F8430400884674D00C
:10114000574E306800F00F00404502D200F06FF8B3
:101150006BD120684E4D810712D5400703D5A86892
:1011600040F4E050A86021780A0703D5A86840F44D
:101170006040A860A968A06821F0F0010143A9605F
:101180002078C10749D56068012802D129688A03FF
:1011900003E0022803D12A68910103D445E02968BD
:1011A0008B0742D5AA6841F28939920840EA820049
:1011B000A860FFF7FBFA0746A868616800F00C001A
:1011C000B0EB810F29D0FFF7F1FAC01B4845F3D3EC
:1011D000032020E02078410705D5A968E06821F4C4
:1011E000E0510143A9602078010706D5A96820696C
:1011F00021F4604141EAC001A96000F022F8AA6828
:101200002849C2F30312895C224AC84010600F20AB
:1012100000F04EF80020BDE8F283306800F00F00C7
:101220008045D7D200F003F8D4D00120F3E731682D
:10123000090948EA01113160326802F00F024245A3
:10124000704718B5184C606800F00C00042802D0F4
:10125000082802D019E0154812BD00232268216831
:1012600048022068C0F3881002F03F024CBF0F49CB
:101270000949A1FB000100F03BF82168C1F30141DD
:10128000491C4900B0FBF1F012BD034812BD00003B
:10129000003802403C0000200024F40000700040B0
:1012A000003C0240DC2F00080438024040787D01F9
:1012B00038B50D4D044629784FF47A700B4AB0FBCF
:1012C000F1F11068B0FBF1F000F07BF950B9102C8F
:1012D00008D2002221464FF0FF3000F03DF9AC600B
:1012E000002032BD012032BD300000203C00002033
:1012F000B3BBD9B1B2F5803F7DD2022A1ED98C464C
:10130000B1FBF2F102FB11C31B0443EA1043B3FB30
:10131000F2FC02FB1C3380B240EA0343B3FBF2F061
:1013200002FB103240EA0C4000237047022A05D924
:101330008446B0FBF2F002FB10C270474AB105D1FF
:1013400000F0010249085FEA3000704700220023E4
:10135000704700F059B90B000200002100207047CF
:10136000904271EB030CF6D3B3F5803F2FD2F0B56A
:10137000B3FA83F7B1FA81F4A7F10F0E3D1B534086
:10138000CEF1200602FA0EF2F3415340B5F10F07F9
:1013900046D80F3C2C444140C4F12006A040F14106
:1013A0004140B1FBF3F603FB1611A2FB0645001BFF
:1013B000A94102D2761E8018594180EA010221FA21
:1013C0000EF362FA0EF200215A403046F0BD30B4FE
:1013D000B1FBF3FC03FB1C11A2FB0C45001BA94154
:1013E00003D2ACF1010C8018594130BC02460B46C7
:1013F000604600217047B2F1807F65D3F0B5B2FA44
:1014000082F7B1FA81F4C7F10F063D1B22FA06F309
:1014100007F1110EF24120355A40B5F10F07B8D946
:101420004140C4F12006A040F1414140B1FBF3FC32
:1014300003FB1C11A2FB0C45001BA94103D2BCF10C
:10144000010C801859410F2F12D30F3FC90341EAF5
:101450005041B1FBF3F603FB1611A2FB0645D4EB9A
:10146000C030A94102D2761E8018594146EACC3CD0
:1014700007B34140C7F12006B840F1414140B1FBFC
:10148000F3F603FB1611A2FB0645001BA94102D28D
:10149000761E8018594180EA010221FA0EF3C7F145
:1014A000200462FA0EF20CFA07F05A402CFA04F10A
:1014B0003043F0BD80EA010221FA0EF3002162FA06
:1014C0000EF260465A40F0BD8C46B1FBF2F102FBD1
:1014D00011C31B0243EA1063B3FBF2FC02FB1C3393
:1014E0001B024CEA002043EA1063B3FBF2FC02FB50
:1014F0001C331B024CEA002043EA1063B3FBF2FCEE
:1015000002FB1C331B024CEA002043EA1063B3FBCE
:10151000F2FC02FB1C324CEA002000237047000062
:101520000901020081B002D43048815405E0304AFC
:1015300000F00F00104400F8041C01B070472D4A61
:101540004FF6FF011368000200F4E0600B401843FF
:10155000294908431060704738B5264B1C68C4F30E
:101560000223C3F10704052C28BF04241D1D072DE9
:1015700034BF0023DB1E012505FA04F4641E21405C
:10158000994005FA03F35B1E1A401143BDE834404D
:10159000C6E7010008D4012200F01F0002FA00F0A3
:1015A000164A490942F821007047010008D4012277
:1015B00000F01F0002FA00F0114A490942F8210028
:1015C0007047401EB0F1807F10B501D3012010BDDF
:1015D0000C4C0F2160604FF0FF30FFF7A1FF00229D
:1015E0000020A2600722226010BD000000E400E09D
:1015F00018ED00E00CED00E00000FA0500E100E06D
:1016000080E100E010E000E0704700002DE9FC47B9
:10161000064600253078A846DFF85C74C1070AD575
:10162000B96821F40001B960BA68706B0243BA600E
:10163000706B00B901253168DFF8404408030ED50E
:10164000A268F06B22F440120243A260F06BB0F586
:10165000801F08BF012502D008B94FF0010830688B
:10166000C1020ED5A168306C21F440010143A16094
:10167000306CB0F5800F08BF012502D008B94FF0DB
:1016800001083068C10148BF0125800632D5386C99
:10169000DFF8EC9340F080503864396C01F08051F1
:1016A00000910098D9F8001041F48071C9F8001039
:1016B000FFF77CF88246D9F80020D00500F1EB80D6
:1016C000FFF774F8A0EB0A006528F4D30320BCE10F
:1016D000FFF76CF8A0EB0A004845C0F0F980F5E789
:1016E000B86820F4F810B860396F306BC0F30B00A5
:1016F000014339673178CA0607D5A06820F08070A9
:10170000A060A168B06B0143A1603068410405D5B9
:10171000E168706E21F440310143E16030680104FA
:1017200005D5E168B06E21F440210143E1603068E5
:10173000C10305D5E168F06E21F440110143E16079
:101740003068810305D5E168306F21F44001014321
:10175000E1603078410605D5E168706C890840EA9F
:101760008101E1603078010605D5E168B06C21F0B7
:101770000C010143E1603068C10505D5E168F06CFA
:1017800021F030010143E1603068810505D5E16851
:10179000306D21F0C0010143E1603068410505D59D
:1017A000E168706D21F440710143E160306801052A
:1017B00005D5E168B06D21F440610143E160306816
:1017C000C10405D5E168F06D21F440510143E160A9
:1017D0003068810405D5E168306E21F44041014351
:1017E000E1603068410205D5E168B06F21F08061A9
:1017F0000143E160306881020BD5E168F06F21F0B0
:1018000000610143E160F06FB0F1006F08BF4FF07D
:1018100001083068010748BF4FF00108400305D5B3
:10182000E168706F21F040710143E16030680102AE
:1018300006D5E168D6F8800021F080510143E160CF
:1018400025B93068B0F1007F40F0A880396821F0F8
:1018500080613960FEF7AAFF05463A6810014BD552
:10186000FEF7A4FF401B6528F7D32FE7FEF79EFF86
:10187000401B6528C0F08E8028E7FEF797FF401BCD
:101880006528C0F0958021E7FEF790FF001B6528D2
:10189000C0F0D6801AE7386F10F440701EBF316B6D
:1018A00001F44071884217D0386F3A6F42F48032A9
:1018B0003A67396F20F4407021F480313967386716
:1018C000386FC10708D5FEF771FF824641F28939AA
:1018D000386F81077FF5FCAE316B01F44072B2F5D1
:1018E000407F7FF4FDAEBB68DFF89801014023F430
:1018F000F8131943B960F7E63178C8070FD5706B54
:1019000068B920682168726800F4403040EA8210AB
:1019100001F070610843B16840EA017020603068EE
:10192000020303D5F16BB1F5801F05D0C00211D5BC
:10193000306CB0F5800F0DD1206821687268F368B3
:1019400000F08FF82060A068716A4009491E41EAE2
:101950004010A0603068C20106D520682168336954
:10196000726800F074F82060306881010BD530692E
:101970007168B268000440EA8110F16840EA0160D1
:1019800040EA02702060386840F080603860FEF7FE
:101990000DFF054639680A017FF568AFB8F1000F01
:1019A00052D0386820F080503860FEF7FFFE0546C0
:1019B00039688A003FF561AF3068020301D5F16BE9
:1019C00019B1C00210D5306C70B960686168726975
:1019D000B36900F046F86060A068B16A20F4F8507E
:1019E000491E40EA0120A060306881020AD5F16FEB
:1019F000B1F1006F06D160686168336A726900F006
:101A000026F860603078010713D5606861687269F4
:101A100001F4403141EA821100F070600843F1693D
:101A200040EA01706060A268F06A22F4403202432A
:101A3000A260386840F080503860FEF7B7FE044678
:101A400039688A007FF520AF0020BDE8F6871B04C7
:101A500043EA821300F0706001F0E041184308434C
:101A6000704700F4403040EA821001F0E04140EA63
:101A70000360084370470000003802408438024089
:101A800000700040FFFCFF0F70B586B0CA48416986
:101A90004FF48054C94DCA4E41F0806141614269A2
:101AA00002F0806200F06DF841F010010160026800
:101AB00002F0100200F065F841F040010160026898
:101AC00002F0400200F05DF841F4807101600268AC
:101AD00002F4807200F055F841F400710160026870
:101AE00002F4007200F04DF8102241F480610160B0
:101AF000006800F4806005900599009202200021A2
:101B0000019002910E22039069460492AD4800F0C4
:101B10006DF909200222049069460094AA480192B6
:101B200000F064F94FF4464000F02FF8284600F02A
:101B30005DF94EF6FF7000F028F8A44800F056F961
:101B4000F72000F022F8304600F050F90120009410
:101B500001906946284600F049F9082101200091CA
:101B600069460190304600F041F90122214628469D
:101B700000F01DFA01220821304600F018FA06B0E4
:101B800070BD0592059901687047022100900E22F0
:101B900001916946049270470020002138B58C4CB1
:101BA000AEB060604FF48A72A0608A4DE060206140
:101BB000282060610920A0613520E0610B202062AF
:101BC00040F21B10A06240F21520606240F21D102E
:101BD000206340F2352000910291E06204F134006C
:101BE0000180817002210491FF217B4805912060D2
:101BF0004FF4F0700CA90392019000228A704FF408
:101C000080610A904FF488700692ADF8302005226A
:101C1000079108210B9005200892C0220D914FF4E6
:101C2000803114900DA8099512921891FFF7EEFCDF
:101C3000204600F0DDF900B1FEE7012269462046AA
:101C400000F04FFA00B1FEE740F2DC5000F0F4FA89
:101C500062480122284469460990204600F041FA72
:101C600000B1FEE72FB030BD1CB500F0F9FA00B1AD
:101C7000FEE75B4C702021688847616870208847C8
:101C8000512800D0FEE7702000F031FCFFF784FF00
:101C9000702000F02DFC0028FAD06A460DF10201F8
:101CA000702000F043FCBDF802003C38A128EFD2C0
:101CB000BDF80000A0F11E01A12905D3A0F5967082
:101CC000A128E5D2022016BD012016BD10B5454C55
:101CD0000022206C20F400002064216A482041F496
:101CE00000012162236A002123F400032362FFF72D
:101CF00033FC002200214920FFF72EFC4820FFF78B
:101D000054FC4920FFF751FC206940F0800020611D
:101D1000216921F080012161206B20F08000206387
:101D2000616C21F080616164606A40F08060606293
:101D3000616A21F0806161622068002120F080509A
:101D4000206029484160016821F07041016002680B
:101D500042F000520260206940F040002061216999
:101D600041F480712161206940F400702061216993
:101D700041F480612161206920F0400020612169E7
:101D800021F480712161206920F4007020612169B3
:101D900021F480612161206B20F040002063216BE1
:101DA00021F480712163206B20F400702063216B8B
:101DB00021F48061216310BD3038024000200240D0
:101DC0000028024000100240001802400024024097
:101DD000400000200000F09000680140000B04006B
:101DE0000000002000380240883802402DE9F84FFA
:101DF0004FF0000E714A724BDFF8C8814FF00F09A7
:101E000006468A46DAF80040012101FA0EF10C403C
:101E10008C4240F0C480DAF804504FEA8E00022D64
:101E200018BF122D12D14FEADE0506EB850C00F02B
:101E30001C0509FA05FBDCF8207027EA0B07DAF825
:101E400010B00BFA05F53D43CCF8205037689AF8EE
:101E500004B04FEA4E0C032505FA0CF5ED432F4074
:101E60000BF0030B0BFA0CFB4BEA07073760DAF8B1
:101E70000470012F18BF022F03D0112F18BF122F8B
:101E800013D1B768DAF80CB02F400BFA0CFB4BEA11
:101E90000707B760776827EA0101DAF80470C7F32B
:101EA000001707FA0EF739437160F1680D40DAF850
:101EB000081001FA0CF12943F160DAF80410C900A6
:101EC0006DD5D8F8001000F00C0009FA00F741F4C5
:101ED0008041C8F80010D8F8005005F480450095FE
:101EE00000994FEA9E0153F8215025EA0707364D25
:101EF000AE4208BF00252CD0344DAE4208BF0125AC
:101F000027D0334DAE4208BF022522D0314DAE421C
:101F100008BF03251DD0304DAE4208BF042518D0A0
:101F20002E4DAE4208BF052513D02D4DAE4208BF41
:101F300006250ED02B4DAE4208BF072509D02A4DED
:101F4000AE4208BF082504D0284DAE420CBF09257B
:101F50000A2505FA00F0384343F821001168DAF841
:101F60000450E0430140ED0348BF21431160516834
:101F7000DAF804500140AD0348BF21435160916835
:101F8000DAF804500140ED0248BF21439160D16866
:101F90000140DAF80400800248BF2143D1600EF10D
:101FA000010EBEF10F0F7FF62DAFBDE8F18F81B0AE
:101FB00002B90904816101B070470000003C014092
:101FC000083801404438024000000240000402404A
:101FD00000080240000C02400010024000140240C1
:101FE00000180240001C0240002002400024024071
:101FF000F8B5040001D10120F2BD04F1A005687814
:1020000020B9002120462970FFF73EFD02216970AA
:102010002068816921F07041816121688A69636863
:10202000A0680343E0680343206903431A438A61BD
:102030002168DFF8FC018A6802408A6021688A68AA
:10204000A669636946EA034632438A602168CA6822
:102050000240CA602168CA68266AE36946EA034604
:102060003243CA6021680A6902400A6121680A692C
:10207000A66A636A46EA034632430A6121684A69EE
:102080001040486120684169236BE26A43EA0243D9
:102090001943416104F13400236841788278DE6A93
:1020A00006F07F46DE622368120442EA0121DF6AFD
:1020B000007801433943D9622068416B41F0040143
:1020C00041632068426B42F00202426320688169EA
:1020D00041F00101816100206860012068700020EA
:1020E000F2BDF8B500F012F801D10220F2BD00F007
:1020F00015F800F007F8226801210020516269708C
:102100002870F2BD3A463146204613E0044604F1F9
:10211000A00528780E461746012870473420012173
:1021200078432970022134226970314620443830C6
:1021300000F09ABAF0B503684C68002703EBC212AE
:10214000D868C0F30B4004198432506800F4704022
:1021500050600D68D868C0F30B4045196D1C45EA06
:1021600004445460C868DC689568C4F30A04201805
:1021700005F4704595608C68DB68C3F30A031C198D
:10218000641C44EA004090601069C008C0001061FF
:102190000B69136101F1300358789C788D69966959
:1021A00097611B7843EA002040EA044040EA05605A
:1021B00090615069000A000250614B695361D36914
:1021C0001C480340D361CC69086A0443D461906A17
:1021D00097624B6A9362086908B904230EE00128EC
:1021E00008BF03230AD0042818BF022803D00328FD
:1021F00018BF072801D1022300E00123D06A00F0B4
:10220000E020D0628C6A4D6808685C432D1A6B43ED
:10221000DB1C43EA0443D362106BC00AC0021063A4
:10222000C96A1163106840F001001060F0BD000041
:1022300000F800F0F8F8FFFF38B50446FEF7B6FAEC
:1022400014F1010F054602D0044801786418FEF726
:10225000ADFA401BA042FAD331BD00BF30000020D0
:102260007CB5914C914820602046FEF701F800288B
:102270005BD100F03DFA8E4D0020E8612862686273
:102280006861E862286368634FF40050E8600020EA
:10229000A86401206864102028644FF48000E8647A
:1022A000012060600420A0601020E0601720206101
:1022B0004FF4A06060610020A061E06120622046D0
:1022C000FDF782FF002830D14FF4807041F288364C
:1022D000A8616620286000206862324600F027F876
:1022E00018BB99203246286000F021F8E8B9204652
:1022F00000F07BF8C8B9204600F01DF8A8B94FF4EB
:1023000040706A46A861EB2028604FF44060E861A5
:102310004FF0407068620A206861002001902946F1
:1023200000902046FEF7FFF800B1012076BD294657
:102330002046FDF7B6BF8521002278B504468FB050
:1023400001914FF080710A914FF480700121079044
:10235000089241F288350992204606920B9101A914
:102360000C920D920E922A46FDF79BFF002839D160
:102370002A4669462046FEF729F8002832D14C4EFD
:102380004FF44070B06106203060002070622A4631
:102390003146FFF7CDFF28BB02202B46B06306F184
:1023A0003802F063052030604FF0407070623146B3
:1023B0002046FEF768F8A8B99DF80010812001902A
:1023C0002A46204601F00F0141F0A0018DF80010CF
:1023D00001A9FDF766FF28B92A4669462046FDF7A0
:1023E0009DFF00B1012010B070BD78B595B04FF4DD
:1023F000807007901020119000214FF48000099107
:10240000069100220C914FF080740D91264D0E9193
:1024100041F288361391652114900120019101A9A0
:10242000089232460B9028460A94FDF73AFF00289E
:1024300037D1324669462846FDF7C8FF002830D11B
:1024400006200021019032460A9101A92846FDF795
:1024500028FF30BB022001220F9033461090052048
:1024600012920FAA019001A90A942846FEF70BF8D0
:10247000B8B96120012101909DF800000B9132460E
:1024800001A900F03F0040F040008DF80000284610
:10249000FDF707FF28B9324669462846FDF73EFF9B
:1024A00000B1012016B070BD38010020001000A05E
:1024B000E800002080B5C82000F003FBBDE8014023
:1024C000C5E0704738B5054600208DF800000324AC
:1024D00000F0BDF8A821E8B200F0D0FA00F092F8C0
:1024E000512801D0641EF5D19DF8000032BDA0E056
:1024F00080B50021C0B28DF80010022100F0BEFAB4
:1025000000F080F800F00F008DF800009DF800103A
:102510000629A4BF00208DF800009DF80010514846
:102520004170002181709DF8000002BD2DE9FC473B
:1025300000234C4D8DF8003095F8028095F801C0CD
:10254000002600270024E0455AD2B8F1090F37D8F9
:10255000DFE808F0050A0F14191E23282D32042382
:102560000326062705242BE00A2309260C270B2423
:1025700026E010230F261227112421E0162315260A
:10258000182717241CE01C231B261E271D2417E0D8
:10259000222321262427232412E0282327262A2742
:1025A00029240DE02E232D2630272F2408E0342364
:1025B00033263627352403E03A2339263C273B24AB
:1025C0008946824690461946C0B200F057FA00F09C
:1025D00038F800F01CF800F01FF83946A880A9F878
:1025E000000000F015F800F00DF8214600F00FF89B
:1025F00000F012F8A880A8F80000A878401CA87085
:10260000BDE8F3878DF800009DF800007047A880B2
:102610005FFA8AF000F032BA8DF80000A8889DF8C1
:102620000010090201F4706108437047012201E0C3
:1026300000BF0022A421C0B200F011BA00207047F0
:1026400070478DF800009DF800003146704710B5C6
:10265000044C207818B900F0FFF90121217010BD59
:1026600000000000D0010020103A07D330B4B1E8D8
:102670003810103AA0E83810F9D230BC530724BF04
:10268000B1E80810A0E8081044BF51F8043B40F836
:10269000043BD20724BF31F8022B20F8022B44BFA1
:1026A0000B7803707047121F17D35B0009D151F8E4
:1026B000043B20F8023B1B0C121F20F8023BF6D211
:1026C0000BE051F8043B00F8013B1B0A20F8023BE9
:1026D0001B0C121F00F8013BF3D238BF121D521E13
:1026E00024BF11F8013B00F8013BF8D87047000007
:1026F00010B586B06348016A634C41F00201016283
:10270000026A02F0020200F0D6F841F00201016014
:10271000026822F002020260836943F002038361CF
:10272000816901F002010591059A816941F0080172
:102730008161826902F0080205920599816940224F
:1027400041F010018161806900F010000590059949
:102750000A2000920490022101200191029020465B
:10276000039100F0A5F804200921009000220491B3
:10277000694602922046FFF739FB4FF400600921B9
:102780000090424C049169462046FFF72FFB4FF41E
:10279000805000F089F80420092100903C4800F0A6
:1027A00086F84FF4005000F07FF806B010BD80B5F9
:1027B00086B03848816841F001018160826802F08A
:1027C000010200F078F841F004010160026802F0B3
:1027D000040200F070F841F008010160026802F0A4
:1027E000080200F068F841F010010160026802F090
:1027F000100200F060F841F020010160026802F070
:10280000200200F058F841F040010160026802F037
:10281000400200F050F8022241F08001016000689F
:1028200000F08000059005990120019202900C2093
:10283000082104900091694603921748FFF7D6FAE1
:102840004CF20372694600921048FFF7CFFA4FF638
:102850008370694600900E48FFF7C8FA4FF63F01B3
:102860000E48009100F024F848F2331069460090B9
:102870000B48FFF7BBFA28210A48009100F018F82E
:1028800007B000BD1838024000040240000C0240AE
:10289000001002403038024000080240001402409C
:1028A00000180240001C02400921009020460491BB
:1028B0006946FFF79BBA05920599016870470000C9
:1028C00070B5744986B0744C88424FF480752069A5
:1028D0003BD140F080008022206121696F4E01F0E1
:1028E000800105910598122100920020019102902B
:1028F000022104200391049069463046FFF776FADE
:10290000009569463046FFF771FA206A002240F4CC
:1029100000002062216A01F40001059105982068F9
:1029200040F4000020602168482021F4000121606B
:102930000F21FEF711FE4820FEF72BFE00220F218B
:102940004920FEF709FE49203BE040F002002061EB
:10295000216901F0020105910598002100951220DE
:102960000291019002200421039004914C4D69468C
:102970002846FFF73BFA4FF400706946009028465E
:10298000FFF734FA216A002241F400112162206A23
:1029900000F4001005900599216841F400112160B0
:1029A00020680F2120F4001020601F20FEF7D4FDC6
:1029B0001F20FEF7EEFD00220F212020FEF7CCFDA8
:1029C0002020FEF7E6FD06B070BD10B50446FEF708
:1029D000F4F8C0B92F4884420CBF32483248206016
:1029E000324860600020A0600120E060002020618B
:1029F0006061E06120622046FFF762FF2046BDE88B
:102A00001040FDF721BF10BD7FB500F011F8FEF7B3
:102A100036F804E07FB500F00BF8FDF796FF0600EE
:102A200003D02946204600F00FF8304604B070BDB0
:102A300004460D46089909984FF47A760190009162
:102A4000294602962046704710B50446FDF753FF0D
:102A50002046BDE81040B8E700BF0E48B5E707B50F
:102A600000F004F80B48FFF7D5FF07BD0A46012127
:102A7000019102AB00930146012370471FB500F09E
:102A800017F804480094FFF7BFFF9DF8080004B052
:102A900010BD00008401002020380240001C0240CC
:102AA00000040240005C0040005400403227914086
:102AB0000A4600218DF80810012302AC014601935B
:102AC0007047FFF7B9BB00002DE9F04391B000F06B
:102AD000BCF8584C0020206000F0B7F8564E306823
:102AE00040F4003000F0B0F800213167BFF34F8FA1
:102AF000F16E43F6E078C1F34E32C1F3C90308EA40
:102B0000421747EA837020611846431E0028F8D117
:102B10001046421E0028F0D1BFF34F8F306840F4BA
:102B2000803000F091F800F095F801210220059125
:102B30004FF480010B9019200C914FF4C8710D9047
:102B400002200E914FF480320F900821069205A8C2
:102B50001091FEF761F900B1FEE700F08FF800B1C7
:102B6000FEE70F20022100904FF4A05001914FF496
:102B70008051002203900491062102926846FEF7DC
:102B8000DAFA00B1FEE7FFF76FF80128DFF8AC9042
:102B900018D14FF010402A4F00257860FFF796F8C3
:102BA00000F0A6F802467868484509D1EB006D1C94
:102BB000002003F14043B5F5FF4FC3E90000F5D312
:102BC00022B1FEE7022834D14846E4E700F03DF8A0
:102BD0003068002120F400303060216000F035F8CA
:102BE0003167BFF34F8F316821F480313160BFF31B
:102BF0004F8FF16EC1F34E32C1F3C90308EA42169A
:102C000046EA837060621846431E0028F8D11046D9
:102C1000421E0028F0D100F018F80A4908607868D0
:102C2000011D0A683A60006880F3088810468047F2
:102C3000FEE7FEE750EF00E014ED00E000007890C2
:102C40002800002010E000E03060BFF34F8FBFF39A
:102C50006F8F704780B50748016841F4807101604B
:102C60000320FEF76CFC0F20FEF722FB00F004F8B7
:102C7000002002BD003C0240704700007CB500F01F
:102C800023F840F4803000F01CF806466168C80361
:102C90000CD4FDF78BFD801BA842F7D3032076BD33
:102CA000FDF784FD801BA84206D3F7E7206840F4B7
:102CB000003000F006F8064661688803F0D5002071
:102CC00076BD2060FDF772BD0848074C016840F2F0
:102CD000E93541F080510160006800F080500090BB
:102CE00000992068704700000070004040380240A2
:102CF00018B599B0002004902D4907200C9106903A
:102D0000042108900020079110210D9002220E90BE
:102D100004200F90402010914FF4807111900020FA
:102D200012914FF4006113904FF4805014910021E0
:102D3000059209920A920B9215901691FFF737FDB2
:102D400005A90CA800F040F808B101202EE00120F0
:102D5000102100904FF6FF7402900020019100F0C6
:102D60002CF80120FFF768FA0220102100900122C0
:102D700000F020F8032010210090082200F01AF83B
:102D80004FF4087004210490102201200091019258
:102D9000224602900499039169460CA800F032F88B
:102DA00040F203610CA800F044F800201AB010BDF6
:102DB000400100A000200191029222460390694642
:102DC0000CA800F01FB8000070B504000D4601D13A
:102DD000012070BD04F12C06307820B90021204676
:102DE000717000F03DF8022131702068211D00F063
:102DF00039F862682068294600F06FF801203070C9
:102E0000002070BD38B504460D4694F82C00022809
:102E10000ED0022184F82C102068294600F09EF87C
:102E2000286802280CBF0521012184F82C100020FD
:102E300032BD10B500F00FF807D0022284F82C2024
:102E4000206800F09DF800F001F810BD012084F822
:102E50002C0000207047044694F82C00022870478C
:102E6000704700002DE9F8454A6A0B6ACC698D6904
:102E70004E690F69D1F80CC0D1F808E0D1F8048090
:102E80000968012910D048EA02024EEA02024CEA1F
:102E900002023A43016832432A4322431A43C90BD0
:102EA00042EAC132026015E00168D0F804A04FEA9E
:102EB000DA3A48EACA3821F4F8410C4323431A436A
:102EC0004EEA080E4CEA0E0C47EA0C073E43354327
:102ED000026045600020BDE8F285F8B58B694C6959
:102EE0000D69CE688F68D1F804C009685B1E641E46
:102EF0006D1E761E7F1E491E012AACF1010C8268F0
:102F000010D041EA036302F0704243EA0C1343EA33
:102F1000072343EA063343EA054343EA04531343D2
:102F2000836015E0D0F80CE00EF0704E41EA0E011F
:102F300041EA0C1141EA072707490A4042EA0636EE
:102F400047EA054546EA045445EA03638460C360E2
:102F50000020F2BD00000000FF0F0FFF18B5002396
:102F600000930C684A6814438A68C968521E44EA90
:102F7000421444EA41240094009A0261002012BDE8
:102F8000426942EA41024261002070470E480168EE
:102F900041F4700101600D490A68002042F001020D
:102FA0000A60002288600B680948034009480B60EA
:102FB0004860086820F480200860CA604FF0006113
:102FC000054A11607047000088ED00E000380240BB
:102FD000FFFFF6FE1030002408ED00E000000000C6
:102FE00000000000010203040607080919E050F878
:102FF000042BD30744BFA9F101039A18091F00232A
:10300000042942F8043BF9D25FEA817C134604D5D7
:103010004FF0000CA2F800C09B1CC90744BF002160
:10302000197050F8041B0029E1D17047B52400083D
:10303000C5240008C3240008EF240008F124000878
:103040002D2500082D260008412600083D260008F1
:103050003126000800000000000000900100000080
:1030600000000000100000000024F40010B450F82C
:10307000041B79B10268436802440830DC0744BF8E
:10308000A9F10104E31852F8044B43F8044B091F5B
:10309000F9D1ECE710BC704710B5074979441831F5
:1030A000064C7C44163404E00A68081D1144884725
:1030B0000146A142F8D110BD2C0000004C000000D8
:1030C0004EF68851CEF20001086840F470000860A6
:1030D000BFF34F8FBFF36F8F4FF00070E1EE100A18
:1030E0007047000009FFFFFF98010000400000202A
:1030F0000000000079FFFFFF4000000030FFFFFFED
:10310000000000200000000000F00DF8002801D0B1
:10311000FFF7C2FFAFF300800020AFF30080FFF79E
:10312000D3FC00F002F80120704700F001B8000065
:103130000746384600F002F8FBE7000080B5AFF321
:103140000080024A11001820ABBEFBE726000200F7
:103150007047FEE7FEE7FEE7FEE7704770477047FF
:1031600000F000B802484168027889184160704751
:103170003000002001488047014800478D2F00089B
:1031800085310008AFF30080FFF79AFFFFF7BCFF1F
:10319000FFF7FEBFFFF7FEBFFFF7FEBFFFF7FEBF63
:1031A000FFF7FEBFFFF7FEBFFFF7FEBFFFF7FEBF53
:1031B000FFF7FEBFFFF7FEBFFFF7FEBFFFF7FEBF43
:1031C000FFF7FEBFFFF7FEBFFFF7FEBFFFF7FEBF33
:0200000490F179
:101AC000DFF79EE75DDF5DDF5DDF5DDF5DDF5DDF53
:101AD0003DDF3DDF3DDF3DDF3DDF5DDF5DDF5DDFC6
:101AE0005DDF5DDF5DDF5DDF5DDF5DDF5DDF5DDF16
:101AF0005DDF5DDF5DDF5DDF5DDF5DDF5DDF5DDF06
:101B00005DDF5DDF5DDF5DDF5DDF5DDF5DDF5DDFF5
:101B10005DDF5DDF5DDF5DDF5DDF5DDF5DDF5DDFE5
:101B20005DDF5DDF5DDF5DDF5DDF5DDF5DDF5DDFD5
:101B30005DDF5DDF5DDF5DDF5DDF5DDF5DDF5DDFC5
:101B40005DDF5DDF5DDF5DDF5DDF5DDF5DDF5DDFB5
:101B50005DDF5DDF5DDF5DDF5DDF5DDF5DDF5DDFA5
:101B60005EDF5DDF5DDF5DDF5DDF5DDF5DDF5DDF94
:101B70005DDF5DDF5DDF5DDF5DDF5DDF5DDF5EDF84
:101B80005EDF5EDF5EDF5EDF5EDF5EDF5EDF5EDF6D
:101B90005EDF5EDF5EDF5EDF5EDF7EDF7EDF7EDFFD
:101BA0007EDF7EDF7EDF7EDF7EDF7EDF7EDF7EDF4D
:101BB0007EDF7EDF7EDF5EDF5EDF5EDF5EDF5EDFDD
:101BC0005EDF5EDF7EDFDFF7FFFFFFFFFFFFFFFF70
:101BD000FFFFFFFFFFFFFFFFFFFFFFFFFFFFFFFF15
:101BE000FFFFFFFFFFFFFFFFFFFFFFFFFFFFFFFF05
:101BF000FFFFFFFFFFFFFFFFFFFFFFFFFFFFFFFFF5
:101C0000FFFFFFFFFFFFFFFFFFFFFFFFFFFFFFFFE4
:101E7000FFFFFFFFFFFFFFFF9EEFDCC65AB61A9E73
:101E8000B98D7885577D3775377D377D377D3775C7
:101E9000377537753775377537753775377D377DD2
:101EA000377D577D377D377D377D377D377D577D52
:101EB000577D577D577D577D577D577D577D577D82
:101EC000577D577D577D577D577D577D577D587D71
:101ED000577D577D577D577D587D587D587D587D5E
:101EE000587D587D587D587D587D587D587D587D4A
:101EF000587D587D587D587D587D587D587D587D3A
:101F0000587D587D787D787D787D787D787D787D69
:101F1000787D787D787D787D787D787D787D787D19
:101F2000787D787D787D787D787D787D787D787D09
:101F3000987D987D997D997D997D997D997D997DF3
:101F40009985998599859985998599859985B98581
:101F50009985B985B985B9859985B985B985B985D1
:101F6000B985B985B985B985B985B985B985B98581
:101F7000B985B985B985B985B985D985D985B98531
:101F8000D985B985B9859CAEFFFFFFFFFFFFFFFF35
:101F9000FFFFFFFFFFFFFFFFFFFFFFFFFFFFFFFF51
:101FA000FFFFFFFFFFFFFFFFFFFFFFFFFFFFFFFF41
:101FB000FFFFFFFFFFFFFFFFFFFFFFFFFFFFFFFF31
:101FC000FFFFFFFFFFFFFFFFFFFFFFFFFFFFFFFF21
:10223000FFFFFFFFFCCE1AA65785B664755C3454C9
:10224000344C144C144C344C144C144C354C354C0C
:10225000354C354C354C354C354C354C554C554C36
:10226000554C554C554C554C554C564C564C764C43
:10227000764C764C764C764C764C764C765476543E
:10228000765476549654965496549654965496543E
:10229000965496549654965496549654B654B654AE
:1022A000B654B654B654B654B65CB65CB65CB65CBE
:1022B000B65CB65CD65CD65CD65CD65CD65CD65CCE
:1022C000D65CD75CD75CD75CD75CD75CD75CD75C77
:1022D000D65CD75CD65CD75CD75CD75CD75CD75C68
:1022E000D75CD75CD75CD75CD75CD75CD75CD75C56
:1022F000B75CD75CB75CB75CB75CB75CB754B75436
:10230000B754B754B754B754B754B754B754B75475
:10231000B754B754B754B754B754B754B754B75465
:10232000B754B754B754B754975496549654B654B8
:10233000965496549654965496549654965496544D
:102340009654B654D75CDA8DFFFFFFFFFFFFFFFF07
:10235000FFFFFFFFFFFFFFFFFFFFFFFFFFFFFFFF8D
:10236000FFFFFFFFFFFFFFFFFFFFFFFFFFFFFFFF7D
:10237000FFFFFFFFFFFFFFFFFFFFFFFFFFFFFFFF6D
:10238000FFFFFFFFFFFFFFFFFFFFFFFFFFFFFFFF5D
:1025F000DCCE9895B5643454F34BF44BF44B144C47
:10260000144C154C154C154C154C154C154C354CA3
:10261000354C364C364C364C564C364C564C564C4B
:10262000574C574C774C774C774C774C774C974CB2
:10263000974C97549754975497549754B754B7540A
:10264000B754B754B854B854B85CD85CD85CD85CAC
:10265000D85CD85CD85CD85CF85CF85CF85CF86452
:10266000F864F864186518651865186518651865C4
:10267000386538653865386D386D386D386D386D4A
:10268000386D386D386D386D386D386D386D386D22
:10269000386D386D18651865186518651865186502
:1026A00018651865F864F864F864F85CF85CF85C20
:1026B000F85CD85CD85CD85CD85CD85CD85CD85C5A
:1026C000B854B854B754B754B754B75497549754F0
:1026D000975497549754974C974C774C774C774C2A
:1026E000774C574C574C564C564C564C564C564CB7
:1026F000364C364C364C364C354C154C154C154C2E
:10270000154C765417655BAEFFFFFFFFFFFFFFFF21
:10271000FFFFFFFFFFFFFFFFFFFFFFFFFFFFFFFFC9
:10272000FFFFFFFFFFFFFFFFFFFFFFFFFFFFFFFFB9
:10273000FFFFFFFFFFFFFFFFFFFFFFFFFFFFFFFFA9
:10274000FFFFFFFFFFFFFFFFFFFFFFFFFFFFFFFF99
:1029A000FFFFFFFFFFFFFFFFFFFFFFFF5DDFB89DA2
:1029B0007464D24BD343F44BF44BF44BF44BF443D9
:1029C000F443F543F54B154C154C154C154C154C73
:1029D000364C364C364C364C364C364C564C564CA7
:1029E000574C574C574C774C774C774C774C774C2F
:1029F000974C974C9754975497549854B854B8544C
:102A0000B854B854B854B854D854D85CD85CD85CCE
:102A1000D85CD85CD85CF85CF85CF85CF85CF85C76
:102A20001865F864186518651865186518651865DF
:102A3000386538653865386D386D386D586D586D46
:102A4000586D586D586D586D586D586D386D386D9E
:102A5000386D386D386538651865186518651865FE
:102A6000186518651865F864F85CF85CF85CF85C43
:102A7000F85CD85CD85CD85CD85CD85CD85CB854BE
:102A8000B854B854B754B854B85498549754975449
:102A900097549754974C974C774C774C774C774C8E
:102AA000774C574C574C564C564C364C364C364C53
:102AB000364C364C364C154C154C154C154CF543D4
:102AC000154C755437755DDFFFFFFFFFFFFFFFFFFC
:102AD000FFFFFFFFFFFFFFFFFFFFFFFFFFFFFFFF06
:102AE000FFFFFFFFFFFFFFFFFFFFFFFFFFFFFFFFF6
:102AF000FFFFFFFFFFFFFFFFFFFFFFFFFFFFFFFFE6
:102B0000FFFFFFFFFFFFFFFFFFFFFFFFFFFFFFFFD5
:102D6000FFFFFFFFFFFFFFFFFFFF9BC6B56CD243D6
:102D7000B243D34BD44BD443D443F443F443F44B46
:102D8000F54BF54B154C154C154C154C154C354C5D
:102D9000364C364C364C364C564C364C564C564CC3
:102DA000564C574C774C774C774C774C774C974C2C
:102DB000974C97549754975497549854B754B75482
:102DC000B754B754B854B854B854D85CD85CD85C2D
:102DD000D85CD85CD85CD85CF85CF85CF864F85CCB
:102DE0001865F8641865186518651865186518651C
:102DF0001865386D386D386D386D386D386D586DB3
:102E0000586D586D586D586D586D386D386D386DFA
:102E1000386D386538653865186518651865186542
:102E200018651865F864F864F85CF85CF85CF85CA0
:102E3000F85CD85CD85CD85CD85CD85CD85CD85CD2
:102E4000B854B854B754B854B854B8549754975465
:102E5000975497549754974C974C774C774C774CA2
:102E6000774C774C574C574C564C564C364C564C2E
:102E7000364C364C364C364C354C154C154C154CA6
:102E8000354C955CD995FFFFFFFFFFFFFFFFFFFF6C
:102E9000FFFFFFFFFFFFFFFFFFFFFFFFFFFFFFFF42
:102EA000FFFFFFFFFFFFFFFFFFFFFFFFFFFFFFFF32
:102EB000FFFFFFFFFFFFFFFFFFFFFFFFFFFFFFFF22
:102EC000FFFFFFFFFFFFFFFFFFFFFFFFFFFFFFFF12
:10312000FFFFFFFFFFFFFFFF19AEF253713BB243FA
:10313000D343D343D443D443F443F44BF44BF44349
:10314000F54BF54B154C154C154C154C154C354C99
:10315000364C364C364C364C564C364C564C564CFF
:10316000564C574C774C774C774C774C774C974C68
:10317000974C97549754975497549854B854B854BC
:10318000B854B754B854D85CB854D85CD85CD85C40
:10319000D85CD85CF85CD85CF85CF85CF864F864DF
:1031A0001865F86418651865186518651865386538
:1031B0001865386D386D386D386D586D586D586DAF
:1031C000586D586D586D586D586D386D586D386D17
:1031D000386D386D386D386518651865186518656F
:1031E00018651865F8641865F85CF864F85CF85CB4
:1031F000F85CD85CD85CD85CD85CD85CD85CD85C0F
:10320000B854B854B754B854B854B85498549754A0
:10321000975497549754974C974C774C774C774CDE
:10322000774C774C574C574C564C564C364C564C6A
:10323000364C364C364C364C354C154C154C154CE2
:10324000344CB564BBC6FFFFFFFFFFFFFFFFFFFF6E
:10325000FFFFFFFFFFFFFFFFFFFFFFFFFFFFFFFF7E
:10326000FFFFFFFFFFFFFFFFFFFFFFFFFFFFFFFF6E
:10327000FFFFFFFFFFFFFFFFFFFFFFFFFFFFFFFF5E
:10328000FFFFFFFFFFFFFFFFFFFFFFFFFFFFFFFF4E
:1034E000FFFFFFFFFFFF989D9143513BB243D34342
:1034F000D343D343D443D443F443F44BF44BF44386
:10350000F54BF54B154C154C154C154C154C364CD4
:10351000364C364C364C564C564C364C564C564C1B
:10352000564C574C774C774C774C774C774C974CA4
:10353000974C97549754975497549854B854B854F8
:10354000B854B754B854D854B854D85CD85CD85C84
:10355000D85CD85CF85CD85CF85CF85CF864F8641B
:103560001865186518651865186518651865386553
:103570001865386D386D386D386D586D586D586DEB
:10358000586D586D586D586D586D386D586D386D53
:10359000386D386D386D38651865186518651865AB
:1035A00018651865F8641865F85CF864F85CF85CF0
:1035B000F85CD85CD85CD85CD85CD85CD85CD85C4B
:1035C000B854B854B754B854B854B85498549754DD
:1035D000975497549754974C974C774C774C774C1B
:1035E000774C774C574C574C564C564C364C564CA7
:1035F000364C364C364C364C354C154C154C154C1F
:10360000134C377DDFF7FFFFFFFFFFFFFFFFFFFFDB
:10361000FFFFFFFFFFFFFFFFFFFFFFFFFFFFFFFFBA
:10362000FFFFFFFFFFFFFFFFFFFFFFFFFFFFFFFFAA
:10363000FFFFFFFFFFFFFFFFFFFFFFFFFFFFFFFF9A
:10364000FFFFFFFFFFFFFFFFFFFFFFFFFFFFFFFF8A
:1038A000FFFFFFFF979D5043303BB243B343D343E9
:1038B000D343D343D443D443F443F44BF44BF443C2
:1038C000F54BF54B154C154C154C154C154C364C11
:1038D000364C364C364C564C564C364C564C564C58
:1038E000564C574C774C774C774C774C774C974CE1
:1038F000974C97549754975497549854B854B85435
:10390000B854B754B854D854B85CD85CD85CD85CB8
:10391000D85CD85CF85CD85CF85CF85CF864F86457
:10392000186518651865186518651865186538658F
:103930001865386D386D386D386D586D586D586D27
:10394000586D586D586D586D586D386D586D386D8F
:10395000386D386D386D38651865186518651865E7
:1039600018651865F864F864F85CF85CF85CF85C55
:10397000F85CD85CD85CD85CD85CD85CD85CD85C87
:10398000B854B854B754B854B854B854975497541A
:10399000975497549754974C974C774C774C774C57
:1039A000774C774C574C574C564C564C364C564CE3
:1039B000364C364C364C364C354C154C154CF44B7D
:1039C000135419A6FFFFFFFFFFFFFFFFFFFFFFFFDD
:1039D000FFFFFFFFFFFFFFFFFFFFFFFFFFFFFFFFF7
:1039E000FFFFFFFFFFFFFFFFFFFFFFFFFFFFFFFFE7
:1039F000FFFFFFFFFFFFFFFFFFFFFFFFFFFFFFFFD7
:103A0000FFFFFFFFFFFFFFFFFFFFFFFFFFFFFFFFC6
:103C6000FFFFF9AD2F3B0F339243B343B343D3432D
:103C7000D343D343D443D443F443F44BF44BF443FE
:103C8000F54BF54B154C154C154C154C154C364C4D
:103C9000364C364C364C564C364C364C564C564CB4
:103CA000564C574C574C774C774C774C774C774C5D
:103CB000974C975497549754975497549754B75494
:103CC000B754B754B854D854B854D85CD85CD85CFE
:103CD000D85CD85CF85CD85CF85CF85CF85CF8649C
:103CE0001865F8641865186518651865186518650D
:103CF0001865386D386D386D386D586D386D586D84
:103D0000586D586D586D586D586D386D386D386DEB
:103D1000386D386538651865186518651865186553
:103D200018651865F864F864F85CF85CF85CF85C91
:103D3000D85CD85CD85CD85CD85CD85CD85CB85C03
:103D4000B854B854B754B754B75498549754975478
:103D5000975497549754974C774C774C774C774CB3
:103D6000774C574C574C564C564C564C364C564C40
:103D7000364C364C364C354C354C154C154CD243E4
:103D800094645DE7FFFFFFFFFFFFFFFFFFFFFFFF03
:103D9000FFFFFFFFFFFFFFFFFFFFFFFFFFFFFFFF33
:103DA000FFFFFFFFFFFFFFFFFFFFFFFFFFFFFFFF23
:103DB000FFFFFFFFFFFFFFFFFFFFFFFFFFFFFFFF13
:103DC000FFFFFFFFFFFFFFFFFFFFFFFFFFFFFFFF03
:10402000BBCE504BCE329243B343B343B343D3439F
:10403000D343D343D443D443F443F44BF44BF4433A
:10404000F54BF54B154C154C154C154C154C154CAA
:10405000364C364C364C564C564C564C564C564CB0
:10406000774C574C774C774C774C984C774C974C17
:10407000984C975497549754B7549854B854B8548C
:10408000B854B854B854D85CD85CD85CD85CD85C08
:10409000D85CD85CF85CF85CF85CF85CF864F864B0
:1040A0001865186518651865186538651865186508
:1040B000386D386D386D386D586D586D586D586D58
:1040C000586D586D586D586D586D586D386D386D08
:1040D000386D386D38653865186518653865186548
:1040E000186518651865F8641865F85CF85CF85C84
:1040F000F85CD85CD85CD85CD85CD85CD85CD85C00
:10410000B854D854B854B854B854B8549754975471
:10411000975497549854974C974C774C774C774CCE
:10412000774C774C574C574C574C564C564C564C3A
:10413000364C364C364C364C364C154CD3439143AA
:10414000578DFFFFFFFFFFFFFFFFFFFFFFFFFFFF99
:10415000FFFFFFFFFFFFFFFFFFFFFFFFFFFFFFFF6F
:10416000FFFFFFFFFFFFFFFFFFFFFFFFFFFFFFFF5F
:10417000FFFFFFFFFFFFFFFFFFFFFFFFFFFFFFFF4F
:10418000FFFFFFFFFFFFFFFFFFFFFFFFFFFFFFFF3F
:1043D000FFFFFFFFFFFFFFFFFFFFFFFFFFFFBEF736
:1043E000F2638D2A513BB343B343B343B343D34347
:1043F000D343D343D443D443F443F44BF44BF44377
:10440000F54BF54B154C154C154C154C154C364CC5
:10441000564C564C564C564C564C574C574C774C69
:10442000774C774C774C774C974C984C984C984CF1
:10443000B85498549854B854B854B854B854D8543C
:10444000D854D85CD85CD85CD85CF85CF85CF85C74
:10445000F85CF85CF85CF85C186518651865186518
:10446000186519653965396539653965396D386D8E
:10447000386D386D586D596D596D596D596D596D4F
:10448000596D596D596D596D596D596D596D596DFC
:10449000586D586D386D386D386D386D38653865C4
:1044A0003865186518651865186518651865F85C2D
:1044B000F85CF85CF85CF85CF85CD85CD85CD85CBC
:1044C000D85CD854D854B854B854B854B854B85424
:1044D000B854985498549854984C984C984C974C7D
:1044E000774C774C774C774C574C564C564C564C37
:1044F000564C364C364C364C364C154C7143D253D8
:10450000BBC6FFFFFFFFFFFFFFFFFFFFFFFFFFFF38
:10451000FFFFFFFFFFFFFFFFFFFFFFFFFFFFFFFFAB
:10452000FFFFFFFFFFFFFFFFFFFFFFFFFFFFFFFF9B
:10453000FFFFFFFFFFFFFFFFFFFFFFFFFFFFFFFF8B
:10454000FFFFFFFFFFFFFFFFFFFFFFFFFFFFFFFF7B
:10479000FFFFFFFFFFFFFFFFFFFFFFFFFFFF779D13
:1047A000AD320F33B343B343B343B343B343D34304
:1047B000D343D343D443D443F443F44BF44BF44BAB
:1047C000F543F54BF54B154C364C364C354C154CEA
:1047D000F44BD3439243723B513B513B513B513BD2
:1047E000513B513B513B713B713B713B723B723BC7
:1047F000723B723B723B723B723B723B723B923B31
:104800007243924392439243924392439243924320
:104810009243924392439243B243B243B243B24370
:10482000B243B243B243B243B243B243B24BB24BD0
:10483000B24BB24BD24BD24BD24BD24BD24BD24BD0
:10484000D24BD24BD24BD24BD24BD24BD24BD24B80
:10485000D24BD24BD24BD24BD24BD24BD24BD24B70
:10486000D24BD24BD24BD24BD24BD243D243D24378
:10487000D243D243B243D243D243B243B243D243F0
:10488000B343B243B243B243B243B243B343B3437D
:10489000B343B343B343B243B243B243B243B2436D
:1048A000B243B243B243B2439243B243B243B24380
:1048B0009243924392439243924371430F339474D1
:1048C000FFFFFFFFFFFFFFFFFFFFFFFFFFFFFFFFF8
:1048D000FFFFFFFFFFFFFFFFFFFFFFFFFFFFFFFFE8
:1048E000FFFFFFFFFFFFFFFFFFFFFFFFFFFFFFFFD8
:1048F000FFFFFFFFFFFFFFFFFFFFFFFFFFFFFFFFC8
:104B5000FFFFFFFFFFFFFFFFFFFFFFFF5DE7704B62
:104B6000CE329243B343B343B343B343B343D3438C
:104B7000D343D443D443D443F443F44BF44BF44BE6
:104B8000F443F54B154C154CF44BB243513BEF320B
:104B9000AE2A6D226D228D2A8D2AAD2AAD2AAD2A2C
:104BA000AD2AAD2AAD2AAD2AAD2AAD2AAD2A8D2A6D
:104BB0008D2A8D2A8D2A8D2A8D2A8D2A8D2AAD2A1D
:104BC000AD2AAD2A8D2A8D2A8D2A8D2A8D2A8D2AED
:104BD0008D2A8D2A8D2A8D2A8D2A8D2A8D2AAD2AFD
:104BE000AD2A8D2A8D2A8D2AAD2AAD2A8D2A8D2AAD
:104BF0008D2AAD2AAD2AAD2AAD2AAD2AAD2AAD2A1D
:104C0000AD2AAD2AAD2AAD2AAD2AAD2AAD2AAD2AEC
:104C1000AE2AAD2AAD2AAD2AAD2AAE2AAE2AAE2AD8
:104C2000AE2AAE32AE32AE32CE32CE32CE32CE320C
:104C3000CE32CE32CE32CE32CE32CE32CE32CE3274
:104C4000CE32CE32CE32CE32CE32CE32CE32CE3264
:104C5000CE32EE32EE32EE32EE32EE32EE32EE3274
:104C6000EE32EF32EF32EF32EF32EF32EF32EF323D
:104C7000EF32EF32EF32EF32EF32CE2A504319B635
:104C8000FFFFFFFFFFFFFFFFFFFFFFFFFFFFFFFF34
:104C9000FFFFFFFFFFFFFFFFFFFFFFFFFFFFFFFF24
:104CA000FFFFFFFFFFFFFFFFFFFFFFFFFFFFFFFF14
:104CB000FFFFFFFFFFFFFFFFFFFFFFFFFFFFFFFF04
:104F1000FFFFFFFFFFFFFFFFFFFFFFFF5695CE32B2
:104F2000303BB343B343B343B343B343B343D3433C
:104F3000D343D443D443D443F443F44BF443F44332
:104F4000154CF54BD343713BCF2A8D22AE2A30430B
:104F5000F25BB47C5695B7A5F8AD19B619B619B67B
:104F600019B619B619B619B619B619B619B619B6C9
:104F700019B619B619B619B619B619B619B619B6B9
:104F800019B619B619B619B6F9B5F9B5F9B5F9B52D
:104F9000F9B5F9B5F9B5F9B5F9B5F9B5F9B5F9B5A1
:104FA000F9B5F9B5F9B5F9B5F9B5F9B5F9B5F9B591
:104FB000F9B5F9B5F9B5F9B5F9B5F8B5F8B5F8B584
:104FC000F8B5F8B5F8B5F8B518B6F8B5F8B5F8B558
:104FD00018B6F8B5F8B5F8B5F8B5F9B519B619B603
:104FE00019B619B619B619B619B619B619B619B649
:104FF00019B619B619B619B619B619B619B619B639
:1050000019B619B619B619B619B619B619B619B628
:1050100019B619B619B619B619B619B619B619B618
:1050200019B619B619B619B619B619B619B619B608
:1050300019B619B619B619B619B619B69AC6BEF781
:10504000FFFFFFFFFFFFFFFFFFFFFFFFFFFFFFFF70
:10505000FFFFFFFFFFFFFFFFFFFFFFFFFFFFFFFF60
:10506000FFFFFFFFFFFFFFFFFFFFFFFFFFFFFFFF50
:10507000FFFFFFFFFFFFFFFFFFFFFFFFFFFFFFFF40
:1052D000FFFFFFFFFFFFFFFFFFFFBEEFD253EF32E5
:1052E0009243B243B243B343B343B343B343D34311
:1052F000D343D443D443D443F443F443F44B154C45
:10530000D443713BAE2A8E225043B47CF9ADDBCE40
:105310003CDF7DEFBEF7DFFFFFFFFFFFFFFFFFFF7B
:10532000FFFFFFFFFFFFFFFFFFFFFFFFFFFFFFFF8D
:10533000FFFFFFFFFFFFFFFFFFFFFFFFFFFFFFFF7D
:10534000FFFFFFFFFFFFFFFFFFFFFFFFFFFFFFFF6D
:10535000FFFFFFFFFFFFFFFFFFFFFFFFFFFFFFFF5D
:10569000FFFFFFFFFFFFFFFFFFFFF9AD303B303B98
:1056A0009243B243B343B343B343B343B343D3434C
:1056B000D343D443D443D443D443F44BF44B924325
:1056C000EF32AE22914B7795DBCE7EEFFFFFFFFFEF
:1056D000FFFFFFFFFFFFFFFFFFFFFFFFFFFFFFFFDA
:1056E000FFFFFFFFFFFFFFFFFFFFFFFFFFFFFFFFCA
:1056F000FFFFFFFFFFFFFFFFFFFFFFFFFFFFFFFFBA
:10570000FFFFFFFFFFFFFFFFFFFFFFFFFFFFFFFFA9
:105A5000FFFFFFFFFFFFFFFFFFFF746C1033724378
:105A60009243B243B343B343B343B343B343D34388
:105A7000D343D443D443D443F44BD4437243AF2AE7
:105A8000103B368DFCD6DEF7FFFFFFFFFFFFFFFF69
:105A9000FFFFFFFFFFFFFFFFFFFFFFFFFFFFFFFF16
:105AA000FFFFFFFFFFFFFFFFFFFFFFFFFFFFFFFF06
:105AB000FFFFFFFFFFFFFFFFFFFFFFFFFFFFFFFFF6
:105AC000FFFFFFFFFFFFFFFFFFFFFFFFFFFFFFFFE6
:105E1000FFFFFFFFFFFFFFFFBBCE914331339243F4
:105E20009243B243B343B343B343B343B343D343C4
:105E3000B343D343D443F44BD343513BAF22F25B40
:105E40007BC6BEF7FFFFFFFFFFFFFFFFFFFFFFFF68
:105E5000FFFFFFFFFFFFFFFFFFFFFFFFFFFFFFFF52
:105E6000FFFFFFFFFFFFFFFFFFFFFFFFFFFFFFFF42
:105E7000FFFFFFFFFFFFFFFFFFFFFFFFFFFFFFFF32
:105E8000FFFFFFFFFFFFFFFFFFFFFFFFFFFFFFFF22
:1061D000FFFFFFFFFFFFFFFF36853133723B924326
:1061E0009243B2439343B343B343B343B343B34341
:1061F000B343D343D443D343713BCF22956CFCD6F6
:10620000FFFFFFFFFFFFFFFFFFFFFFFFFFFFFFFF9E
:10621000FFFFFFFFFFFFFFFFFFFFFFFFFFFFFFFF8E
:10622000FFFFFFFFFFFFFFFFFFFFFFFFFFFFFFFF7E
:10623000FFFFFFFFFFFFFFFFFFFFFFFFFFFFFFFF6E
:10659000FFFFFFFFFFFF7DE7F35331339243924349
:1065A000924392439243B343B343B343B343B3439E
:1065B000B343D443D3437243D022D5745DDFFFFF8E
:1065C000FFFFFFFFFFFFFFFFFFFFFFFFFFFFFFFFDB
:1065D000FFFFFFFFFFFFFFFFFFFFFFFFFFFFFFFFCB
:1065E000FFFFFFFFFFFFFFFFFFFFFFFFFFFFFFFFBB
:1065F000FFFFFFFFFFFFFFFFFFFFFFFFFFFFFFFFAB
:10695000FFFFFFFFFFFFD9A5723B513B92439243DC
:1069600092439243B243B343B343B343B343B343BA
:10697000D343D343B243F02A956C5DDFFFFFFFFFA3
:10698000FFFFFFFFFFFFFFFFFFFFFFFFFFFFFFFF17
:10699000FFFFFFFFFFFFFFFFFFFFFFFFFFFFFFFF07
:1069A000FFFFFFFFFFFFFFFFFFFFFFFFFFFFFFFFF7
:1069B000FFFFFFFFFFFFFFFFFFFFFFFFFFFFFFFFE7
:106D1000FFFFFFFFFFFF956C723B9243924392434C
:106D200092439243B243B243B343B343B343B343F7
:106D3000D343B3433133F34B1CD7FFFFFFFFFFFFB8
:106D4000FFFFFFFFFFFFFFFFFFFFFFFFFFFFFFFF53
:106D5000FFFFFFFFFFFFFFFFFFFFFFFFFFFFFFFF43
:106D6000FFFFFFFFFFFFFFFFFFFFFFFFFFFFFFFF33
:106D7000FFFFFFFFFFFFFFFFFFFFFFFFFFFFFFFF23
:1070D000FFFFFFFF7BBED343723B92439243924339
:1070E00092439243B243B343B343B343B343B34333
:1070F000B343923B52337BBEFFFFFFFFFFFFFFFF17
:10710000FFFFFFFFFFFFFFFFFFFFFFFFFFFFFFFF8F
:10711000FFFFFFFFFFFFFFFFFFFFFFFFFFFFFFFF7F
:10712000FFFFFFFFFFFFFFFFFFFFFFFFFFFFFFFF6F
:10713000FFFFFFFFFFFFFFFFFFFFFFFFFFFFFFFF5F
:10749000FFFFFFFF3785933B724372437243924372
:1074A00092439243B243B343B343B343B343B3436F
:1074B000D343322B3785BEF7FFFFFFFFFFFFFFFFF0
:1074C000FFFFFFFFFFFFFFFFFFFFFFFFFFFFFFFFCC
:1074D000FFFFFFFFFFFFFFFFFFFFFFFFFFFFFFFFBC
:1074E000FFFFFFFFFFFFFFFFFFFFFFFFFFFFFFFFAC
:1074F000FFFFFFFFFFFFFFFFFFFFFFFFFFFFFFFF9C
:10785000FFFF3DDF3554933B7243714392439243A4
:107860009243924392439243B343B343B343B343EC
:10787000933BB3431DD7FFFFFFFFFFFFFFFFFFFF5A
:10788000FFFFFFFFFFFFFFFFFFFFFFFFFFFFFFFF08
:10789000FFFFFFFFFFFFFFFFFFFFFFFFFFFFFFFFF8
:1078A000FFFFFFFFFFFFFFFFFFFFFFFFFFFFFFFFE8
:1078B000FFFFFFFFFFFFFFFFFFFFFFFFFFFFFFFFD8
:107C1000FFFFB99DD443923B724372439243924318
:107C2000924392439243B243B343B343B343D343E8
:107C3000522B588DBFF7FFFFFFFFFFFFFFFFFFFF36
:107C4000FFFFFFFFFFFFFFFFFFFFFFFFFFFFFFFF44
:107C5000FFFFFFFFFFFFFFFFFFFFFFFFFFFFFFFF34
:107C6000FFFFFFFFFFFFFFFFFFFFFFFFFFFFFFFF24
:107C7000FFFFFFFFFFFFFFFFFFFFFFFFFFFFFFFF14
:107FD000DFF7B764B43B92437143724392439243D9
:107FE000924392439243B243B343B243B343D44325
:107FF000B43BFCCEFFFFFFFFFFFFFFFFFFFFFFFFD4
:10800000FFFFFFFFFFFFFFFFFFFFFFFFFFFFFFFF80
:10801000FFFFFFFFFFFFFFFFFFFFFFFFFFFFFFFF70
:10802000FFFFFFFFFFFFFFFFFFFFFFFFFFFFFFFF60
:10803000FFFFFFFFFFFFFFFFFFFFFFFFFFFFFFFF50
:108390005BB6354CB33B7143714372439243924396
:1083A000924392439243B243B343B243D343933392
:1083B000B76C9EEFFFFFFFFFFFFFFFFFFFFFFFFF19
:1083C000FFFFFFFFFFFFFFFFFFFFFFFFFFFFFFFFBD
:1083D000FFFFFFFFFFFFFFFFFFFFFFFFFFFFFFFFAD
:1083E000FFFFFFFFFFFFFFFFFFFFFFFFFFFFFFFF9D
:1083F000FFFFFFFFFFFFFFFFFFFFFFFFFFFFFFFF8D
:10875000387DF543924371437143724392437243B0
:108760009243924392439243B3439243F4439433EC
:10877000FA9DDFF7FFFFFFFFFFFFFFFFFFFFFFFF98
:10878000FFFFFFFFFFFFFFFFFFFFFFFFFFFFFFFFF9
:10879000FFFFFFFFFFFFFFFFFFFFFFFFFFFFFFFFE9
:1087A000FFFFFFFFFFFFFFFFFFFFFFFFFFFFFFFFD9
:1087B000FFFFFFFFFFFFFFFFFFFFFFFFFFFFFFFFC9
:108B0000FFFFFFFFFFFFFFFFFFFFFFFFFFFF1DCF87
:108B10007754D43B7143714372437243724372433F
:108B20009243924392439243B2439243F443D53BE0
:108B3000DCC6FFFFFFFFFFFFFFFFFFFFFFFFFFFFA1
:108B4000FFFFFFFFFFFFFFFFFFFFFFFFFFFFFFFF35
:108B5000FFFFFFFFFFFFFFFFFFFFFFFFFFFFFFFF25
:108B6000FFFFFFFFFFFFFFFFFFFFFFFFFFFFFFFF15
:108B7000FFFFFFFFFFFFFFFFFFFFFFFFFFFFFFFF05
:108EC000FFFFFFFFFFFFFFFFFFFFFFFFFFFFBA9561
:108ED0003644B343714371437143724372439243C7
:108EE00092439243924392439243B343F543565481
:108EF0007EE7FFFFFFFFFFFFFFFFFFFFFFFFFFFF1B
:108F0000FFFFFFFFFFFFFFFFFFFFFFFFFFFFFFFF71
:108F1000FFFFFFFFFFFFDFF7FCCEDCC6DCC6DCC6D1
:108F2000DCC6DCC6DCC6DCC6DCC6DCC6DCC6DCC631
:108F3000DCC6DCC6DCC6DCC6FCC6FCC6FCC6FCC6A1
:108F4000FCC6FCC6FCC6FCC6FCC6FCC6FCC6FCC611
:108F5000FCC6FCC6FCC6FCC6FCC6FCC6FCC6FCC601
:108F6000FCC6FDC6FDC6FDC6FDC6FDC6FDC6FDC6EA
:108F7000FDC6FDC6FDC6FCC6FCC6FCC6FCC6FCC6DE
:108F8000FCC6FCC6FCC6FCC6FCC6FCC6FCC6FCC6D1
:108F9000FCC6FCC61DCFFFFFFFFFFFFFFFFFFFFF6B
:108FA000FFFFFFFFFFFFFFFFFFFFFFFFFFFFFFFFD1
:108FB000FFFFFFFFFFFFFFFFFFFFFFFFFFFF1CD7CC
:108FC0009BBE9BBEBBC6BBC6BBC6BBC6BBC6BBC6E9
:108FD000BBC6BCC6DCC6DCC6DCC6DCC6DCC6FCC6A2
:108FE000FCC6FCC6FCC6FCC6FCC6FCC65DDFFFFFBB
:108FF000FFFFFFFFFFFFFFFFFFFFFFFFFFFFFFFF81
:10900000FFFFFFFFFFFFFFFFFFFFFFFFFFFFFFFF70
:10901000FFFFFFFFFFFFFFFFFFFFFFFFFFFFFFFF60
:10902000FFFFFFFFFFFFFFFFFFFFFFFFFFFFFFFF50
:10928000FFFFFFFFFFFFFFFFFFFFFFFF9EEFF86401
:10929000F5437243514371437143724372439243A6
:1092A00092439243924392439243B343D53BF86433
:1092B0009EEFFFFFFFFFFFFFFFFFFFFFFFFFFFFF2F
:1092C000FFFFFFFFFFFFFFFFFFFFFFFFFFFFFFFFAE
:1092D000FFFFFFFFDCC63775B65CB65CB664D664CC
:1092E000D664D664D664D664D664D664D664D664AE
:1092F000D664F664D664F664F664F664F664F664DE
:10930000F664F664F764F764F76417651765176524
:10931000176D176D176D176D176D176D176D376D0D
:10932000176D376D376D376D376D376D376D386D3C
:10933000386D386D386D586D586D586D586D586D65
:10934000586D586D586D586D586D586D586D586DF5
:10935000586D586D38659BB6FFFFFFFFFFFFFFFF9D
:10936000FFFFFFFFFFFFFFFFFFFFFFFFFFFFFFFF0D
:10937000FFFFFFFFFFFFFFFFFFFFBEF75785D24B49
:10938000F24B13541354335434545454745C745C7B
:10939000755C955CB55CB664D664D664F664176596
:1093A000176D176D376D586D586D3865997D3DD7C0
:1093B000FFFFFFFFFFFFFFFFFFFFFFFFFFFFFFFFBD
:1093C000FFFFFFFFFFFFFFFFFFFFFFFFFFFFFFFFAD
:1093D000FFFFFFFFFFFFFFFFFFFFFFFFFFFFFFFF9D
:1093E000FFFFFFFFFFFFFFFFFFFFFFFFFFFFFFFF8D
:10964000FFFFFFFFFFFFFFFFFFFFFFFF5BAE774C5A
:10965000D443714351437143714371437243724325
:1096600072439243924392439243D343D533597DFD
:10967000BEEFFFFFFFFFFFFFFFFFFFFFFFFFFFFF4B
:10968000FFFFFFFFFFFFFFFFFFFFFFFFFFFFFFFFEA
:10969000FFFFFCCE7454344C144C144C144C144C3A
:1096A000144C144C144C154C354C354C354C354C35
:1096B000354C554C554C564C554C564C564C564CBE
:1096C000764C764C764C7654765476547654965442
:1096D0009654975497549754975497549754B75413
:1096E0009754B754B754B754B754B754B75CB7543A
:1096F000D75CD75CB75CD75CD75CD75CD75CD75CF2
:10970000D75CD75CD75CD85CF75CF75CF85CF85C3E
:10971000F85C1765D75C5BA6FFFFFFFFFFFFFFFF4D
:10972000FFFFFFFFFFFFFFFFFFFFFFFFFFFFFFFF49
:10973000FFFFFFFFFFFFFFFFDFF7B89D5033F34B45
:10974000564C554C554C564C564C564C564C564C0B
:10975000764C764C764C7654764C764C76547654E1
:1097600076549654965496549754F75C58755DD732
:10977000FFFFFFFFFFFFFFFFFFFFFFFFFFFFFFFFF9
:10978000FFFFFFFFFFFFFFFFFFFFFFFFFFFFFFFFE9
:10979000FFFFFFFFFFFFFFFFFFFFFFFFFFFFFFFFD9
:1097A000FFFFFFFFFFFFFFFFFFFFFFFFFFFFFFFFC9
:109A0000FFFFFFFFFFFFFFFFFFFFFFFF5975374419
:109A100092435143514371437143724372437243C2
:109A200092439243924392437243D443F633BA8DA6
:109A3000BFF7FFFFFFFFFFFFFFFFFFFFFFFFFFFF7E
:109A4000FFFFFFFFFFFFFFFFFFFFFFFFFFFFFFFF26
:109A5000FFFFF674D24BD34BD443D443D443D44307
:109A6000F443F443F443F54BF54BF54B154C154CCF
:109A7000154C154C154C364C364C364C364C364C39
:109A8000364C364C564C564C574C574C574C774CE2
:109A9000774C774C774C774C774C774C974C974C6E
:109AA000974C975497549754975498549754975465
:109AB000B754B754B754B754B754B754B854B8544C
:109AC000B854B854B854B854B854B854B854B85436
:109AD000D85CD664D65C7EE7FFFFFFFFFFFFFFFF89
:109AE000FFFFFFFFFFFFFFFFFFFFFFFFFFFFFFFF86
:109AF000FFFFFFFFFFFFFFFF7EE7D24B923BB75414
:109B0000B8549854985498549854984C974C974CEF
:109B1000974C774C774C774C774C574C574C574C6D
:109B2000564C564C364C364C76541765DA95FFFF3A
:109B3000FFFFFFFFFFFFFFFFFFFFFFFFFFFFFFFF35
:109B4000FFFFFFFFFFFFFFFFFFFFFFFFFFFFFFFF25
:109B5000FFFFFFFFFFFFFFFFFFFFFFFFFFFFFFFF15
:109B6000FFFFFFFFFFFFFFFFFFFFFFFFFFFFFFFF05
:109DC000FFFFFFFFFFFFFFFFFFFFDDC6D85CF5438E
:109DD0005143514371437143714371437243724321
:109DE00092439243924392437243D44B1634DA9592
:109DF000BFF7FFFFFFFFFFFFFFFFFFFFFFFFFFFFBB
:109E0000FFFFFFFFFFFFFFFFFFFFFFFFFFFFFFFF62
:109E10009EEFF253B243D343D343D443D443D4430A
:109E2000F443F443F443F443F54BF54BF54B154C35
:109E3000154C154C154C164C364C364C364C364C95
:109E4000364C364C364C564C564C574C574C774C3F
:109E5000774C774C774C774C774C774C774C974CCA
:109E6000974C974C975497549754975497549854A9
:109E7000B8549854B854B854B854B754B854B854A3
:109E8000B854B854B854B854B854B854B854D85452
:109E9000B75C54547885FFFFFFFFFFFFFFFFFFFF14
:109EA000FFFFFFFFFFFFFFFFFFFFFFFFFFFFFFFFC2
:109EB000FFFFFFFFFFFFFFFF19B6EF2A144CB85456
:109EC0009754975497549754974C974C974C774C7A
:109ED000774C774C774C774C574C574C574C574CEA
:109EE000564C564C364C364C9654176DBBBEFFFF45
:109EF000FFFFFFFFFFFFFFFFFFFFFFFFFFFFFFFF72
:109F0000FFFFFFFFFFFFFFFFFFFFFFFFFFFFFFFF61
:109F1000FFFFFFFFFFFFFFFFFFFFFFFFFFFFFFFF51
:109F2000FFFFFFFFFFFFFFFFFFFFFFFFFFFFFFFF41
:10A18000FFFFFFFFFFFFFFFFFFFFDA95984CB34390
:10A19000504351437143714371437143714372435F
:10A1A00072439243924392437243D44B163CFB95C5
:10A1B000BEF7FFFFFFFFFFFFFFFFFFFFFFFFFFFFF8
:10A1C000FFFFFFFFFFFFFFFFFFFFFFFFFFFFFFFF9F
:10A1D000DEF7B14B7143B343D443D443D443F44388
:10A1E000F443F44BF44BF443F54BF54BF54B154C62
:10A1F000154C154C154C354C364C364C364C364CB3
:10A20000564C564C364C564C564C574C564C574C5C
:10A21000774C774C774C774C774C774C974C974CE6
:10A22000974C9754975497549754975497549754DE
:10A230009854B854B854B854B854B854B754B754E0
:10A24000B754B854B854B854B854B854B854D8548F
:10A250007554F34BDBC6FFFFFFFFFFFFFFFFFFFF60
:10A26000FFFFFFFFFFFFFFFFFFFFFFFFFFFFFFFFFE
:10A27000FFFFFFFFFFFFBEF733640F337754B8547F
:10A28000975497549754974C974C974C774C774CDE
:10A29000774C774C774C774C774C574C574C564C07
:10A2A000564C564C364C564CB65C587DDFF7FFFF8B
:10A2B000FFFFFFFFFFFFFFFFFFFFFFFFFFFFFFFFAE
:10A2C000FFFFFFFFFFFFFFFFFFFFFFFFFFFFFFFF9E
:10A2D000FFFFFFFFFFFFFFFFFFFFFFFFFFFFFFFF8E
:10A2E000FFFFFFFFFFFFFFFFFFFFFFFFFFFFFFFF7E
:10A54000FFFFFFFFFFFFFFFF7EE7396D564C7143B2
:10A55000503B5143514371437143714372437243C2
:10A5600072437243924392437143D34B3644DA8D24
:10A57000BFF7FFFFFFFFFFFFFFFFFFFFFFFFFFFF33
:10A58000FFFFFFFFFFFFFFFFFFFFFFFFFFFFFFFFDB
:10A59000FFFFF584AE2A5143D443D443D443D4437C
:10A5A000D443F44BF44BF443F44BF44B154C154C9F
:10A5B000154C154C154C154C354C364C364C364C10
:10A5C000364C564C364C564C564C564C574C574CB9
:10A5D000574C774C774C774C774C774C774C974C63
:10A5E000974C974C974C975497549754975497542B
:10A5F000975497549854B854B854B8549854B8547D
:10A60000B854B754B754B754B754B854B85497540F
:10A61000D24B745CFFFFFFFFFFFFFFFFFFFFFFFF59
:10A62000FFFFFFFFFFFFFFFFFFFFFFFFFFFFFFFF3A
:10A63000FFFFFFFFFFFFBBCECE2AB243B8549754B3
:10A64000974C9754974C974C974C974C774C774C2A
:10A65000774C774C574C774C574C574C564C564C84
:10A66000364C364C364C7654B55C1AA6FFFFFFFFCD
:10A67000FFFFFFFFFFFFFFFFFFFFFFFFFFFFFFFFEA
:10A68000FFFFFFFFFFFFFFFFFFFFFFFFFFFFFFFFDA
:10A69000FFFFFFFFFFFFFFFFFFFFFFFFFFFFFFFFCA
:10A6A000FFFFFFFFFFFFFFFFFFFFFFFFFFFFFFFFBA
:10A90000FFFFFFFFFFFFFFFF5BA6F85CF44B304348
:10A91000503B51435143514371437143714372431F
:10A9200072439243924392437243D34B57449A8566
:10A93000BEEFFFFFFFFFFFFFFFFFFFFFFFFFFFFF78
:10A94000FFFFFFFFFFFFFFFFFFFFFFFFFFFFFFFF17
:10A95000FFFFBEF7B1536C220F3BD343F44BD443FC
:10A96000F443D443F44BF44BF443F54BF54B154C03
:10A97000154C154C154C154C354C164C364C364C6C
:10A98000364C364C564C364C564C564C564C574C16
:10A99000574C574C774C774C774C774C774C774CDF
:10A9A000974C974C774C974C9754974C9754975497
:10A9B00097549754975497549854B854B854B854DB
:10A9C000B8549854B854B854B854B754D854144CD4
:10A9D0003033D8A5FFFFFFFFFFFFFFFFFFFFFFFFA3
:10A9E000FFFFFFFFFFFFFFFFFFFFFFFFFFFFFFFF77
:10A9F000FFFFFFFFDEF7D47C8D22354CB854974C17
:10AA00009754974C974C974C774C774C774C774CA6
:10AA1000774C574C774C574C574C564C564C564CE1
:10AA2000364C564C564C5554F66C5DDFFFFFFFFF1D
:10AA3000FFFFFFFFFFFFFFFFFFFFFFFFFFFFFFFF26
:10AA4000FFFFFFFFFFFFFFFFFFFFFFFFFFFFFFFF16
:10AA5000FFFFFFFFFFFFFFFFFFFFFFFFFFFFFFFF06
:10AA6000FFFFFFFFFFFFFFFFFFFFFFFFFFFFFFFFF6
:10ACC000FFFFFFFFFFFFFFF7BA7DB7549243303B12
:10ACD0005043514351437143714371437143714335
:10ACE00072437243724392437243B343764C597535
:10ACF0009EEFFFFFFFFFFFFFFFFFFFFFFFFFFFFFD5
:10AD0000FFFFFFFFFFFFFFFFFFFFFFFFFFFFFFFF53
:10AD1000FFFFFFFF7EEFB1532C1AEF3AD343F44B02
:10AD2000D443D443F44BF44BF443F44BF44BF54B82
:10AD3000154C154C154C154C154C354C364C364CA9
:10AD4000364C364C364C564C364C564C564C564C73
:10AD5000574C574C774C774C774C774C774C774C1B
:10AD6000774C774C974C974C974C97549754974CFB
:10AD7000975497549754975497549754975498547A
:10AD8000B854B854B854B8549754B854B8547043DD
:10AD9000503B9EEFFFFFFFFFFFFFFFFFFFFFFFFFA7
:10ADA000FFFFFFFFFFFFFFFFFFFFFFFFFFFFFFFFB3
:10ADB000FFFFFFFF5DE7EE32103398549854974C35
:10ADC000974C974C974C774C774C774C774C774C0B
:10ADD000574C774C574C574C564C564C564C564C3F
:10ADE000564C364C354C5454988DFFFFFFFFFFFFF7
:10ADF000FFFFFFFFFFFFFFFFFFFFFFFFFFFFFFFF63
:10AE0000FFFFFFFFFFFFFFFFFFFFFFFFFFFFFFFF52
:10AE1000FFFFFFFFFFFFFFFFFFFFFFFFFFFFFFFF42
:10AE2000FFFFFFFFFFFFFFFFFFFFFFFFFFFFFFFF32
:10B08000FFFFFFFFFFFFDCC6596D354C3043303BFF
:10B09000514351435143714351437143714372438F
:10B0A00072437243924392437243924376541865BB
:10B0B0007EE7FFFFFFFFFFFFFFFFFFFFFFFFFFFF39
:10B0C000FFFFFFFFFFFFFFFFFFFFFFFFFFFFFFFF90
:10B0D000FFFFFFFFFFFFBEF712644D1A0F33B343AC
:10B0E000F44BF443D443F44BF44BF443F543F54BA6
:10B0F000154C154C154C154C154C154C354C364C07
:10B10000364C364C364C564C564C364C364C564CCF
:10B11000564C574C574C774C774C774C774C774C78
:10B12000774C774C774C974C774C974C974C97547F
:10B1300097549754975497549754975497549754B7
:10B1400097549754985498549854D854144C8D2A22
:10B150009474FFFFFFFFFFFFFFFFFFFFFFFFFFFFF5
:10B16000FFFFFFFFFFFFFFFFFFFFFFFFFFFFFFFFEF
:10B17000FFFFDFF7769D2B1AD343B954974C774CDA
:10B18000974C974C774C774C774C774C774C574C87
:10B19000774C574C574C574C564C564C364C364CBB
:10B1A000564C364C344C745C9BBEFFFFFFFFFFFFD8
:10B1B000FFFFFFFFFFFFFFFFFFFFFFFFFFFFFFFF9F
:10B1C000FFFFFFFFFFFFFFFFFFFFFFFFFFFFFFFF8F
:10B1D000FFFFFFFFFFFFFFFFFFFFFFFFFFFFFFFF7F
:10B1E000FFFFFFFFFFFFFFFFFFFFFFFFFFFFFFFF6F
:10B44000FFFFFFFFFFFF1B961865B24B303B303B01
:10B4500051435043514351435143714371437143ED
:10B4600072437243924392439243513B7654D75472
:10B47000FDCEFFFFFFFFFFFFFFFFFFFFFFFFFFFF0F
:10B48000FFFFFFFFFFFFFFFFFFFFFFFFFFFFFFFFCC
:10B49000FFFFFFFFFFFFFFFFFFFF746C6D220F3BFD
:10B4A000B343F44BD443F44BF44BF44BF443F54B1C
:10B4B000F54B154C154C154C154C154C354C154C85
:10B4C000354C364C364C364C564C564C364C564C0D
:10B4D000564C564C574C574C574C774C574C774C16
:10B4E000774C774C774C774C974C974C774C974CE4
:10B4F000974C9754975497549754975497549754FC
:10B5000097549754975497549854B854303B4C22BE
:10B51000DBCEFFFFFFFFFFFFFFFFFFFFFFFFFFFF90
:10B52000FFFFFFFFFFFFFFFFFFFFFFFFFFFFFFFF2B
:10B53000FFFFBEF7704B8D2A774CB854774C974C71
:10B54000774C774C774C774C774C774C574C774C03
:10B55000574C574C564C564C564C364C364C564C19
:10B56000364C354C134CF674FFFFFFFFFFFFFFFF17
:10B57000FFFFFFFFFFFFFFFFFFFFFFFFFFFFFFFFDB
:10B58000FFFFFFFFFFFFFFFFFFFFFFFFFFFFFFFFCB
:10B59000FFFFFFFFFFFFFFFFFFFFFFFFFFFFFFFFBB
:10B5A000FFFFFFFFFFFFFFFFFFFFFFFFFFFFFFFFAB
:10B80000FFFFFFFF5DDFBA7D965C5043103B504366
:10B81000513B504351435143714351437143714331
:10B8200072437243724372439243513B1454D75450
:10B830005BA6DFF7FFFFFFFFFFFFFFFFFFFFFFFF3D
:10B84000FFFFFFFFFFFFFFFFFFFFFFFFFFFFFFFF08
:10B85000FFFFFFFFFFFFFFFFFFFFFFFFD57C8E22F3
:10B86000103BB343F44BD443F44BF44BF443F44355
:10B87000F44B154CF54B154C154C154C154C354CE3
:10B88000164C364C364C364C364C564C364C564C88
:10B89000364C564C564C574C574C574C774C574C93
:10B8A000774C774C774C774C774C774C974C974C40
:10B8B000774C974C974C97549754974C9754975470
:10B8C0009754975497549754B854354C6D2A9153C4
:10B8D000FFFFFFFFFFFFFFFFFFFFFFFFFFFFFFFF78
:10B8E000FFFFFFFFFFFFFFFFFFFFFFFFFFFFFFFF68
:10B8F000FFFF7ABE6D22723BB854974C774C774C61
:10B90000774C774C774C774C774C774C774C574C3F
:10B91000574C564C564C564C364C364C564C364C76
:10B92000364CF44BF24BD9A5FFFFFFFFFFFFFFFFA3
:10B93000FFFFFFFFFFFFFFFFFFFFFFFFFFFFFFFF17
:10B94000FFFFFFFFFFFFFFFFFFFFFFFFFFFFFFFF07
:10B95000FFFFFFFFFFFFFFFFFFFFFFFFFFFFFFFFF7
:10B96000FFFFFFFFFFFFFFFFFFFFFFFFFFFFFFFFE7
:10BBC000FFFFFFFF7BAE796D134C103B303B5043C2
:10BBD000303B5043514351435143514371437143AF
:10BBE000714372437243924392437243B243F75C90
:10BBF000997DBEEFFFFFFFFFFFFFFFFFFFFFFFFF8E
:10BC0000FFFFFFFFFFFFFFFFFFFFFFFFFFFFFFFF44
:10BC1000FFFFFFFFFFFFFFFFFFFFFFFFFFFF168597
:10BC2000AF22303BB343F44BF443F44BF44BF443B7
:10BC3000F543F54B154CF54B154C154C154C154C67
:10BC4000354C164C364C364C364C364C564C364CE5
:10BC5000364C364C564C564C574C574C574C774CF0
:10BC6000774C774C774C774C774C774C774C774CBC
:10BC7000974C974C774C974C974C975497549754B4
:10BC80009754974C97549754B85492434C1AD8A54C
:10BC9000FFFFFFFFFFFFFFFFFFFFFFFFFFFFFFFFB4
:10BCA000FFFFFFFFFFFFFFFFFFFFFFFFFFFFFFFFA4
:10BCB000DEF7746C8E22364CB854774C774C774C48
:10BCC000774C774C774C574C774C574C574C574CDC
:10BCD000564C564C564C364C364C564C364C364CD4
:10BCE000364CD24354647EE7FFFFFFFFFFFFFFFFA8
:10BCF000FFFFFFFFFFFFFFFFFFFFFFFFFFFFFFFF54
:10BD0000FFFFFFFFFFFFFFFFFFFFFFFFFFFFFFFF43
:10BD1000FFFFFFFFFFFFFFFFFFFFFFFFFFFFFFFF33
:10BD2000FFFFFFFFFFFFFFFFFFFFFFFFFFFFFFFF23
:10BF8000FFFFDFF7FA85F75C71430F3B3043304327
:10BF9000303B513B504351435143714371437143D3
:10BFA000714372437243724372439243513BB65C96
:10BFB000385D1DCFFFFFFFFFFFFFFFFFFFFFFFFF0C
:10BFC000FFFFFFFFFFFFFFFFFFFFFFFFFFFFFFFF81
:10BFD000FFFFFFFFFFFFFFFFFFFFFFFFFFFFFFFF71
:10BFE0007795CF22313BB343F443F44BF44BF44BFE
:10BFF000F443F54BF54B154C154C154C154C154CA5
:10C00000154C354C364C364C364C364C364C564C22
:10C01000564C364C364C564C564C574C574C574C4D
:10C02000574C774C574C774C774C774C774C774C38
:10C03000774C774C974C974C974C774C974C974C48
:10C04000974C975497549854774CEF32303BFFFFFE
:10C05000FFFFFFFFFFFFFFFFFFFFFFFFFFFFFFFFF0
:10C06000FFFFFFFFFFFFFFFFFFFFFFFFFFFFFFFFE0
:10C070003DDF1033723B984C774C774C774C774CC4
:10C08000774C774C574C774C574C574C574C564C39
:10C09000564C364C564C364C564C364C364C364C30
:10C0A000F44B91433685FFFFFFFFFFFFFFFFFFFFCC
:10C0B000FFFFFFFFFFFFFFFFFFFFFFFFFFFFFFFF90
:10C0C000FFFFFFFFFFFFFFFFFFFFFFFFFFFFFFFF80
:10C0D000FFFFFFFFFFFFFFFFFFFFFFFFFFFFFFFF70
:10C0E000FFFFFFFFFFFFFFFFFFFFFFFFFFFFFFFF60
:10C34000FFFFBCBE796D3454303B0F3B303B304374
:10C350005043303B50435143514351437143714328
:10C36000714371437243724392439243513BF34B87
:10C37000F75CDA8DBEF7FFFFFFFFFFFFFFFFFFFF58
:10C38000FFFFFFFFFFFFFFFFFFFFFFFFFFFFFFFFBD
:10C39000FFFFFFFFFFFFFFFFFFFFFFFFFFFFFFFFAD
:10C3A000FFFFD9A5F022513BD343F443F44BF44BA8
:10C3B000F443F443F54BF54B154C154C154C154C0B
:10C3C000154C154C354C364C364C364C364C364CA0
:10C3D000564C564C364C364C564C564C564C574C8C
:10C3E000574C574C774C774C774C774C774C774C75
:10C3F000774C774C774C774C774C974C974C974CC5
:10C40000774C974C974CB854F4438E22F684FFFF38
:10C41000FFFFFFFFFFFFFFFFFFFFFFFFFFFFFFFF2C
:10C42000FFFFFFFFFFFFFFFFFFFFFFFFFFFFDFF744
:10C430007895AF22154C984C774C774C774C774CCD
:10C44000574C774C774C574C564C574C564C564C97
:10C45000364C364C364C564C364C364C364C364CAC
:10C460009243B14BBBC6FFFFFFFFFFFFFFFFFFFF84
:10C47000FFFFFFFFFFFFFFFFFFFFFFFFFFFFFFFFCC
:10C48000FFFFFFFFFFFFFFFFFFFFFFFFFFFFFFFFBC
:10C49000FFFFFFFFFFFFFFFFFFFFFFFFFFFFFFFFAC
:10C4A000FFFFFFFFFFFFFFFFFFFFFFFFFFFFFFFF9C
:10C70000FFFFFB95F85C92430F3B303B303B3043DF
:10C710003043303B513B50435143514351437143AC
:10C720007143714372437243724392437243714344
:10C73000B65CF8541DCFFFFFFFFFFFFFFFFFFFFFB9
:10C74000FFFFFFFFFFFFFFFFFFFFFFFFFFFFFFFFF9
:10C75000FFFFFFFFFFFFFFFFFFFFFFFFFFFFFFFFE9
:10C76000FFFFFFFF1AAE112B723BD343F44BF44B88
:10C77000F44BF443F443F44BF54B154C154C154C6A
:10C78000154C154C154C354C364C364C364C364CFD
:10C79000364C364C564C364C364C564C564C564C09
:10C7A000574C574C574C574C774C774C774C774CF1
:10C7B000774C774C774C774C774C774C774C774C61
:10C7C000974C974C974C974C713BF02A3DDFFFFFFD
:10C7D000FFFFFFFFFFFFFFFFFFFFFFFFFFFFFFFF69
:10C7E000FFFFFFFFFFFFFFFFFFFFFFFFFFFFBEEFAA
:10C7F000D34B7233774C974C774C774C574C774CE4
:10C80000774C574C574C574C564C564C564C364C14
:10C81000364C564C564C364C364C364C364CF44B0B
:10C82000503B946CFFFFFFFFFFFFFFFFFFFFFFFF89
:10C83000FFFFFFFFFFFFFFFFFFFFFFFFFFFFFFFF08
:10C84000FFFFFFFFFFFFFFFFFFFFFFFFFFFFFFFFF8
:10C85000FFFFFFFFFFFFFFFFFFFFFFFFFFFFFFFFE8
:10C86000FFFFFFFFFFFFFFFFFFFFFFFFFFFFFFFFD8
:10CAC0001DCF796D554C303B0F3B303B303B3043F5
:10CAD00030435043513B50435143514371435143C1
:10CAE0007143714371437243724392439243514382
:10CAF000F34BD7545975BEEFFFFFFFFFFFFFFFFF5A
:10CB0000FFFFFFFFFFFFFFFFFFFFFFFFFFFFFFFF35
:10CB1000FFFFFFFFFFFFFFFFFFFFFFFFFFFFFFFF25
:10CB2000FFFFFFFFFFFF7BBE522B723BD343F44B53
:10CB3000F44BF44BF443F543F44B154CF54B154CC7
:10CB4000154C154C154C154C354C364C364C364C5A
:10CB5000364C364C364C564C364C564C364C564C65
:10CB6000564C564C574C574C574C574C774C774C6F
:10CB7000774C774C774C774C774C774C774C774C9D
:10CB8000774C774C984C364CF02A5464FFFFFFFFEB
:10CB9000FFFFFFFFFFFFFFFFFFFFFFFFFFFFFFFFA5
:10CBA000FFFFFFFFFFFFFFFFFFFFFFFFFFFF7BB662
:10CBB000322B154C974C774C574C774C774C574C45
:10CBC000574C564C574C564C564C364C564C364C93
:10CBD000564C564C364C364C364C364C364C9243B2
:10CBE0002F3BD8A5FFFFFFFFFFFFFFFFFFFFFFFF6A
:10CBF000FFFFFFFFFFFFFFFFFFFFFFFFFFFFFFFF45
:10CC0000FFFFFFFFFFFFFFFFFFFFFFFFFFFFFFFF34
:10CC1000FFFFFFFFFFFFFFFFFFFFFFFFFFFFFFFF24
:10CC2000FFFFFFFFFFFFFFFFFFFFFFFFFFFFFFFF14
:10CE80001B9EF85CB2430F3B0F3B303B303B303BCB
:10CE900030433043503B514350435143514351433E
:10CEA000714371437143724372437243924392439D
:10CEB000513B5554B74C1B96DFFFFFFFFFFFFFFFB1
:10CEC000FFFFFFFFFFFFFFFFFFFFFFFFFFFFFFFF72
:10CED000FFFFFFFFFFFFFFFFFFFFFFFFFFFFFFFF62
:10CEE000FFFFFFFFFFFFFFFFBCC673339333D44345
:10CEF000F44BF44BF44BF443F543F54B154CF54B25
:10CF0000154C154C154C154C154C354C164C364CD7
:10CF1000364C364C364C364C564C364C364C364CE1
:10CF2000564C564C564C564C574C574C574C574CED
:10CF3000774C574C774C774C774C774C774C774CF9
:10CF4000774C774C984CD443102B7BBEFFFFFFFFF0
:10CF5000FFFFFFFFFFFFFFFFFFFFFFFFFFFFFFFFE1
:10CF6000FFFFFFFFFFFFFFFFFFFFFFFFDFF7D76CB4
:10CF70007333564C774C574C774C574C574C564C58
:10CF8000574C564C564C564C364C364C364C564CF0
:10CF9000364C364C364C364C364C364CF54B0F3303
:10CFA000D153BEEFFFFFFFFFFFFFFFFFFFFFFFFFBC
:10CFB000FFFFFFFFFFFFFFFFFFFFFFFFFFFFFFFF81
:10CFC000FFFFFFFFFFFFFFFFFFFFFFFFFFFFFFFF71
:10CFD000FFFFFFFFFFFFFFFFFFFFFFFFFFFFFFFF61
:10CFE000FFFFFFFFFFFFFFFFFFFFFFFFFFFFFFFF51
:10D23000FFFFFFFFFFFFFFFFFFFFFFFFFFFF9EE777
:10D240005A75764C50430F3B303B303B303B303BC4
:10D2500030433043303B513B504351435143714382
:10D2600051437143714371437243724392439243FA
:10D27000724372439754974C7BAEFFFFFFFFFFFF53
:10D28000FFFFFFFFFFFFFFFFFFFFFFFFFFFFFFFFAE
:10D29000FFFFFFFFFFFFFFFFFFFFFFFFFFFFFFFF9E
:10D2A000FFFFFFFFFFFFFFFFFFFF1DD7B43B9333DF
:10D2B000F443F44BF44BF44BF443F54BF54B154C62
:10D2C000F54B154C154C154C154C154C354C164C56
:10D2D000354C364C364C364C364C564C564C364CFF
:10D2E000564C364C564C564C564C564C574C574C4C
:10D2F000574C574C774C774C774C574C774C774C76
:10D30000774C774C574C723BD34BFFFFFFFFFFFF2F
:10D31000FFFFFFFFFFFFFFFFFFFFFFFFFFFFFFFF1D
:10D32000FFFFFFFFFFFFFFFFFFFFFFFF3DD7B4330E
:10D330001544774C774C574C574C564C574C564CE1
:10D34000564C564C364C564C364C564C564C364C2D
:10D35000364C364C364C364C364C364CB243CE32CC
:10D36000F584FFFFFFFFFFFFFFFFFFFFFFFFFFFF52
:10D37000FFFFFFFFFFFFFFFFFFFFFFFFFFFFFFFFBD
:10D38000FFFFFFFFFFFFFFFFFFFFFFFFFFFFFFFFAD
:10D39000FFFFFFFFFFFFFFFFFFFFFFFFFFFFFFFF9D
:10D3A000FFFFFFFFFFFFFFFFFFFFFFFFFFFFFFFF8D
:10D5F000FFFFFFFFFFFFFFFFFFFFFFFFFFFF7BAE10
:10D60000F95CD3430F3B0F3B2F3B2F3B303B303B71
:10D61000303B30435043303B5143504351435143DF
:10D620007143714371437143724372437243724356
:10D6300092437143B2439754974C7CB6FFFFFFFF70
:10D64000FFFFFFFFFFFFFFFFFFFFFFFFFFFFFFFFEA
:10D65000FFFFFFFFFFFFFFFFFFFFFFFFFFFFFFFFDA
:10D66000FFFFFFFFFFFFFFFFFFFFFFFF3DDFF54372
:10D67000B433F54BF443F44BF443F443F54BF54B1F
:10D68000154CF54B154C154C154C154C154C354C93
:10D69000154C364C364C364C364C364C364C564C7B
:10D6A000564C364C364C364C564C564C564C564CCA
:10D6B000574C564C574C574C574C774C774C774CF3
:10D6C000574C774C1544522BB995FFFFFFFFFFFFD6
:10D6D000FFFFFFFFFFFFFFFFFFFFFFFFFFFFFFFF5A
:10D6E000FFFFFFFFFFFFFFFFFFFFDFF79A8DB5335F
:10D6F000564C574C574C564C574C564C564C564C17
:10D70000364C364C364C564C564C364C364C364CC9
:10D71000364C364C364C364C364C1544AE2AAD2A77
:10D72000BBCEFFFFFFFFFFFFFFFFFFFFFFFFFFFF7E
:10D73000FFFFFFFFFFFFFFFFFFFFFFFFFFFFFFFFF9
:10D74000FFFFFFFFFFFFFFFFFFFFFFFFFFFFFFFFE9
:10D75000FFFFFFFFFFFFFFFFFFFFFFFFFFFFFFFFD9
:10D76000FFFFFFFFFFFFFFFFFFFFFFFFFFFFFFFFC9
:10D9B000FFFFFFFFFFFFFFFFFFFFFFFFFFFF5A75A6
:10D9C0003644513B0F3B30432F3B103B303B303B09
:10D9D000303B30433043303B513B50435143514344
:10D9E00051435143714371437143724372439243B4
:10D9F000724392437143B343975477445BAEFFFF46
:10DA0000FFFFFFFFFFFFFFFFFFFFFFFFFFFFFFFF26
:10DA1000FFFFFFFFFFFFFFFFFFFFFFFFFFFFFFFF16
:10DA2000FFFFFFFFFFFFFFFFFFFFFFFFFFFF9EE77F
:10DA3000364CD533154CF443F44BF443F443F54BD7
:10DA4000F54B154CF54B154C154C154C154C154C10
:10DA5000354C154C364C364C364C364C364C364CD8
:10DA6000364C564C564C364C364C364C564C564C26
:10DA7000564C564C574C574C564C574C574C574C91
:10DA8000774C574CF443933B9EEFFFFFFFFFFFFFA4
:10DA9000FFFFFFFFFFFFFFFFFFFFFFFFFFFFFFFF96
:10DAA000FFFFFFFFFFFFFFFFFFFFBEEF774C364496
:10DAB000574C574C564C564C564C564C364C364C94
:10DAC000364C364C564C364C364C364C364C364C26
:10DAD000364C364C154CF543D53B312BEB11B1533D
:10DAE000FFFFFFFFFFFFFFFFFFFFFFFFFFFFFFFF46
:10DAF000FFFFFFFFFFFFFFFFFFFFFFFFFFFFFFFF36
:10DB0000FFFFFFFFFFFFFFFFFFFFFFFFFFFFFFFF25
:10DB1000FFFFFFFFFFFFFFFFFFFFFFFFFFFFFFFF15
:10DD7000FFFFFFFFFFFFFFFFFFFFFFFF9CB67844A1
:10DD8000532B8D2A8D2ACF320F3B30433043304303
:10DD9000303B303B303B503B303B51435043514391
:10DDA00051437143714371437143724372437243F0
:10DDB0009243924392437143B343774C573C1B9E2B
:10DDC000FFFFFFFFFFFFFFFFFFFFFFFFFFFFFFFF63
:10DDD000FFFFFFFFFFFFFFFFFFFFFFFFFFFFFFFF53
:10DDE000FFFFFFFFFFFFFFFFFFFFFFFFFFFFFFFF43
:10DDF000BFF77654D533364CF443F44BF443F44335
:10DE0000F54BF54BF54B154C154C154C154C154C6D
:10DE1000154C154C354C164C354C364C364C364C56
:10DE2000364C364C364C564C364C364C364C364CC2
:10DE3000564C564C564C564C564C564C574C564CD1
:10DE4000574C364C94331775FFFFFFFFFFFFFFFF62
:10DE5000FFFFFFFFFFFFFFFFFFFFFFFFFFFFFFFFD2
:10DE6000FFFFFFFFFFFFFFFFFFFF7CB61634774C7D
:10DE7000564C564C564C564C364C364C364C364C12
:10DE8000564C564C364C364C364C564C364C164C42
:10DE9000F543D53BB433B433B433AE222C1AB7A513
:10DEA000FFFFFFFFFFFFFFFFFFFFFFFFFFFFFFFF82
:10DEB000FFFFFFFFFFFFFFFFFFFFFFFFFFFFFFFF72
:10DEC000FFFFFFFFFFFFFFFFFFFFFFFFFFFFFFFF62
:10DED000FFFFFFFFFFFFFFFFFFFFFFFFFFFFFFFF52
:10E13000FFFFFFFFFFFFFFFFFFFFFFFF7A7DF633CB
:10E14000F02A6D226D226D228D2AAE2AEF320F3B0E
:10E150003043304330433043503B513B50435143B5
:10E16000514351435143714371437143714372436E
:10E1700072437243924392437243B243774C373CAB
:10E18000DA95FFFFFFFFFFFFFFFFFFFFFFFFFFFF2E
:10E19000FFFFFFFFFFFFFFFFFFFFFFFFFFFFFFFF8F
:10E1A000FFFFFFFFFFFFFFFFFFFFFFFFFFFFFFFF7F
:10E1B000FFFFFFFFB85CF633564CF443D443F44BF7
:10E1C000F443F543F44BF54B154C154C154C154CDD
:10E1D000154C154C154C354C154C364C364C364CB4
:10E1E000364C364C364C364C564C564C564C364CBF
:10E1F000364C364C364C564C564C564C564C564C6F
:10E20000564C364CB433FCCEFFFFFFFFFFFFFFFF41
:10E21000FFFFFFFFFFFFFFFFFFFFFFFFFFFFFFFF0E
:10E22000FFFFFFFFFFFFFFFFDFF7196D5744574C5C
:10E23000364C364C364C364C364C364C564C564C8E
:10E24000564C564C564C364C1544F543D43BB433DF
:10E25000B43394339433B43373334D1A5043FFFFC4
:10E26000FFFFFFFFFFFFFFFFFFFFFFFFFFFFFFFFBE
:10E27000FFFFFFFFFFFFFFFFFFFFFFFFFFFFFFFFAE
:10E28000FFFFFFFFFFFFFFFFFFFFFFFFFFFFFFFF9E
:10E29000FFFFFFFFFFFFFFFFFFFFFFFFFFFFFFFF8E
:10E4F000FFFFFFFFFFFFFFFFFFFF3DD7784C732BB0
:10E500008E2A6C228D228D2A8D2A8D226E228E22B9
:10E51000AE2ACF32103B303B50435143514350431E
:10E5200051435143714351437143714372437243A9
:10E530007243924372439243924372439243564CC6
:10E5400017349A85FFFFFFFFFFFFFFFFFFFFFFFF6D
:10E55000FFFFFFFFFFFFFFFFFFFFFFFFFFFFFFFFCB
:10E56000FFFFFFFFFFFFFFFFFFFFFFFFFFFFFFFFBB
:10E57000FFFFFFFFFFFF186DF633774CF443D443E2
:10E58000F44BF443F443F54BF54B154CF54B154C5C
:10E59000154C154C154C154C154C354C154C364C32
:10E5A000364C364C364C364C364C364C364C564C3B
:10E5B000564C564C364C364C364C364C364C564CEB
:10E5C000564C1644975CFFFFFFFFFFFFFFFFFFFF66
:10E5D000FFFFFFFFFFFFFFFFFFFFFFFFFFFFFFFF4B
:10E5E000FFFFFFFFFFFFFFFF1DD777449754364C17
:10E5F000564C364C364C364C564C564C564C564C6B
:10E60000364C1544F53BD533B433B433B433B4335B
:10E61000B4339433B4339433112B6D1AF684FFFF63
:10E62000FFFFFFFFFFFFFFFFFFFFFFFFFFFFFFFFFA
:10E63000FFFFFFFFFFFFFFFFFFFFFFFFFFFFFFFFEA
:10E64000FFFFFFFFFFFFFFFFFFFFFFFFFFFFFFFFDA
:10E65000FFFFFFFFFFFFFFFFFFFFFFFFFFFFFFFFCA
:10E8B000FFFFFFFFFFFFFFFFFFFFBA95D533F02AF1
:10E8C0006D226D228D2A8D228D2A8E2A8E2A8E2AE5
:10E8D0008E2A8E22AE22AE2ACF2AEF32303B504310
:10E8E00051437143714371437143714371437143A8
:10E8F00072437243924392439243924372439243D0
:10E90000364CD633597DFFFFFFFFFFFFFFFFFFFFB0
:10E91000FFFFFFFFFFFFFFFFFFFFFFFFFFFFFFFF07
:10E92000FFFFFFFFFFFFFFFFFFFFFFFFFFFFFFFFF7
:10E93000FFFFFFFFFFFFFFFF597516349854F44B9C
:10E94000D343F44BF443F443F54BF54B154CF54BE3
:10E95000154C154C154C154C154C154C354C354C6F
:10E96000164C354C364C364C364C364C364C364CB8
:10E97000364C364C564C564C564C364C364C364C27
:10E98000574CF6333BA6FFFFFFFFFFFFFFFFFFFFE4
:10E99000FFFFFFFFFFFFFFFFFFFFFFFFFFFFFFFF87
:10E9A000FFFFFFFFFFFFDFFFDA8D774C7754364C18
:10E9B000564C564C564C564C364C1644F543D53BAB
:10E9C000B533B433B433B433B433B433B433B4330E
:10E9D0009433B43394339333D02210333DDFFFFFAD
:10E9E000FFFFFFFFFFFFFFFFFFFFFFFFFFFFFFFF37
:10E9F000FFFFFFFFFFFFFFFFFFFFFFFFFFFFFFFF27
:10EA0000FFFFFFFFFFFFFFFFFFFFFFFFFFFFFFFF16
:10EA1000FFFFFFFFFFFFFFFFFFFFFFFFFFFFFFFF06
:10EC7000FFFFFFFFFFFFFFFFBFF7975C33238E2AE5
:10EC80004C226D2A8D2A6D228D2A8D2A8D2A8E2A5C
:10EC9000AE2AAE2AAE2AAE2AAE2AAE22AE2AAF2ABB
:10ECA000CF2A1033303B5143714371439143724338
:10ECB000724372437243724392439243924392432C
:10ECC0009243154CB52BF86CFFFFFFFFFFFFFFFFD2
:10ECD000FFFFFFFFFFFFFFFFFFFFFFFFFFFFFFFF44
:10ECE000FFFFFFFFFFFFFFFFFFFFFFFFFFFFFFFF34
:10ECF000FFFFFFFFFFFFFFFFFFFFBA85573CD85C18
:10ED0000F54BD343F44BF443F443F54BF54BF54B40
:10ED1000154CF54B154C154C154C154C154C154C0C
:10ED2000354C354C154C364C364C364C364C364CF6
:10ED3000364C364C364C364C364C564C564C364C83
:10ED4000774C5744DFFFFFFFFFFFFFFFFFFFFFFF91
:10ED5000FFFFFFFFFFFFFFFFFFFFFFFFFFFFFFFFC3
:10ED6000FFFFFFFFFFFFBEEFF85CD85C564C564C30
:10ED7000364C1644F543D53BD533B433B433B433B2
:10ED8000B433B433B433B433B433B4339433B4336B
:10ED9000943394339433522BD022756CFFFFFFFFD2
:10EDA000FFFFFFFFFFFFFFFFFFFFFFFFFFFFFFFF73
:10EDB000FFFFFFFFFFFFFFFFFFFFFFFFFFFFFFFF63
:10EDC000FFFFFFFFFFFFFFFFFFFFFFFFFFFFFFFF53
:10EDD000FFFFFFFFFFFFFFFFFFFFFFFFFFFFFFFF43
:10F03000FFFFFFFFFFFFFFFF1AA6B433D0226D2AA8
:10F040006C226D2A6D2A8D228D228D2A8E2A8E2A7F
:10F050008E2A8E2AAE2AAE2AAE2AAE2AAE2AAF2A2F
:10F06000AF2AAF2AAF2ACF2AEF2A1033303B513BC9
:10F070007143724392439243924392439243924329
:10F0800092439243F443742BB764DFF7FFFFFFFF13
:10F09000FFFFFFFFFFFFFFFFFFFFFFFFFFFFFFFF80
:10F0A000FFFFFFFFFFFFFFFFFFFFFFFFFFFFFFFF70
:10F0B000FFFFFFFFFFFFFFFFFFFFFFFFFA95774412
:10F0C000F85CF44BD343F44BF443F443F443F44B74
:10F0D000F54B154CF54B154C154C154C154C154C6A
:10F0E000154C154C154C354C154C364C354C364C96
:10F0F000364C364C364C364C364C364C364C764CC0
:10F100005744BA8DFFFFFFFFFFFFFFFFFFFFFFFF29
:10F11000FFFFFFFFFFFFFFFFFFFFFFFFFFFFFFFFFF
:10F12000FFFFFFFFFFFF9CB6B74C9754D53BD53B85
:10F13000D533B533B433B433B533B433B433B43374
:10F14000B433B433B433B4339433B43394339433E7
:10F15000943393339433122B312B5AB6FFFFFFFFB6
:10F16000FFFFFFFFFFFFFFFFFFFFFFFFFFFFFFFFAF
:10F17000FFFFFFFFFFFFFFFFFFFFFFFFFFFFFFFF9F
:10F18000FFFFFFFFFFFFFFFFFFFFFFFFFFFFFFFF8F
:10F19000FFFFFFFFFFFFFFFFFFFFFFFFFFFFFFFF7F
:10F3F000FFFFFFFFFFFFFFFFD66C11238E224C2281
:10F400006D226D226D2A6D2A6D228D2A8D2A8D2AFC
:10F410008E2AAE2A8E2AAE2AAE2AAE2AAF2AAF2A6A
:10F42000CF2AAF2ACF2ACF2ACF2ACF2ACF2AD02A33
:10F43000F02AF0323033313B713B72439243B24396
:10F44000B24BB243B243F44B732B5554BEF7FFFF9C
:10F45000FFFFFFFFFFFFFFFFFFFFFFFFFFFFFFFFBC
:10F46000FFFFFFFFFFFFFFFFFFFFFFFFFFFFFFFFAC
:10F47000FFFFFFFFFFFFFFFFFFFFFFFFFFFFFA950B
:10F48000B74C1865D443D443F44BF443F443F443EA
:10F49000F54BF54BF54B154CF54B154C154C154CE8
:10F4A000154C154C154C154C154C354C354C164C13
:10F4B000364C354C364C364C364C364C164CB75CCC
:10F4C000774C5EDFFFFFFFFFFFFFFFFFFFFFFFFF48
:10F4D000FFFFFFFFFFFFFFFFFFFFFFFFFFFFFFFF3C
:10F4E000FFFFFFFFFFFF586DB74CD5339433B433A4
:10F4F000B433B533B533B433B433B433B433B433D2
:10F50000B433B4339433B433B43394339433943343
:10F5100094339333933332233554FFFFFFFFFFFFC0
:10F52000FFFFFFFFFFFFFFFFFFFFFFFFFFFFFFFFEB
:10F53000FFFFFFFFFFFFFFFFFFFFFFFFFFFFFFFFDB
:10F54000FFFFFFFFFFFFFFFFFFFFFFFFFFFFFFFFCB
:10F55000FFFFFFFFFFFFFFFFFFFFFFFFFFFFFFFFBB
:10F7B000FFFFFFFFFFFFBBC6933BAF1A6D224C223A
:10F7C0006D226D226D2A6D2A8D228D228D2A8E2A20
:10F7D0008E2A8E2A8E2AAE2AAE2AAE2AAE2AAE2AC9
:10F7E000AF2AAF2ACF2ACF2ACF2ACF2ACF2AEF2A71
:10F7F000D02AD02AF02AF02AF02AF02A102B31330E
:10F800003133523B723B9243D343522B144CBEEFE5
:10F81000FFFFFFFFFFFFFFFFFFFFFFFFFFFFFFFFF8
:10F82000FFFFFFFFFFFFFFFFFFFFFFFFFFFFFFFFE8
:10F83000FFFFFFFFFFFFFFFFFFFFFFFFFFFFFFFFD8
:10F84000B985185DD764B343F44BF44BF44BF443E0
:10F85000F443F443F54BF54B154C154CF54B154C57
:10F86000154C154C154C154C154C154C154C154C90
:10F87000354C154C164C364C354C154C564CF85CEA
:10F880007975FFFFFFFFFFFFFFFFFFFFFFFFFFFF98
:10F89000FFFFFFFFFFFFFFFFFFFFFFFFFFFFFFFF78
:10F8A000FFFFFFFF1DCF9644974C9433B533B5331C
:10F8B000B433B433B433B433B433B433B433B43310
:10F8C0009433B433B43394339433943394339333C1
:10F8D00093337333732B532B9995FFFFFFFFFFFF78
:10F8E000FFFFFFFFFFFFFFFFFFFFFFFFFFFFFFFF28
:10F8F000FFFFFFFFFFFFFFFFFFFFFFFFFFFFFFFF18
:10F90000FFFFFFFFFFFFFFFFFFFFFFFFFFFFFFFF07
:10F91000FFFFFFFFFFFFFFFFFFFFFFFFFFFFFFFFF7
:10FB7000FFFFFFFFFFFF1685D0226D224C224C2293
:10FB80004D226D226D226D2A6D2A6D228D2A8D2ABD
:10FB90008D2A8E2AAE2A8E2AAE2AAE2AAE2AAF2A05
:10FBA000AE2ACF2AAF2ACF2ACF2ACF2ACF2AD02ACD
:10FBB000D02AF02AF02AF02AF02AF02AF02AF02A95
:10FBC000F02AF02A112B112B112B3133B01A52339A
:10FBD0005DE7FFFFFFFFFFFFFFFFFFFFFFFFFFFFEF
:10FBE000FFFFFFFFFFFFFFFFFFFFFFFFFFFFFFFF25
:10FBF000FFFFFFFFFFFFFFFFFFFFFFFFFFFFFFFF15
:10FC0000FFFF386D796D5554B343F44BF44BF44317
:10FC1000F443F443F443F54BF44BF54B154CF54BDF
:10FC2000154C154C154C154C154C154C154C354CAC
:10FC3000354C354C354C354C364C154CD764D75477
:10FC4000DCC6FFFFFFFFFFFFFFFFFFFFFFFFFFFF20
:10FC5000FFFFFFFFFFFFFFFFFFFFFFFFFFFFFFFFB4
:10FC6000FFFFFFFF997D764415449433B433B433DA
:10FC7000B433B433B433B433B4339433B433B4336C
:10FC8000943394339433943393339433933393333F
:10FC900073339333942B1544BFEFFFFFFFFFFFFF38
:10FCA000FFFFFFFFFFFFFFFFFFFFFFFFFFFFFFFF64
:10FCB000FFFFFFFFFFFFFFFFFFFFFFFFFFFFFFFF54
:10FCC000FFFFFFFFFFFFFFFFFFFFFFFFFFFFFFFF44
:10FCD000FFFFFFFFFFFFFFFFFFFFFFFFFFFFFFFF34
:10FF3000FFFFFFFF5DE7B24B6E1A6C224C224C2292
:10FF40004C226D226D226D2A6D2A8D226D228D2A02
:10FF50008E2A8E2A8E2A8E2AAE2AAE2AAE2AAE2A61
:10FF6000AF2AAF2ACF2AAF2ACF2ACF2ACF2ACF2A29
:10FF7000F02AD02AF02AF02AF02AF02A102BF02AB0
:10FF8000112B112B112B112B112B112B112B6E124D
:10FF9000B01A1CDFFFFFFFFFFFFFFFFFFFFFFFFFA8
:10FFA000FFFFFFFFFFFFFFFFFFFFFFFFFFFFFFFF61
:10FFB000FFFFFFFFFFFFFFFFFFFFFFFFFFFFFFFF51
:10FFC000FFFF3DD7D754586DD443D44BF44BF44B7B
:10FFD000F44BF44B144C154C144C154C154C154C5F
:10FFE000154C154C154C15441544F543F543F54394
:10FFF000F543F443D43BD53BB433D43B175DF85CB5
:0200000490F278
:10000000FFFFFFFFFFFFFFFFFFFFFFFFFFFFFFFF00
:10001000FFFFFFFFFFFFFFFFFFFFFFFFFFFFFFFFF0
:10002000FFFF7EE77644764C9433B433B433B43375
:10003000B433B4339433B433B433B43394339433E8
:10004000943394339333943393339333733393339D
:1000500073339433D52B387DFFFFFFFFFFFFFFFF86
:10006000FFFFFFFFFFFFFFFFFFFFFFFFFFFFFFFFA0
:10007000FFFFFFFFFFFFFFFFFFFFFFFFFFFFFFFF90
:10008000FFFFFFFFFFFFFFFFFFFFFFFFFFFFFFFF80
:10009000FFFFFFFFFFFFFFFFFFFFFFFFFFFFFFFF70
:1002F000FFFFFFFF779DAE224C1A4C224C224C226E
:100300006D226D226D226D226D2A6D2A6D228D2245
:100310008D2A8E2A8E2AAE2A8E2AAE2AAE2AAE2A9E
:10032000AE2AAF2AAF2ACF2ACF2ACF2ACF2ACF2A66
:10033000CF2AF02AF02AF02AF02AF02AF02A102BED
:10034000F02A112B112B112B112B112B312B1133C7
:100350004E124E12DCCEFFFFFFFFFFFFFFFFFFFF3D
:10036000FFFFFFFFFFFFFFFFFFFFFFFFFFFFFFFF9D
:10037000FFFFFFFFFFFFFFFFFFFFFFFFFFFFFFFF8D
:10038000FFFFFFFF797DB74C554C523393339333C6
:10039000733393339333933393339333933393334D
:1003A000933393339333933393339433943394331A
:1003B0009333943394339433732B564CB74C1A9E27
:1003C000FFFFFFFFFFFFFFFFFFFFFFFFFFFFFFFF3D
:1003D000FFFFFFFFFFFFFFFFFFFFFFFFFFFFFFFF2D
:1003E000FFFFFB9516341544732BB433B4339433A9
:1003F000B433B433B4339433943394339433943365
:1004000094339333933393337333933393337333FB
:100410007333D633373CFDC6FFFFFFFFFFFFFFFFFF
:10042000FFFFFFFFFFFFFFFFFFFFFFFFFFFFFFFFDC
:10043000FFFFFFFFFFFFFFFFFFFFFFFFFFFFFFFFCC
:10044000FFFFFFFFFFFFFFFFFFFFFFFFFFFFFFFFBC
:10045000FFFFFFFFFFFFFFFFFFFFFFFFFFFFFFFFAC
:1006B000FFFFFFFFF25B0C124C224C224C224C221B
:1006C0004C224C226D226D226D2A6D2A8D2A6D22BC
:1006D0008D2A8D2A8D2A8E2AAE2A8E2AAE2AAE2AFD
:1006E000AE2AAE2AAF2AAF2AAF2ACF2ACF2ACF2AE4
:1006F000CF2ACF2ACF2AF02AF02AF02AF02AF02A8D
:10070000102B102B102B112B112B112B312B3233C3
:1007100011332D12EC099BC6FFFFFFFFFFFFFFFF08
:10072000FFFFFFFFFFFFFFFFFFFFFFFFFFFFFFFFD9
:10073000FFFFFFFFFFFFFFFFFFFFFFFFFFFFFFFFC9
:10074000FFFFFFFFBEEF3634974C5233522B52332C
:10075000522B532B732B73337333733373337333C2
:1007600073337333733393339333943393339333B8
:1007700094339433943394339333B75477449EEF44
:10078000FFFFFFFFFFFFFFFFFFFFFFFFFFFFFFFF79
:10079000FFFFFFFFFFFFFFFFFFFFFFFFFFFFFFFF69
:1007A000DFF7774C363CB4339433B433B4339433FB
:1007B0009433943394339433933393339433933304
:1007C0009333933373337333933373337333733399
:1007D000943316341965FFFFFFFFFFFFFFFFFFFF94
:1007E000FFFFFFFFFFFFFFFFFFFFFFFFFFFFFFFF19
:1007F000FFFFFFFFFFFFFFFFFFFFFFFFFFFFFFFF09
:10080000FFFFFFFFFFFFFFFFFFFFFFFFFFFFFFFFF8
:10081000FFFFFFFFFFFFFFFFFFFFFFFFFFFFFFFFE8
:100A7000FFFF19B68D2AEB114C224C224C224C223E
:100A80004C226C224C226D226D226D2A6D2A8D2AF9
:100A90008D228D2A8E2A8E2A8E2AAE2AAE2AAE2A40
:100AA000AE2AAE2AAE2AAF2ACF2AAF2ACF2ACF2A21
:100AB000CF2ACF2AF02AD02AF02AF02AF02AF02AC8
:100AC000F02AF02A102B102B112B112B112B112B8C
:100AD000523310332C12AB0139B6FFFFFFFFFFFF7B
:100AE000FFFFFFFFFFFFFFFFFFFFFFFFFFFFFFFF16
:100AF000FFFFFFFFFFFFFFFFFFFFFFFFFFFFFFFF06
:100B0000FFFFFFFFFFFF99853734F53B322B723330
:100B100072335233733373337333733373337333C7
:100B200073339333933373339333933393339333D5
:100B30009433933393337333F53B97443975FFFF05
:100B4000FFFFFFFFFFFFFFFFFFFFFFFFFFFFFFFFB5
:100B5000FFFFFFFFFFFFFFFFFFFFFFFFFFFFFFFFA5
:100B60009CB6D5231644733394339433943394331F
:100B70009433933393339433933393339333933343
:100B80007333733393337333733373337333733315
:100B9000F53B573C3BA6FFFFFFFFFFFFFFFFFFFFBB
:100BA000FFFFFFFFFFFFFFFFFFFFFFFFFFFFFFFF55
:100BB000FFFFFFFFFFFFFFFFFFFFFFFFFFFFFFFF45
:100BC000FFFFFFFFFFFFFFFFFFFFFFFFFFFFFFFF35
:100BD000FFFFFFFFFFFFFFFFFFFFFFFFFFFFFFFF25
:100E3000FFFF74742C1A4C224C224C224C224C2260
:100E40004C224C226D226D226D226D226D2A6D2A5C
:100E50006D2A8D228D2A8D2A8E2A8E2A8E2AAE2ADE
:100E6000AE2AAE2AAE2AAE2AAF2ACF2AAF2ACF2A7E
:100E7000CF2ACF2ACF2AEF2AD02AF02AF02AF02A26
:100E8000F02AF02AF02A102B102B112B112B112BEA
:100E9000112B5233102B0C124901B8A5FFFFFFFF95
:100EA000FFFFFFFFFFFFFFFFFFFFFFFFFFFFFFFF52
:100EB000FFFFFFFFFFFFFFFFFFFFFFFFFFFFFFFF42
:100EC000FFFFFFFFFFFF7EE7F62B3644323352333E
:100ED0005233723353337233733373337333733325
:100EE0007333733373337333933373337333933392
:100EF00093339333933373335644F62BFDC6FFFF7E
:100F0000FFFFFFFFFFFFFFFFFFFFFFFFFFFFFFFFF1
:100F1000FFFFFFFFFFFFFFFFFFFFFFFFFFFFDFFF01
:100F2000D85CD62BB43393339433933393339333C6
:100F300094339333933393339333733373339333C0
:100F40007333733373337333733373335333933371
:100F50005744F85CFFFFFFFFFFFFFFFFFFFFFFFFAE
:100F6000FFFFFFFFFFFFFFFFFFFFFFFFFFFFFFFF91
:100F7000FFFFFFFFFFFFFFFFFFFFFFFFFFFFFFFF81
:100F8000FFFFFFFFFFFFFFFFFFFFFFFFFFFFFFFF71
:100F9000FFFFFFFFFFFFFFFFFFFFFFFFFFFFFFFF61
:1011F000FCD6303B2C1A4C224C224C224C224C2246
:101200004C224C226C224C226D226D226D2A6D2ABA
:101210008D2A6D228D2A8D2A8E2A8E2AAE2A8E2A1A
:10122000AE2AAE2AAE2AAE2AAE2AAF2ACF2ACF2ABB
:10123000CF2ACF2ACF2ACF2AEF2AD02AF02AF02A83
:10124000F02AF02AF02AF02A102B102B112B112B48
:10125000112B112B5233102B0C1A2801569DFFFF16
:10126000FFFFFFFFFFFFFFFFFFFFFFFFFFFFFFFF8E
:10127000FFFFFFFFFFFFFFFFFFFFFFFFFFFFFFFF7E
:10128000FFFFFFFFFFFFFFFFB854F72B9333322B15
:1012900052335233523372335333723373337333A3
:1012A00073337333733373337333733393337333EE
:1012B0007333933373339433373C774CFFFFFFFF23
:1012C000FFFFFFFFFFFFFFFFFFFFFFFFFFFFFFFF2E
:1012D000FFFFFFFFFFFFFFFFFFFFFFFFFFFF3DD708
:1012E000B623F63373339333933393339333933378
:1012F000933393337333733373339333733373335E
:101300007333733373337333733352335233F53B65
:10131000974CDA95FFFFFFFFFFFFFFFFFFFFFFFF87
:10132000FFFFFFFFFFFFFFFFFFFFFFFFFFFFFFFFCD
:10133000FFFFFFFFFFFFFFFFFFFFFFFFFFFFFFFFBD
:10134000FFFFFFFFFFFFFFFFFFFFFFFFFFFFFFFFAD
:10135000FFFFFFFFFFFFFFFFFFFFFFFFFFFFFFFF9D
:1015B000368D8E224C224C224C224C224C224C2224
:1015C0004C224C224C226D226D226D226D226D2AFE
:1015D0006D2A8D2A8D228D2A8D2A8E2A8E2AAE2A58
:1015E000AE2AAE2AAE2AAE2AAF2AAF2AAF2AAF2A37
:1015F000CF2ACF2ACF2ACF2ACF2AEF2AD02AF02AE1
:10160000F02AF02AF02AF02AF02A102B102B112BA6
:10161000112B112B112B523331334D1A4901168DD9
:10162000FFFFFFFFFFFFFFFFFFFFFFFFFFFFFFFFCA
:10163000FFFFFFFFFFFFFFFFFFFFFFFFFFFFFFFFBA
:10164000FFFFFFFFFFFFFFFFFA9D751BB433322B37
:101650005233523352335233523372335233533341
:10166000723373337333733373337333733373334B
:10167000733373337333F53B9623FB95FFFFFFFF03
:10168000FFFFFFFFFFFFFFFFFFFFFFFFFFFFFFFF6A
:10169000FFFFFFFFFFFFFFFFFFFFFFFFFFFF597D82
:1016A000541BB433733393339333733373337333C0
:1016B00073339333733373337333733373337333DA
:1016C0007333733373337233533352337233764C11
:1016D000F85C7EDFFFFFFFFFFFFFFFFFFFFFFFFF65
:1016E000FFFFFFFFFFFFFFFFFFFFFFFFFFFFFFFF0A
:1016F000FFFFFFFFFFFFFFFFFFFFFFFFFFFFFFFFFA
:10170000FFFFFFFFFFFFFFFFFFFFFFFFFFFFFFFFE9
:10171000FFFFFFFFFFFFFFFFFFFFFFFFFFFFFFFFD9
:10196000FFFFFFFFFFFFFFFFFFFFFFFFFFFFBEF7D0
:10197000F25B6D1A6D224C224C224C224C224C22DE
:101980004C224C224C224C224C226D226D226D2284
:101990006D2A6D2A6D228D2A8D2A8D2A8E2A8E2AF5
:1019A0008E2AAE2AAE2AAE2AAE2AAE2AAF2ACF2A75
:1019B000AF2ACF2ACF2ACF2ACF2ACF2AEF2AF02A3E
:1019C000F02AF02AF02AF02A102BF02A102B102BE4
:1019D000112B112B112B112B323331338E226A0133
:1019E000D57CFFFFFFFFFFFFFFFFFFFFFFFFFFFFB4
:1019F000FFFFFFFFFFFFFFFFFFFFFFFFFFFFFFFFF7
:101A0000FFFFFFFFFFFFFFFF5DDF331B9333323329
:101A1000523352335233523352335233523372337E
:101A200052335333723373337333733373337333C8
:101A3000733373337333D533952BBFF7FFFFFFFF3A
:101A4000FFFFFFFFFFFFFFFFFFFFFFFFFFFFFFFFA6
:101A5000FFFFFFFFFFFFFFFFFFFFFFFFBEEF742B46
:101A6000942B9333733373337333933373337333ED
:101A70007333733373337333733373337333733336
:101A8000733372335333723352335233D43BF8547B
:101A9000B985FFFFFFFFFFFFFFFFFFFFFFFFFFFF16
:101AA000FFFFFFFFFFFFFFFFFFFFFFFFFFFFFFFF46
:101AB000FFFFFFFFFFFFFFFFFFFFFFFFFFFFFFFF36
:101AC000FFFFFFFFFFFFFFFFFFFFFFFFFFFFFFFF26
:101AD000FFFFFFFFFFFFFFFFFFFFFFFFFFFFFFFF16
:101D2000FFFFFFFFFFFFFFFFFFFFFFFFFFFFF9AD1B
:101D3000F0326D224C224C224C224C224C224C225E
:101D40004C224C224C224C226C224C226D226D22C1
:101D50006D2A6D2A8D2A6D228D2A8D2A8D2A8E2A32
:101D6000AE2A8E2AAE2AAE2AAE2AAE2AAE2AAF2AD2
:101D7000CF2AAF2ACF2ACF2ACF2ACF2ACF2ACF2ABB
:101D8000F02AF02AF02AF02AF02AF02AF02A102B62
:101D9000102B112B112B112B112B3133312BAE2A80
:101DA0008B019474FFFFFFFFFFFFFFFFFFFFFFFFAB
:101DB000FFFFFFFFFFFFFFFFFFFFFFFFFFFFFFFF33
:101DC000FFFFFFFFFFFFFFFFFFFF7233322B523396
:101DD00032335233523352335233523352335233FB
:101DE0005233723352335233533372337333733348
:101DF000733373339333331BD76CFFFFFFFFFFFF46
:101E0000FFFFFFFFFFFFFFFFFFFFFFFFFFFFFFFFE2
:101E1000FFFFFFFFFFFFFFFFFFFFFFFFF9A5B10A75
:101E20009333733373337333733373337333733362
:101E30007333733373337333733373337233533393
:101E400052335233723352335233522B764C385D05
:101E5000DCBEFFFFFFFFFFFFFFFFFFFFFFFFFFFFF6
:101E6000FFFFFFFFFFFFFFFFFFFFFFFFFFFFFFFF82
:101E7000FFFFFFFFFFFFFFFFFFFFFFFFFFFFFFFF72
:101E8000FFFFFFFFFFFFFFFFFFFFFFFFFFFFFFFF62
:101E9000FFFFFFFFFFFFFFFFFFFFFFFFFFFFFFFF52
:1020E000FFFFFFFFFFFFFFFFFFFFFFFFFFFFB574D5
:1020F000AF226D224C224C224C224C224C224C22EC
:102100004C224C224C224C224C226D226D226D22FC
:102110006D226D2A6D2A8D2A8D228D2A8E2A8E2A75
:102120008E2AAE2A8E2AAE2AAE2AAE2AAE2AAE2A2F
:10213000AF2ACF2AAF2ACF2ACF2ACF2ACF2AD02A16
:10214000CF2AF02AF02AF02AF02AF02AF02AF02AE0
:10215000102B102B112B112B112B112B312B313359
:10216000CF2A8B019474FFFFFFFFFFFFFFFFFFFFEC
:10217000FFFFFFFFFFFFFFFFFFFFFFFFFFFFFFFF6F
:10218000FFFFFFFFFFFFFFFFFFFFD34BB01A5233EC
:102190005233322B3233523352335233523352335F
:1021A00052335233523352337233523352335333E6
:1021B00072337333522BB112FCCEFFFFFFFFFFFFD0
:1021C000FFFFFFFFFFFFFFFFFFFFFFFFFFFFFFFF1F
:1021D000FFFFFFFFFFFFFFFFFFFFDFFFB343D11A4A
:1021E00073337333733373337333733373337333BF
:1021F0007333733373337233533352335233723313
:102200005233523352335233522B933BD754797556
:10221000FFFFFFFFFFFFFFFFFFFFFFFFFFFFFFFFCE
:10222000FFFFFFFFFFFFFFFFFFFFFFFFFFFFFFFFBE
:10223000FFFFFFFFFFFFFFFFFFFFFFFFFFFFFFFFAE
:10224000FFFFFFFFFFFFFFFFFFFFFFFFFFFFFFFF9E
:1024A000FFFFFFFFFFFFFFFFFFFFFFFFBBCE9243DA
:1024B0008E226D2A4C224C224C224C224C224C2241
:1024C0004C224C224C224C224C224C224C226D227B
:1024D0006D226D226D2A6D2A6D2A8D228D2A8D2AFC
:1024E0008E2A8E2AAE2A8E2AAE2AAE2AAE2AAE2A8C
:1024F000AE2AAF2ACF2AAF2ACF2ACF2ACF2ACF2A75
:10250000CF2ACF2AF02AF02AF02AF02AF02AF02A3D
:10251000102BF02A102B112B112B112B112B312BDF
:102520003133F02AAC0119AEFFFFFFFFFFFFFFFFC1
:10253000FFFFFFFFFFFFFFFFFFFFFFFFFFFFFFFFAB
:10254000FFFFFFFFFFFFFFFFFFFF54644D12312B22
:102550003233322B522B322B3233523352335233EB
:102560005233523352335233523352335233723323
:1025700073335233B01A923BFFFFFFFFFFFFFFFFA1
:10258000FFFFFFFFFFFFFFFFFFFFFFFFFFFFFFFF5B
:10259000FFFFFFFFFFFFFFFFFFFFBBC64E0A322B0F
:1025A00073337333733373337333733372337233FD
:1025B00052335333523352337233523352335233D2
:1025C000523352335233522B32331544D8543B9E3C
:1025D000FFFFFFFFFFFFFFFFFFFFFFFFFFFFFFFF0B
:1025E000FFFFFFFFFFFFFFFFFFFFFFFFFFFFFFFFFB
:1025F000FFFFFFFFFFFFFFFFFFFFFFFFFFFFFFFFEB
:10260000FFFFFFFFFFFFFFFFFFFFFFFFFFFFFFFFDA
:10286000FFFFFFFFFFFFFFFFFFFFFFFF578DF02A76
:102870006D224C224C224C224C224C224C224C22C7
:102880004C224C224C224C224C224C226C224C22B8
:102890006D226D226D2A6D2A8D2A6D228D2A8D2A38
:1028A0008D2A8E2A8E2AAE2AAE2AAE2AAE2AAE2AC9
:1028B000AF2AAE2AAF2ACF2ACF2ACF2ACF2ACF2AB1
:1028C000CF2AD02ACF2AF02AF02AF02AF02AF02A9A
:1028D000F02A102BF02A112B102B112B112B112B5E
:1028E000312B31336E1A924BDFFFFFFFFFFFFFFFEB
:1028F000FFFFFFFFFFFFFFFFFFFFFFFFFFFFFFFFE8
:10290000FFFFFFFFFFFFFFFFFFFF7474CB09112BD9
:102910005233312B31333233322B522B322B323371
:10292000523352335233523352335233523352337F
:102930007333102BEC01B89DFFFFFFFFFFFFFFFF7C
:10294000FFFFFFFFFFFFFFFFFFFFFFFFFFFFFFFF97
:10295000FFFFFFFFFFFFFFFFFFFF33642D0A52332E
:1029600073337233723352335333523352335233DD
:10297000723352335233523352335233523352330F
:10298000523352335233323352337644F85CBEEF13
:10299000FFFFFFFFFFFFFFFFFFFFFFFFFFFFFFFF47
:1029A000FFFFFFFFFFFFFFFFFFFFFFFFFFFFFFFF37
:1029B000FFFFFFFFFFFFFFFFFFFFFFFFFFFFFFFF27
:1029C000FFFFFFFFFFFFFFFFFFFFFFFFFFFFFFFF17
:102C2000FFFFFFFFFFFFFFFFFFFF7EE7135CAF2209
:102C30006D222C224C224C224C224C224C224C2223
:102C40004C224C224C224C224C224C224C226C22F4
:102C50004C226D226D226D2A6D228D226D228D2ACD
:102C60008D2A8D2A8E2A8E2A8E2AAE2AAE2AAE2A46
:102C7000AE2AAE2AAF2AAF2AAF2ACF2ACF2ACF2A2E
:102C8000CF2ACF2AD02ACF2AF02AF02AF02AF02AF7
:102C9000F02AF02A102BF02A112B102B112B112BBC
:102CA000112B112BD02AF02ABEF7FFFFFFFFFFFFE9
:102CB000FFFFFFFFFFFFFFFFFFFFFFFFFFFFFFFF24
:102CC000FFFFFFFFFFFFFFFFFFFF53748A01F02AA2
:102CD0005233313331333233313332333233522B97
:102CE000322B323352335233523352335233523304
:102CF00052334D1A4D1AFFFFFFFFFFFFFFFFFFFF8B
:102D0000FFFFFFFFFFFFFFFFFFFFFFFFFFFFFFFFD3
:102D1000FFFFFFFFFFFFFFFF5DE72D12AE227333C2
:102D2000533352335233723352335233523352335A
:102D3000523352335233523352335233523352336B
:102D400052335233322B312BB43B77449985FFFFFA
:102D5000FFFFFFFFFFFFFFFFFFFFFFFFFFFFFFFF83
:102D6000FFFFFFFFFFFFFFFFFFFFFFFFFFFFFFFF73
:102D7000FFFFFFFFFFFFFFFFFFFFFFFFFFFFFFFF63
:102D8000FFFFFFFFFFFFFFFFFFFFFFFFFFFFFFFF53
:102FE000FFFFFFFFFFFFFFFFFFFFB8A511338D229B
:102FF0004C222C222C222C222C222C222C222C2241
:103000002C222C222C222C222C222C224C224C2210
:103010004C224C224C226D226D226D226D226D229B
:103020006D228D228D228D228E2A8E2A8E2AAE2A04
:10303000AE2AAE2AAE2AAE2AAF2AAF2AAF2AAF2ACC
:10304000CF2ACF2ACF2ACF2AEF2AD02AF02AF02A55
:10305000F02AF02AF02A102BF02A102B102B112B1B
:10306000112B11338F1A7243DFF7FFFFFFFFFFFFB2
:10307000FFFFFFFFFFFFFFFFFFFFFFFFFFFFFFFF60
:10308000FFFFFFFFFFFFFFFFFFFF3364CA09102BA5
:103090003233312B312B313331333233313331331E
:1030A0003233322B522B322B32335233523373336F
:1030B000CF2A6901536CFFFFFFFFFFFFFFFFFFFFF8
:1030C000FFFFFFFFFFFFFFFFFFFFFFFFFFFFFFFF10
:1030D000FFFFFFFFFFFFFFFF158D6A01102B73330A
:1030E00052335233523352335233523352335233B8
:1030F00052335233523352335233523332333233E8
:10310000322B522B312B312B153C7744FDC6FFFF60
:10311000FFFFFFFFFFFFFFFFFFFFFFFFFFFFFFFFBF
:10312000FFFFFFFFFFFFFFFFFFFFFFFFFFFFFFFFAF
:10313000FFFFFFFFFFFFFFFFFFFFFFFFFFFFFFFF9F
:10314000FFFFFFFFFFFFFFFFFFFFFFFFFFFFFFFF8F
:1033A000FFFFFFFFFFFFFFFFFFFF756CAF22CF2A7C
:1033B000AF2ACF2ACF2ACF2ACF2ACF2ACF2ACF2A65
:1033C000CF2ACF2ACF2ACF2ACF2ACF2ACF2ACF2A35
:1033D000CF2ACF2ACF2ACF2ACF2ACF2ACF2ACF2A25
:1033E000CF2ACF2ACF2ACF2AD02AD02AD02AD02A11
:1033F000F02AF02AF02AF02AF02AF02AF02AF02AFD
:10340000F02AF02AF02AF02AF02AF02AF02AF02AEC
:10341000F02AF02AF02AF02AF02AF02AF02AF02ADC
:10342000F032D02A2E0AF9ADFFFFFFFFFFFFFFFFAA
:10343000FFFFFFFFFFFFFFFFFFFFFFFFFFFFFFFF9C
:10344000FFFFFFFFFFFFFFFFFFFFB1532C12112B08
:10345000312B112B112B312B312B312B3133312BC4
:103460003233313332333233322B522B322B52330D
:103470006D22AA091CDFFFFFFFFFFFFFFFFFFFFF19
:10348000FFFFFFFFFFFFFFFFFFFFFFFFFFFFFFFF4C
:10349000FFFFFFFFFFFFDFF78D2AEB11523373337E
:1034A00052335233523352335233523352335233F4
:1034B0005233523352333233322B322B522B322B84
:1034C00032333133312B7333373CF864FFFFFFFF66
:1034D000FFFFFFFFFFFFFFFFFFFFFFFFFFFFFFFFFC
:1034E000FFFFFFFFFFFFFFFFFFFFFFFFFFFFFFFFEC
:1034F000FFFFFFFFFFFFFFFFFFFFFFFFFFFFFFFFDC
:10350000FFFFFFFFFFFFFFFFFFFFFFFFFFFFFFFFCB
:10376000FFFFFFFFFFFFFFFFDFF795748F1AAF2208
:10377000D022B022B022B022B022B022B022B02299
:10378000B022B022B022B022B022B022B022B022A9
:10379000B022B022B022B022B022B022B022B02299
:1037A000B022B022B022B022B022B022B022AF228A
:1037B000AF22AF22AF22AF22AF22AF22AF22AF2281
:1037C000AF22AF22AF22AF22AF22AF22AF22AF2271
:1037D000AF22AF22AF22AF22AF22AF22AF22AF2261
:1037E000AF221033D9A5FFFFFFFFFFFFFFFFFFFF51
:1037F000FFFFFFFFFFFFFFFFFFFFFFFFFFFFFFFFD9
:10380000FFFFFFFFFFFFFFFFFFFF103B8E22112B8B
:10381000112B112B312B112B112B312B312B312B48
:103820003133312B312B3233313332335233112B8D
:103830000C12914BFFFFFFFFFFFFFFFFFFFFFFFF9A
:10384000FFFFFFFFFFFFFFFFFFFFFFFFFFFFFFFF88
:10385000FFFFFFFFFFFF19B68A01CF2A73335233F0
:103860005233523352335233523352335233323350
:10387000322B322B322B522B323332333133313322
:10388000322B312B312BB43337341B9EFFFFFFFF1C
:10389000FFFFFFFFFFFFFFFFFFFFFFFFFFFFFFFF38
:1038A000FFFFFFFFFFFFFFFFFFFFFFFFFFFFFFFF28
:1038B000FFFFFFFFFFFFFFFFFFFFFFFFFFFFFFFF18
:1038C000FFFFFFFFFFFFFFFFFFFFFFFFFFFFFFFF08
:103B2000FFFFFFFFFFFFFFFFFFFFDFF7DCD69BC6B6
:103B3000BBCEBBCEBBCEBBCEBBCEBBCEBBCEBBCE3D
:103B4000BBCEBBCEBBCEBBCEBBCEBBCEBBCEBBCE2D
:103B5000BBCEBBCEBBCEBBCEBBCEBBCEBBCEBBCE1D
:103B6000BBCEBBCEBBCEBBCEBBCEBBCEBBCEBBCE0D
:103B7000BBCEBBCEBBCEBBCEBBCEBBCEBBCEBBCEFD
:103B8000BBCEBBCEBBCEBBCEBBCEBBCEBBCEBBCEED
:103B9000BBCEBBCEBBCEBBCEBBCEBBCEBBC6BBC6ED
:103BA000FCD6FFFFFFFFFFFFFFFFFFFFFFFFFFFF51
:103BB000FFFFFFFFFFFFFFFFFFFFFFFFFFFFFFFF15
:103BC000FFFFFFFFFFFFFFFF9EEF8F22F02A112B69
:103BD000112B112B112B112B312B112B112B112BE5
:103BE000312B312B312B3133312B312B5233F02A06
:103BF000EC093AB6FFFFFFFFFFFFFFFFFFFFFFFFEC
:103C0000FFFFFFFFFFFFFFFFFFFFFFFFFFFFFFFFC4
:103C1000FFFFFFFFFFFFB253EC0931335233323362
:103C2000323332333233322B322B322B322B522B74
:103C300032333233323331333133312B312B313371
:103C4000312B312B322BD633774CDFF7FFFFFFFFC1
:103C5000FFFFFFFFFFFFFFFFFFFFFFFFFFFFFFFF74
:103C6000FFFFFFFFFFFFFFFFFFFFFFFFFFFFFFFF64
:103C7000FFFFFFFFFFFFFFFFFFFFFFFFFFFFFFFF54
:103C8000FFFFFFFFFFFFFFFFFFFFFFFFFFFFFFFF44
:103F8000FFFFFFFFFFFFFFFF5ABE6E121033102B23
:103F9000102B112B112B112B112B112B112B312B22
:103FA000112B112B112B312B312B312B3133AF2A0C
:103FB000F032FFFFFFFFFFFFFFFFFFFFFFFFFFFFED
:103FC000FFFFFFFFFFFFFFFFFFFFFFFFFFFFFFFF01
:103FD000FFFFFFFF3CDF2D12AF2A5233322B522B53
:103FE000322B322B322B32333233323331333133C3
:103FF0003133312B312B312B3133312B312B312BD1
:10400000312B112B522BB52B597DFFFFFFFFFFFFEB
:10401000FFFFFFFFFFFFFFFFFFFFFFFFFFFFFFFFB0
:10402000FFFFFFFFFFFFFFFFFFFFFFFFFFFFFFFFA0
:10403000FFFFFFFFFFFFFFFFFFFFFFFFFFFFFFFF90
:10404000FFFFFFFFFFFFFFFFFFFFFFFFFFFFFFFF80
:10434000FFFFFFFFFFFFFFFFB5746F1A102BF02A6E
:10435000F02A102B102B112B112B112B112B112BA1
:10436000112B112B312B112B112B312B31334E12E1
:10437000378DFFFFFFFFFFFFFFFFFFFFFFFFFFFF87
:10438000FFFFFFFFFFFFFFFFFFFFFFFFFFFFFFFF3D
:10439000FFFFFFFFF6840D0A3133523331333133DF
:1043A000313331333133312B312B312B312B312B15
:1043B0003133312B312B312B312B312B112B112B55
:1043C000112B3133532BB4331DCFFFFFFFFFFFFF02
:1043D000FFFFFFFFFFFFFFFFFFFFFFFFFFFFFFFFED
:1043E000FFFFFFFFFFFFFFFFFFFFFFFFFFFFFFFFDD
:1043F000FFFFFFFFFFFFFFFFFFFFFFFFFFFFFFFFCD
:10440000FFFFFFFFFFFFFFFFFFFFFFFFFFFFFFFFBC
:10470000FFFFFFFFFFFFFFFF1133D02AF02AF02A3F
:10471000102BF02AF02A102B112B102B112B112B00
:10472000112B112B112B112B112B312BF02A8F1A3E
:104730009EEFFFFFFFFFFFFFFFFFFFFFFFFFFFFFFA
:10474000FFFFFFFFFFFFFFFFFFFFFFFFFFFFFFFF79
:10475000FFFFBEF7F032AF223233322B312B312B39
:10476000312B312B3133312B312B312B312B312B61
:10477000312B312B112B112B112B112B112B112B19
:10478000112B312B32239664FFFFFFFFFFFFFFFF4A
:10479000FFFFFFFFFFFFFFFFFFFFFFFFFFFFFFFF29
:1047A000FFFFFFFFFFFFFFFFFFFFFFFFFFFFFFFF19
:1047B000FFFFFFFFFFFFFFFFFFFFFFFFFFFFFFFF09
:1047C000FFFFFFFFFFFFFFFFFFFFFFFFFFFFFFFFF9
:104AC000FFFFFFFFFFFF5ABE6E121033F02AF02ADD
:104AD000F02AF02A102BF02AF02A102B102B102B82
:104AE000102B112B112B112B112B11336F1A346436
:104AF000FFFFFFFFFFFFFFFFFFFFFFFFFFFFFFFFC6
:104B0000FFFFFFFFFFFFFFFFFFFFFFFFFFFFFFFFB5
:104B1000FFFFF9AD2E0A3133312B312B312B312BE5
:104B2000312B312B312B312B312B112B112B112B05
:104B3000112B112B312B112B112B112B112B112B75
:104B4000112BF122112B9BC6FFFFFFFFFFFFFFFF81
:104B5000FFFFFFFFFFFFFFFFFFFFFFFFFFFFFFFF65
:104B6000FFFFFFFFFFFFFFFFFFFFFFFFFFFFFFFF55
:104B7000FFFFFFFFFFFFFFFFFFFFFFFFFFFFFFFF45
:104B8000FFFFFFFFFFFFFFFFFFFFFFFFFFFFFFFF35
:104E8000FFFFFFFFFFFFF3538F22F02AF02AF02AE3
:104E9000F02AF02AF02AF02AF02AF02AF02AF02A42
:104EA000102B102B102B102B112B11334E12BBC6B5
:104EB000FFFFFFFFFFFFFFFFFFFFFFFFFFFFFFFF02
:104EC000FFFFFFFFFFFFFFFFFFFFFFFFFFFFFFFFF2
:104ED000FFFFB24B8F1A3133112B112B112B112BDA
:104EE000112B112B112B112B112B112B112B112BE2
:104EF000112B112B112B112B112B112B112B112BD2
:104F0000F02AAF1A7564FFFFFFFFFFFFFFFFFFFFEF
:104F1000FFFFFFFFFFFFFFFFFFFFFFFFFFFFFFFFA1
:104F2000FFFFFFFFFFFFFFFFFFFFFFFFFFFFFFFF91
:104F3000FFFFFFFFFFFFFFFFFFFFFFFFFFFFFFFF81
:104F4000FFFFFFFFFFFFFFFFFFFFFFFFFFFFFFFF71
:10524000FFFFFFFFDCCE6E1AF032CF2AF02AF02AE1
:10525000F02AF02AF02AF02AF02AF02AF02AF02A7E
:10526000F02AF02AF02A102B102BAF22513BFFFF1F
:10527000FFFFFFFFFFFFFFFFFFFFFFFFFFFFFFFF3E
:10528000FFFFFFFFFFFFFFFFFFFFFFFFFFFFFFFF2E
:10529000FCD66E1AF032112B112B112B112B112B66
:1052A000112B112B112B112B112B112B112B112B1E
:1052B000112B112B112B112B102B102B112BF02A32
:1052C0006D1AEF2A3DDFFFFFFFFFFFFFFFFFFFFF2C
:1052D000FFFFFFFFFFFFFFFFFFFFFFFFFFFFFFFFDE
:1052E000FFFFFFFFFFFFFFFFFFFFFFFFFFFFFFFFCE
:1052F000FFFFFFFFFFFFFFFFFFFFFFFFFFFFFFFFBE
:10530000FFFFFFFFFFFFFFFFFFFFFFFFFFFFFFFFAD
:10560000FFFFFFFFB24BAF22F02ACF2ACF2AD02ACA
:10561000F02AF02AF02AF02AF02AF02AF02AF02ABA
:10562000F02AF02AF02AF02A10334E12989DFFFF3C
:10563000FFFFFFFFFFFFFFFFFFFFFFFFFFFFFFFF7A
:10564000FFFFFFFFFFFFFFFFFFFFFFFFFFFFFFFF6A
:10565000B5744E121133112B112B112B112B112B51
:10566000112B112B112B112B112B112B112B102B5B
:10567000102B102B102B102B102B102BF02A4D1A47
:105680002C12979DFFFFFFFFFFFFFFFFFFFFFFFFB4
:10569000FFFFFFFFFFFFFFFFFFFFFFFFFFFFFFFF1A
:1056A000FFFFFFFFFFFFFFFFFFFFFFFFFFFFFFFF0A
:1056B000FFFFFFFFFFFFFFFFFFFFFFFFFFFFFFFFFA
:1056C000FFFFFFFFFFFFFFFFFFFFFFFFFFFFFFFFEA
:1059C000FFFFD9A54E12F032CF2ACF2ACF2ACF2AF5
:1059D000CF2ACF2AD02AF02AF02AF02AF02AF02A59
:1059E000F02AF02AF02AF02AF02AAF22DFF7FFFF90
:1059F000FFFFFFFFFFFFFFFFFFFFFFFFFFFFFFFFB7
:105A0000FFFFFFFFFFFFFFFFFFFFFFFFFFFF9EEF17
:105A1000CF2AF02A112B112B112B112B112B102B0C
:105A2000102B102B102B102B102B102B102BF02ABF
:105A3000F02AF02AF02AF02A102BF02A6D22CA113F
:105A4000536CFFFFFFFFFFFFFFFFFFFFFFFFFFFFA5
:105A5000FFFFFFFFFFFFFFFFFFFFFFFFFFFFFFFF56
:105A6000FFFFFFFFFFFFFFFFFFFFFFFFFFFFFFFF46
:105A7000FFFFFFFFFFFFFFFFFFFFFFFFFFFFFFFF36
:105A8000FFFFFFFFFFFFFFFFFFFFFFFFFFFFFFFF26
:105D80007DE7AF22D02ACF2ACF2ACF2ACF2ACF2A07
:105D9000CF2ACF2AEF2ACF2AD02AD02AF02AF02AD7
:105DA000F02AF02AF02A10336F1A9574FFFFFFFFD4
:105DB000FFFFFFFFFFFFFFFFFFFFFFFFFFFFFFFFF3
:105DC000FFFFFFFFFFFFFFFFFFFFFFFFFFFF989DAC
:105DD0002E121133102B102B102B102B102B102BDD
:105DE000102BF02AF02AF02AF02AF02AF02AF02AC2
:105DF000102BF02AF02AF02AF02A8E220C12B1532E
:105E0000FFFFFFFFFFFFFFFFFFFFFFFFFFFFFFFFA2
:105E1000FFFFFFFFFFFFFFFFFFFFFFFFFFFFFFFF92
:105E2000FFFFFFFFFFFFFFFFFFFFFFFFFFFFFFFF82
:105E3000FFFFFFFFFFFFFFFFFFFFFFFFFFFFFFFF72
:10614000924B8F1AF02AAF2ACF2ACF2ACF2ACF2AF2
:10615000CF2ACF2ACF2ACF2ACF2AEF2ACF2AD02A56
:10616000D02AF02AF02A10334E121CD7FFFFFFFF6F
:10617000FFFFFFFFFFFFFFFFFFFFFFFFFFFFFFFF2F
:10618000FFFFFFFFFFFFFFFFFFFFFFFFDFFF714389
:10619000AF22102BF02AF02AF02AF02AF02AF02A57
:1061A000F02A102BF02AF02AF02AF02AF02AF02AFE
:1061B000F02AF02AF02AF02AAE222D1AD253BEF786
:1061C000FFFFFFFFFFFFFFFFFFFFFFFFFFFFFFFFDF
:1061D000FFFFFFFFFFFFFFFFFFFFFFFFFFFFFFFFCF
:1061E000FFFFFFFFFFFFFFFFFFFFFFFFFFFFFFFFBF
:1061F000FFFFFFFFFFFFFFFFFFFFFFFFFFFFFFFFAF
:1064F000FFFFFFFFFFFFFFFFFFFFFFFFFFFF746CCA
:106500006F12F032AF2AAF2AAF2AAF2ACF2ACF2A92
:10651000CF2ACF2ACF2ACF2ACF2ACF2ACF2ACF2AB3
:10652000EF2ACF2AF02A8F22B24BFFFFFFFFFFFF97
:10653000FFFFFFFFFFFFFFFFFFFFFFFFFFFFFFFF6B
:10654000FFFFFFFFFFFFFFFFFFFFFFFF9BC64E1296
:106550001033F02AF02AF02AF02AF02AF02AF02A42
:10656000F02AF02AF02AF02AF02AF02AF02AF02A5B
:10657000F02AF02AF02AAF228E22546CDFFFFFFFB0
:10658000FFFFFFFFFFFFFFFFFFFFFFFFFFFFFFFF1B
:10659000FFFFFFFFFFFFFFFFFFFFFFFFFFFFFFFF0B
:1065A000FFFFFFFFFFFFFFFFFFFFFFFFFFFFFFFFFB
:1065B000FFFFFFFFFFFFFFFFFFFFFFFFFFFFFFFFEB
:1068B000FFFFFFFFFFFFFFFFFFFFFFFFB5746E123B
:1068C000F032AE2AAE2AAF2AAF2AAF2AAF2AAF2AB9
:1068D000AF2ACF2ACF2ACF2ACF2ACF2ACF2ACF2A10
:1068E000CF2ACF2A10334E1219AEFFFFFFFFFFFF52
:1068F000FFFFFFFFFFFFFFFFFFFFFFFFFFFFFFFFA8
:10690000FFFFFFFFFFFFFFFFFFFFFFFF54646E1A53
:10691000F032F02AF02AF02AF02AF02AF02AF02A9F
:10692000F02AF02AF02AF02AF02AF02AF02AF02A97
:10693000F02AF02AD022F02A578DFFFFFFFFFFFF39
:10694000FFFFFFFFFFFFFFFFFFFFFFFFFFFFFFFF57
:10695000FFFFFFFFFFFFFFFFFFFFFFFFFFFFFFFF47
:10696000FFFFFFFFFFFFFFFFFFFFFFFFFFFFFFFF37
:10697000FFFFFFFFFFFFFFFFFFFFFFFFFFFFFFFF27
:106C7000FFFFFFFFFFFFFFFFDFF7956C4E12F032C3
:106C8000AE2AAE2AAE2AAE2AAE2AAE2AAF2AAF2A42
:106C9000AF2AAF2AAF2ACF2ACF2ACF2ACF2ACF2A8C
:106CA000CF2ACF2AD02AF02AFFFFFFFFFFFFFFFFE6
:106CB000FFFFFFFFFFFFFFFFFFFFFFFFFFFFFFFFE4
:106CC000FFFFFFFFFFFFFFFFFFFF5DE7AF22F02A9F
:106CD000F02AF02AF02AF02AF02AF02AF02AF02AE4
:106CE000F02AF02AF02AF02AF02AF02AD02AD02A14
:106CF000D02AD02AD3539BC6FFFFFFFFFFFFFFFF21
:106D0000FFFFFFFFFFFFFFFFFFFFFFFFFFFFFFFF93
:106D1000FFFFFFFFFFFFFFFFFFFFFFFFFFFFFFFF83
:106D2000FFFFFFFFFFFFFFFFFFFFFFFFFFFFFFFF73
:106D3000FFFFFFFFFFFFFFFFFFFFFFFFFFFFFFFF63
:10703000FFFFFFFFFFFF1CDFD3536E12F032AE2ABB
:107040008E2AAE2AAE2AAE2AAE2AAE2AAE2AAE2AA0
:10705000AF2AAF2AAF2AAF2AAF2ACF2ACF2ACF2A08
:10706000CF2AF02A4E121685FFFFFFFFFFFFFFFF1A
:10707000FFFFFFFFFFFFFFFFFFFFFFFFFFFFFFFF20
:10708000FFFFFFFFFFFFFFFFFFFF378D4E121033A3
:10709000CF2AF02AF02AF02AF02AF02AF02AF02A41
:1070A000F02AF02ACF2ACF2ACF2AD02AD02AD02AD3
:1070B000924B989DFFFFFFFFFFFFFFFFFFFFFFFFCA
:1070C000FFFFFFFFFFFFFFFFFFFFFFFFFFFFFFFFD0
:1070D000FFFFFFFFFFFFFFFFFFFFFFFFFFFFFFFFC0
:1070E000FFFFFFFFFFFFFFFFFFFFFFFFFFFFFFFFB0
:1070F000FFFFFFFFFFFFFFFFFFFFFFFFFFFFFFFFA0
:1073F000DFF77EEF989DD0224E12F02AAF2A8E2220
:10740000AF2AAE2AAF22AF22AF2AAF2AAF2AAF2AC5
:10741000AF2AAF2AAF22AF22AF22AF22AF2AAF2AC4
:10742000CF2AAF22AF229EEFFFFFFFFFFFFFFFFF3C
:10743000FFFFFFFFFFFFFFFFFFFFFFFFFFFFFFFF5C
:10744000FFFFFFFFFFFFFFFFDFFF11338F1AD02A7F
:10745000CF2ACF2ACF2ACF2ACF2ACF2ACF2ACF2A64
:10746000CF2AD02AD02AD02AD02A313B345CB8A5E2
:10747000DFF7FFFFFFFFFFFFFFFFFFFFFFFFFFFF44
:10748000FFFFFFFFFFFFFFFFFFFFFFFFFFFFFFFF0C
:10749000FFFFFFFFFFFFFFFFFFFFFFFFFFFFFFFFFC
:1074A000FFFFFFFFFFFFFFFFFFFFFFFFFFFFFFFFEC
:1074B000FFFFFFFFFFFFFFFFFFFFFFFFFFFFFFFFDC
:1077B0007BBEB24B6E12CF22113310331033113314
:1077C0001133113311331133113311331133113399
:1077D000113311331133113311331133113310338A
:1077E000F02A513B5ABEFFFFFFFFFFFFFFFFFFFFE5
:1077F000FFFFFFFFFFFFFFFFFFFFFFFFFFFFFFFF99
:10780000FFFFFFFFFFFFFFFFDFF7B24BAF22103399
:10781000103310331033103310331033113311334E
:10782000313B7243F353956C989D1CD7FFFFFFFFCC
:10783000FFFFFFFFFFFFFFFFFFFFFFFFFFFFFFFF58
:10784000FFFFFFFFFFFFFFFFFFFFFFFFFFFFFFFF48
:10785000FFFFFFFFFFFFFFFFFFFFFFFFFFFFFFFF38
:10786000FFFFFFFFFFFFFFFFFFFFFFFFFFFFFFFF28
:107B70009BC6D9A57BBE7BBE7BBE7BBE7BBE7BBED0
:107B80007BBE7BBE7BBE7BBE7BBE7BBE7BBE7BBE2D
:107B90007BBE7BBE7BBE7BBE7BBE7BBE7BBE7BBE1D
:107BA0007BBEBFF7FFFFFFFFFFFFFFFFFFFFFFFFF2
:107BB000FFFFFFFFFFFFFFFFFFFFFFFFFFFFFFFFD5
:107BC000FFFFFFFFFFFFFFFFFFFFBEEF5AB67BBEC9
:107BD0007BBE7BBE7BBE7BBE7BBE7BBE7BBEBBC695
:107BE0001CD79EEFFFFFFFFFFFFFFFFFFFFFFFFF21
:107BF000FFFFFFFFFFFFFFFFFFFFFFFFFFFFFFFF95
:107C0000FFFFFFFFFFFFFFFFFFFFFFFFFFFFFFFF84
:107C1000FFFFFFFFFFFFFFFFFFFFFFFFFFFFFFFF74
:107C2000FFFFFFFFFFFFFFFFFFFFFFFFFFFFFFFF64
:10ABA000FFFFFFFFFFFFFFFFBFEFBFEFFFF7FFFF5D
:10ABB000FFFFFFFFFFFFFFFFFFFFFFFFFFFFDFF7CD
:10ABC000DFF7FFFFFFFFFFFFFFFFFFFFFFFFFFFFBD
:10ABD000FFFFFFFFFFFFFFFFFFFFFFFFFFFFFFFF85
:10ABE000FFFFFFFFFFFFFFFFFFFFFFFFFFFFFFFF75
:10ABF000FFFFFFFFFFFFFFFFFFFFFFFFFFFFFFFF65
:10AC0000FFFFFFFFFFFFFFFFFFFFFFFFFFFFFFFF54
:10AF5000FFFFFFFF5ED7FEB61EBF1EC7BFEFFFFF9E
:10AF6000FFFFFFFFFFFFDFF7FFA69E969EE7FFFFB5
:10AF7000FFFFFFFFFFFFFFFFFFFFDFF75ED71FB7FA
:10AF80001EBFBFEFFFFFFFFFFFFFFFFFFFFFFFFF42
:10AF9000FFFFFFFFFFFFFFFFFFFFFFFFFFFFFFFFC1
:10AFA000FFFFFFFFFFFFFFFFFFFFFFFFFFFFFFFFB1
:10AFB000FFFFFFFFFFFFFFFFFFFFFFFFFFFFFFFFA1
:10AFC000FFFFFFFFFFFFFFFFFFFFFFFFFFFFFFFF91
:10AFD000FFFFFFFFFFFFFFFFFFFFFFFFFFFFFFFF81
:10AFE000FFFFFFFFFFFFFFFFFFFFFFFFFFFFFFFF71
:10AFF000FFFFFFFFFFFFFFFFFFFFFFFFFFFFFFFF61
:10B00000FFFFFFFFFFFFFFFFFFFFFFFFFFFFFFFF50
:10B01000FFFFFFFFFFFFFFFFFFFFFFFFFFFFFFFF40
:10B02000FFFFFFFFFFFFFFFFFFFFFFFFFFFFFFFF30
:10B03000FFFFFFFFFFFFFFFFFFFFFFFFFFFFFFFF20
:10B04000FFFFFFFFFFFFFFFFFFFFFFFFFFFFFFFF10
:10B05000FFFFFFFFFFFFFFFFFFFFFFFFFFFFFFFF00
:10B06000FFFFFFFFFFFFFFFFFFFFFFFFFFFFFFFFF0
:10B07000FFFFFFFFFFFFFFFFFFFFFFFFFFFFFFFFE0
:10B08000FFFFBEF797AD97ADFFFFFFFFFFFFFFFF8D
:10B09000FFFFFFFFFFFFFFFFFFFFFFFFFFFFFFFFC0
:10B0A000FFFFFFFFFFFFFFFFFFFFFFFFFFFFFFFFB0
:10B0B000FFFFFFFFFFFFFFFFFFFFFFFFFFFFFFFFA0
:10B0C000FFFFFFFFFFFF1CDF56A57ACEFFFFFFFF4C
:10B0D000FFFFFFFFFFFFFFFFFFFFFFFFFFFFFFFF80
:10B0E000FFFFFFFFFFFFFFFFFFFFFFFFFFFFFFFF70
:10B0F000FFFFFFFFFFFFFFFFFFFFFFFFFFFFFFFF60
:10B10000FFFFFFFFFFFFFFFFFFFFFFFFFFFFFFFF4F
:10B31000FFFFFFFF5D969D559D4D7C551EC7FFFFAE
:10B32000FFFFFFFFFFFFBFF79F7EDD5D5ED7FFFFE3
:10B33000FFFFFFFFFFFFFFFFFFFF1EBFDD653E5E5C
:10B340009E969EE7FFFFFFFFFFFFFFFFFFFFFFFF50
:10B35000FFFFFFFFFFFFFFFFFFFFFFFFFFFFFFFFFD
:10B36000FFFFFFFFFFFFFFFFFFFFFFFFFFFFFFFFED
:10B37000FFFFFFFFFFFFFFFFFFFFFFFFFFFFFFFFDD
:10B38000FFFFFFFFFFFFFFFFFFFFFFFFFFFFFFFFCD
:10B39000FFFFFFFFFFFFFFFFFFFFFFFFFFFFFFFFBD
:10B3A000FFFFFFFFFFFFFFFFFFFFFFFFFFFFFFFFAD
:10B3B000FFFFFFFFFFFFFFFFFFFFFFFFFFFFFFFF9D
:10B3C000FFFFFFFFFFFFFFFFFFFFFFFFFFFFFFFF8D
:10B3D000FFFFFFFFFFFFFFFFFFFFFFFFFFFFFFFF7D
:10B3E000FFFFFFFFFFFFFFFFFFFFFFFFFFFFFFFF6D
:10B3F000FFFFFFFFFFFFFFFFFFFFFFFFFFFFFFFF5D
:10B40000FFFFFFFFFFFFFFFFFFFFFFFFFFFFFFFF4C
:10B41000FFFFFFFFFFFFFFFFFFFFFFFFFFFFFFFF3C
:10B42000FFFFFFFFFFFFFFFFFFFFFFFFFFFFFFFF2C
:10B43000FFFFFFFFFFFFFFFFFFFFFFFFFFFFFFFF1C
:10B44000FFFF3DE76A216A19BEF7FFFFFFFFFFFF1D
:10B45000FFFFFFFFFFFFFFFFFFFFFFFFFFFFFFFFFC
:10B46000FFFFFFFFFFFFFFFFFFFFFFFFFFFFFFFFEC
:10B47000FFFFFFFFFFFFFFFFFFFFFFFFFFFFFFFFDC
:10B48000FFFFFFFFFFFF77A56700916BFFFFFFFF47
:10B49000FFFFFFFFFFFFFFFFFFFFFFFFFFFFFFFFBC
:10B4A000FFFFFFFFFFFFFFFFFFFFFFFFFFFFFFFFAC
:10B4B000FFFFFFFFFFFFFFFFFFFFFFFFFFFFFFFF9C
:10B4C000FFFFFFFFFFFFFFFFFFFFFFFFFFFFFFFF8C
:10B6D000FFFFFFFF5ED71EBF1D7E7C551EC7FFFF0D
:10B6E000FFFFFFFFFFFFDFF7BE9E7E969EE7FFFF97
:10B6F000FFFFFFFFFFFFFFFF5ED71E6EDD65DEAEC3
:10B700009FE7FFFFFFFFFFFFFFFFFFFFFFFFFFFFC1
:10B71000FFFFFFFFFFFFFFFFFFFFFFFFFFFFFFFF39
:10B72000FFFFFFFFFFFFFFFFFFFFFFFFFFFFFFFF29
:10B73000FFFFFFFFFFFFFFFFFFFFFFFFFFFFFFFF19
:10B74000FFFFFFFFFFFFFFFFFFFFFFFFFFFFFFFF09
:10B75000FFFFFFFFFFFFFFFFFFFFFFFFFFFFFFFFF9
:10B76000FFFFFFFFFFFFFFFFFFFFFFFFFFFFFFFFE9
:10B77000FFFFFFFFFFFFFFFFFFFFFFFFFFFFFFFFD9
:10B78000FFFFFFFFFFFFFFFFFFFFFFFFFFFFFFFFC9
:10B79000FFFFFFFFFFFFFFFFFFFFFFFFFFFFFFFFB9
:10B7A000FFFFFFFFFFFFFFFFFFFFFFFFFFFFFFFFA9
:10B7B000FFFFFFFFFFFFFFFFFFFFFFFFFFFFFFFF99
:10B7C000FFFFFFFFFFFFFFFFFFFFFFFFFFFFFFFF89
:10B7D000FFFFFFFFFFFFFFFFFFFFFFFFFFFFFFFF79
:10B7E000FFFFFFFFFFFFFFFFFFFFFFFFFFFFFFFF69
:10B7F000FFFFFFFFFFFFFFFFFFFFFFFFFFFFFFFF59
:10B80000FFFF3DE7AB29CB29BEF7FFFFFFFFFFFF9F
:10B81000FFFFFFFFFFFFFFFFFFFFFFFFFFFFFFFF38
:10B82000FFFFFFFFFFFFFFFFFFFFFFFFFFFFFFFF28
:10B83000FFFFFFFFFFFFFFFFFFFFFFFFFFFFFFFF18
:10B84000FFFFFFFFFFFF97ADA700B26BFFFFFFFFFA
:10B85000FFFFFFFFFFFFFFFFFFFFFFFFFFFFFFFFF8
:10B86000FFFFFFFFFFFFFFFFFFFFFFFFFFFFFFFFE8
:10B87000FFFFFFFFFFFFFFFFFFFFFFFFFFFFFFFFD8
:10B88000FFFFFFFFFFFFFFFFFFFFFFFFFFFFFFFFC8
:10BA9000FFFFFFFFFFFFFFFF7D9E7C553EC7FFFFBF
:10BAA000FFFFFFFFFFFFFFFFDFF7DFF7FFFFFFFFF6
:10BAB000FFFFFFFFFFFFFFFF9DA69D551EBFFFFF7E
:10BAC000FFFFFFFFFFFFFFFFFFFFFFFFFFFFFFFF86
:10BAD000FFFFFFFFFFFFFFFFFFFFFFFFFFFFFFFF76
:10BAE000FFFFFFFFFFFFFFFFFFFFFFFFFFFFFFFF66
:10BAF000FFFFFFFFFFFFFFFFFFFFFFFFFFFFFFFF56
:10BB0000FFFFFFFFFFFFFFFFFFFFFFFFFFFFFFFF45
:10BB1000FFFFFFFFFFFFFFFFFFFFFFFFFFFFFFFF35
:10BB2000FFFFFFFFFFFFFFFFFFFFFFFFFFFFFFFF25
:10BB3000FFFFFFFFFFFFFFFFFFFFFFFFFFFFFFFF15
:10BB4000FFFFFFFFFFFFFFFFFFFFFFFFFFFFFFFF05
:10BB5000FFFFFFFFFFFFFFFFFFFFFFFFFFFFFFFFF5
:10BB6000FFFFFFFFFFFFFFFFFFFFFFFFFFFFFFFFE5
:10BB7000FFFFFFFFFFFFFFFFFFFFFFFFFFFFFFFFD5
:10BB8000FFFFFFFFFFFFFFFFFFFFFFFFFFFFFFFFC5
:10BB9000FFFFFFFFFFFFFFFFFFFFFFFFFFFFFFFFB5
:10BBA000FFFFFFFFFFFFFFFFFFFFFFFFFFFFFFFFA5
:10BBB000FFFFFFFFFFFFFFFFFFFFFFFFFFFFFFFF95
:10BBC000FFFF7DEFCB29CB29FFFFFFFFFFFFFFFF2B
:10BBD000FFFFFFFFFFFFFFFFFFFFFFFFFFFFFFFF75
:10BBE000FFFFFFFFFFFFFFFFFFFFFFFFFFFFFFFF65
:10BBF000FFFFFFFFFFFFFFFFFFFFFFFFFFFFFFFF55
:10BC0000FFFFFFFFFFFF97ADA808D273FFFFFFFF05
:10BC1000FFFFFFFFFFFFFFFFFFFFFFFFFFFFFFFF34
:10BC2000FFFFFFFFFFFFFFFFFFFFFFFFFFFFFFFF24
:10BC3000FFFFFFFFFFFFFFFFFFFFFFFFFFFFFFFF14
:10BC4000FFFFFFFFFFFFFFFFFFFFFFFFFFFFFFFF04
:10BE5000FFFFFFFFFFFFFFFF7D967C553EC7FFFF03
:10BE6000FFFFFFFFDFF7BFEFBFEFBFEFDFF7FFFF22
:10BE7000FFFFFFFFBFEFDFF73D8E5B4D1EBFBFEF44
:10BE8000DFF7FFFFFFFFFFFFFFFFFFFFFFFFFFFFEA
:10BE9000BFEF9FE7BFEFFFFFFFFFFFFFFFFFFFFFCA
:10BEA000FFFFFFFFFFFFFFFFFFFFFFFFFFFFFFFFA2
:10BEB000FFFFFFFFFFFFFFFFFFFFFFFFFFFFFFFF92
:10BEC000BEF7DBD65AC619BE7AC61CDFFFFFFFFFDE
:10BED0007DEF1CDFDEF7FFFFFFFFDFF71CDF7DEFED
:10BEE000FFFFFFFFFFFFFFFFFFFFFFFFFFFF9EEFD3
:10BEF0001CDFBEF7FFFFFFFFFFFFFFFFFFFFDFFFBE
:10BF0000FCDE5AC619BE7AC63CE7FFFFFFFF5DE7BD
:10BF1000FCDEDFFFFFFFFFFFFCDE5DE7FFFF3CE72E
:10BF20005AC639BE9BCE9EEFFFFFFFFFFFFFDFFF2C
:10BF3000DBD63AC639C6DBD6DEF7FFFFFFFFFFFFD1
:10BF4000FFFFFFFFFFFFFFFFFFFFFFFFFCDE5AC603
:10BF500039BE7ACE3DE7FFFFFFFFFFFFFFFFFFFF88
:10BF6000FFFFBEF71CDF9EEFFFFF3DE77ACE39C62D
:10BF70007AC61CDFFFFFFFFFFFFFFFFFFFFF7DEF24
:10BF80003DE79ACECB29AB293DE73CE73DE7DFFF14
:10BF9000FFFFFFFFFFFFFFFF7DEFBBD639C63AC6AD
:10BFA000BBD69EEFFFFFFFFFFFFFFFFFFFFFFFFF7F
:10BFB000FFFFFFFFFFFFFFFF1CDF7ACE39C65AC627
:10BFC000FCDEDFF7FFFF97ADA808D273FFFFFFFF8E
:10BFD000FFFFFFFFFFFFFFFFFFFFFFFFFFFFFFFF71
:10BFE000FFFFFFFFFFFFFFFFFFFFFFFFFFFFFFFF61
:10BFF000FFFFFFFFFFFFFFFFFFFFFFFFFFFFFFFF51
:10C00000FFFFFFFFFFFFFFFFFFFFFFFFFFFFFFFF40
:10C21000FFFFFFFFFFFFFFFF7D967C553EC7FFFF3F
:10C22000FFFFFFFFFEBE7E8E9E8E5D865ECFFFFF10
:10C23000FFFFFFFFDEAE9E8EDD655C555E7E5E8697
:10C240005ED7FFFFFFFFFFFFFFFFDFF75ED7FFAE09
:10C250009E967E8EBE96DEAE5ED7FFFFFFFFFFFF8F
:10C26000FFFFFFFFFFFFFFFFFFFFFFFFFFFFFFFFDE
:10C27000FFFFFFFFFFFFFFFFFFFFFFFFFFFFBBD63B
:10C2800074848E426A214919AB21105356A5DFFFF1
:10C29000F59C1053DBD6FFFFFFFF1CDF7163B48CEE
:10C2A000DFFFFFFFFFFFFFFFFFFFFFFFFFFF97AD78
:10C2B000305319BEFFFFFFFFFFFFFFFFFCDEB58C11
:10C2C000CF4A6A214A19AB21305B77ADFFFFD59485
:10C2D000EF4A3DE7FFFFFFFFCE4AD273BBD6505B6C
:10C2E0006A214A190C3213749ACEFFFF5DE7948CD1
:10C2F0008E424A194A196E42948C1CDFFFFFFFFFE1
:10C30000FFFFFFFFFFFFFFFFFCDEB58CCF4A6A2176
:10C310004A19CB29515B57A57DEFFFFFFFFFFFFFB8
:10C32000FFFF9BCE1053369D7ACE7163AB294A191D
:10C330008B211053369D7DEFFFFFFFFFBEF7D59495
:10C340001053EF52291929190F531053B26B3DE7BF
:10C35000FFFFFFFFDFF719BED2732D3A4A196A219A
:10C360004D3A337C5AC6DFFFFFFFFFFFFFFFFFFFA1
:10C37000FFFFFFFF1CDF169D1053CB294A198B21AD
:10C38000CF4AD5943DE7F8B5C808D273FFFFFFFF49
:10C39000FFFFFFFFFFFFFFFFFFFFFFFFFFFFFFFFAD
:10C3A000FFFFFFFFFFFFFFFFFFFFFFFFFFFFFFFF9D
:10C3B000FFFFFFFFFFFFFFFFFFFFFFFFFFFFFFFF8D
:10C3C000FFFFFFFFFFFFFFFFFFFFFFFFFFFFFFFF7D
:10C5D000FFFFFFFFFFFFFFFF7D967C553EC7FFFF7C
:10C5E000FFFFFFFFDDB67E7E3F6E7D45DEB6FFFFBF
:10C5F000FFFFFFFF9E9E7F76DD5D5C4D3E6E3E6ED3
:10C600003ECFFFFFFFFFFFFFBFEFFEB6DD65DE5D44
:10C610005F765F7E5F769D551E6EFEB6DFF7FFFF8D
:10C62000FFFFFFFFFFFFFFFFFFFFFFFFFFFFFFFF1A
:10C63000FFFFFFFFFFFFFFFFFFFFFFFFB8B50C325B
:10C640002A116E42305B916B0F530D32A800748437
:10C65000AE4A470019BEFFFFFFFF7ACEC908AE4AB7
:10C66000DEF7FFFFFFFFFFFFFFFFFFFFFFFF33844A
:10C670006800F594FFFFFFFFFFFF7ACEAE4AA800E7
:10C680006E3A2F5BB16BEF520D326700369DAE4AAA
:10C690000600DBD6FFFFFFFF2600E8086A21EC2931
:10C6A0000F537163CF4AE908CC29BBD670632600CB
:10C6B0008E42506370638E426700EF527EEFFFFF41
:10C6C000FFFFFFFFFFFF9BCEAF4A67006E420F5395
:10C6D0009163EF52EC318700D2735DE7FFFFFFFFFC
:10C6E000FFFFD8B54700EB290C32AC21EF52706345
:10C6F000CF52CC298700137CBEF7FFFF9EF7537CF7
:10C700004E3A4D3A091109116E424D3A10531CDF51
:10C71000FFFFBEF7F694AB214A19CF4A70637063EE
:10C720008E426B198B2156A5FFFFFFFFFFFFFFFF16
:10C73000FFFF9BCE0F53E9080C320F537163305B40
:10C740004D3A4A190F5353842911D273FFFFFFFF4B
:10C75000FFFFFFFFFFFFFFFFFFFFFFFFFFFFFFFFE9
:10C76000FFFFFFFFFFFFFFFFFFFFFFFFFFFFFFFFD9
:10C77000FFFFFFFFFFFFFFFFFFFFFFFFFFFFFFFFC9
:10C78000FFFFFFFFFFFFFFFFFFFFFFFFFFFFFFFFB9
:10C99000FFFFFFFFFFFFFFFF7D967C553EC7FFFFB8
:10C9A000FFFFFFFFDFF7DFF79DA67C55DEB6FFFF39
:10C9B000FFFFFFFFBFEFBFEF3D8E7C55FEBE9EE742
:10C9C000DFF7FFFFFFFFFFFFBEA6FE5D1E76DEB6B0
:10C9D0007EDFBEEF7EDFDEB67E7EFE5DDEAEDFF7A3
:10C9E000FFFFFFFFFFFFFFFFFFFFFFFFFFFFFFFF57
:10C9F000FFFFFFFFFFFFFFFFFFFF19BE6A19AB211B
:10CA0000B48C1CDFFFFFFFFFFFFF9ACE5063C80806
:10CA10006A2167005AC6FFFFFFFFBBD60911305BD2
:10CA2000DFF7FFFFFFFFFFFFFFFFFFFFFFFFB48CFC
:10CA3000880056A5FFFFFFFF3CE7EC310A11337C6D
:10CA4000FCDEFFFFFFFFFFFF9ACE105BA800AB29C3
:10CA50004600FCDEFFFFFFFFE808C808CC299BCE9C
:10CA6000FFFFFFFFDEF7159DC900CB29470050638C
:10CA70003DE7FFFFFFFF3DE7916B4700B16BFFFF15
:10CA8000FFFFFFFF3DE70D32090953841CDFFFFF65
:10CA9000FFFFFFFF5AC6305BA8007163FFFFFFFF77
:10CAA000FFFF19BE6700C9084D3A39C6FFFFFFFFF7
:10CAB000DFFFF8B54D3AC908D594FFFFFFFF7DEFC2
:10CAC0001CDF7ACEAB29AB29FCDE3CE73CE7FFFF5D
:10CAD000FFFF56A52A116D3A97AD9EF7FFFFFFFFA6
:10CAE0005DEF169DCC29291197ADFFFFFFFFFFFFDA
:10CAF000FCDECE4AA808916B9ACEFFFFFFFFFFFF36
:10CB0000FCDE5384AB2909112919F273FFFFFFFFE3
:10CB1000FFFFFFFFFFFFFFFFFFFFFFFFFFFFFFFF25
:10CB2000FFFFFFFFFFFFFFFFFFFFFFFFFFFFFFFF15
:10CB3000FFFFFFFFFFFFFFFFFFFFFFFFFFFFFFFF05
:10CB4000FFFFFFFFFFFFFFFFFFFFFFFFFFFFFFFFF5
:10CD5000FFFFFFFFFFFFFFFF7D967C553EC7FFFFF4
:10CD6000FFFFFFFFFFFFFFFFDDB67C55FEB6FFFFB5
:10CD7000FFFFFFFFFFFFFFFF5D967C555ED7FFFFC4
:10CD8000FFFFFFFFFFFFFEBEFE5D5E7E9EE7FFFF33
:10CD9000FFFFFFFFFFFFFFFF9EE77E7EDD5D5ECFB3
:10CDA000FFFFFFFFFFFFFFFFFFFFFFFFFFFFFFFF93
:10CDB000FFFFFFFFFFFFFFFFDFF76D42091177ADB8
:10CDC000FFFFFFFFFFFFFFFFFFFFFFFFFFFF305BE6
:10CDD000E91047005AC6FFFFFFFFBBD60A112F5BC1
:10CDE000DFF7FFFFFFFFFFFFFFFFFFFFFFFFB48C39
:10CDF000880056A5FFFFFFFF0F5B88007484FFFFCC
:10CE0000FFFFFFFFFFFFFFFFFFFFFFFFCE4AC8004E
:10CE10004600FCDEFFFFFFFFA80887007AC6FFFF81
:10CE2000FFFFFFFFFFFFFFFFCE52A8002911FFFF0A
:10CE3000FFFFFFFFFFFFFFFFFFFF4A19C808DFFFEB
:10CE4000FFFFFFFF91636800B48CFFFFFFFFFFFF50
:10CE5000FFFFFFFFFFFFBEF70F53880077A5FFFF1F
:10CE6000FFFF19BE47008A219ACEFFFFFFFFFFFF99
:10CE7000FFFFFFFF7ACEE908CC29FFFFFFFFFFFF8E
:10CE8000FFFF7DEFCB29CB29FFFFFFFFFFFFFFFF58
:10CE9000BBD6AB210C329ACEFFFFFFFFFFFFFFFF97
:10CEA000FFFFFFFFF9BD6A212D3A3DE7FFFFBEF707
:10CEB000948CC808B26BDEF7FFFFFFFFFFFFFFFF98
:10CEC000FFFFFFFFF5942911E910F273FFFFFFFF49
:10CED000FFFFFFFFFFFFFFFFFFFFFFFFFFFFFFFF62
:10CEE000FFFFFFFFFFFFFFFFFFFFFFFFFFFFFFFF52
:10CEF000FFFFFFFFFFFFFFFFFFFFFFFFFFFFFFFF42
:10CF0000FFFFFFFFFFFFFFFFFFFFFFFFFFFFFFFF31
:10D11000FFFFFFFFFFFFFFFF7D967C553EC7FFFF30
:10D12000FFFFFFFFFFFFFFFFDDAE7C55FEB6FFFFF9
:10D13000FFFFFFFFFFFFFFFF5D965C555ECFFFFF28
:10D14000FFFFFFFFFFFF3E7EDD657EDFFFFFFFFF8E
:10D15000FFFFFFFFFFFFFFFFFFFF5EDF3E667E96E4
:10D16000BFEFFFFFFFFFFFFFFFFFFFFFFFFFFFFF1F
:10D17000FFFFFFFFFFFFFFFF97AD2A117163DEF78F
:10D18000FFFFFFFFFFFFFFFFFFFFFFFFFFFF3CE78A
:10D19000AB2947005AC6FFFFFFFFBBD60A112F5B22
:10D1A000DFF7FFFFFFFFFFFFFFFFFFFFFFFFB48C75
:10D1B000880056A5FFFF3CE7A800CB29FFFFFFFF33
:10D1C000FFFFFFFFFFFFFFFFFFFFFFFF5DE7E9102E
:10D1D0004600FCDEFFFFFFFF6700C808FFFFFFFF00
:10D1E000FFFFFFFFFFFFFFFF97AD6800CE52FFFF7D
:10D1F000FFFFFFFFFFFFFFFFFFFF506388007ACEB6
:10D20000FFFF5DE787002D3AFFFFFFFFFFFFFFFFF6
:10D21000FFFFFFFFFFFFFFFF5DE709110C32FFFF7C
:10D22000FFFFF9BD67008E42FFFFFFFFFFFFFFFF1B
:10D23000FFFFFFFFBEF7CE4A4A197ACEFFFFFFFF7E
:10D24000FFFF5DE7CB29AB29BEF7FFFFFFFFBEF76E
:10D25000B594C908F594FFFFFFFFFFFFFFFFFFFF35
:10D26000FFFFFFFFFFFFF5940911B48CFFFFDBD632
:10D27000EC312D32FCDEFFFFFFFFFFFFFFFFFFFF62
:10D28000FFFFFFFF5DE75063C808F273FFFFFFFF7A
:10D29000FFFFFFFFFFFFFFFFFFFFFFFFFFFFFFFF9E
:10D2A000FFFFFFFFFFFFFFFFFFFFFFFFFFFFFFFF8E
:10D2B000FFFFFFFFFFFFFFFFFFFFFFFFFFFFFFFF7E
:10D2C000FFFFFFFFFFFFFFFFFFFFFFFFFFFFFFFF6E
:10D4D000FFFFFFFFFFFFFFFF7D967C553EC7FFFF6D
:10D4E000FFFFFFFFFFFFFFFFDDAE7C55FEB6FFFF36
:10D4F000FFFFFFFFFFFFFFFF5D965C555ECFFFFF65
:10D50000FFFFFFFF5ED75F6E5E865ED77EDF7EDF4A
:10D510007EDF7EDF7EDF7EDF7EDFBFEF1D769C5D00
:10D520009EDFFFFFFFFFFFFFFFFFFFFFFFFFFFFF8C
:10D53000FFFFFFFFFFFFFFFFB16B8800F8B5FFFFA4
:10D54000FFFFFFFFFFFFFFFFFFFFFFFFFFFFFFFFEB
:10D55000EF5267005AC6FFFFFFFFBBD60A112F5BD1
:10D56000DFF7FFFFFFFFFFFFFFFFFFFFFFFFB48CB1
:10D57000880056A5FFFF36A58800948CFFFFFFFFAB
:10D58000FFFFFFFFFFFFFFFFFFFFFFFFFFFF6D42FA
:10D590004700FCDEFFFFFFFF46006A21FFFFFFFFA1
:10D5A000FFFFFFFFFFFFFFFF5AC64700B16BFFFF02
:10D5B000FFFFFFFFFFFFFFFFFFFF337C8800D8B5B1
:10D5C000FFFF97AD68002F5B39C6D8B5D8B5D8B581
:10D5D000D8B5D8B5D8B5D8B5D8B5AB2909113CE779
:10D5E000FFFFF9BD8800916BFFFFFFFFFFFFFFFF0B
:10D5F000FFFFFFFFBEF7337C0A11B7ADFFFFFFFF50
:10D60000FFFF5DE7CB29AB29BEF7FFFFFFFF5DE71B
:10D61000EF526B19F594F9BDD8B5D8B5D8B5D8B5D2
:10D62000D8B5D8B5F9BDB5948700EF52FFFF19BE44
:10D63000A7005063FFFFFFFFFFFFFFFFFFFFFFFF9C
:10D64000FFFFFFFFFFFF56A5A800F273FFFFFFFFDC
:10D65000FFFFFFFFFFFFFFFFFFFFFFFFFFFFFFFFDA
:10D66000FFFFFFFFFFFFFFFFFFFFFFFFFFFFFFFFCA
:10D67000FFFFFFFFFFFFFFFFFFFFFFFFFFFFFFFFBA
:10D68000FFFFFFFFFFFFFFFFFFFFFFFFFFFFFFFFAA
:10D89000FFFFFFFFFFFFFFFF7D967C553EC7FFFFA9
:10D8A000FFFFFFFFFFFFFFFFDDAE7C55FEB6FFFF72
:10D8B000FFFFFFFFFFFFFFFF5D965C555ECFFFFFA1
:10D8C000FFFFFFFF1EC71E66BD65DC6DDC6DDC6DF6
:10D8D000DC6DDC6DDC6DDC6DDC6DFC759D5D7C559F
:10D8E0007EDFFFFFFFFFFFFFFFFFFFFFFFFFFFFFE9
:10D8F000FFFFFFFFFFFFFFFFEF5267009BCEFFFF21
:10D90000FFFFFFFFFFFFFFFFFFFFFFFFFFFFFFFF27
:10D91000F27388005AC6FFFFFFFFBBD60911305BC8
:10D92000DFF7FFFFFFFFFFFFFFFFFFFFFFFFB48CED
:10D93000880056A5FFFF537C6800D8B5FFFFFFFFA6
:10D94000FFFFFFFFFFFFFFFFFFFFFFFFFFFFB16BC9
:10D950002700FCDEFFFFFFFF26008A21FFFFFFFFFD
:10D96000FFFFFFFFFFFFFFFF5AC62700B16BFFFF5E
:10D97000FFFFFFFFFFFFFFFFFFFF337C8800B8B50D
:10D98000FFFF948C88004A19491929192919291966
:10D990002919291929192919491909114A195AC680
:10D9A000FFFFF9BD8800D26BFFFFFFFFFFFFFFFF06
:10D9B000FFFFFFFFDEF774840A1177ADFFFFFFFF63
:10D9C000FFFF5DE7CB29AB29BEF7FFFFFFFF3CE779
:10D9D0004D3AC9086A192919291929192919291922
:10D9E0002919291949194919C808AE4AFFFF98ADE4
:10D9F0008800127CFFFFFFFFFFFFFFFFFFFFFFFF1D
:10DA0000FFFFFFFFFFFFF9BDE810B26BFFFFFFFF55
:10DA1000FFFFFFFFFFFFFFFFFFFFFFFFFFFFFFFF16
:10DA2000FFFFFFFFFFFFFFFFFFFFFFFFFFFFFFFF06
:10DA3000FFFFFFFFFFFFFFFFFFFFFFFFFFFFFFFFF6
:10DA4000FFFFFFFFFFFFFFFFFFFFFFFFFFFFFFFFE6
:10DC5000FFFFFFFFFFFFFFFF7D967C553EC7FFFFE5
:10DC6000FFFFFFFFFFFFFFFFDDAE7C55FEB6FFFFAE
:10DC7000FFFFFFFFFFFFFFFF5D965C555ECFFFFFDD
:10DC8000FFFFFFFF1EC71E66FD6D3D8E3D8E3D8E64
:10DC90003D8E3D8E3D8E3D8E3D8E3D8E9E969D9E53
:10DCA0009FEFFFFFFFFFFFFFFFFFFFFFFFFFFFFFF4
:10DCB000FFFFFFFFFFFFFFFF2F5B67005AC6FFFF5D
:10DCC000FFFFFFFFFFFFFFFFFFFFFFFFFFFFFFFF64
:10DCD000B16B87005AC6FFFFFFFFBBD60911305B4F
:10DCE000DFF7FFFFFFFFFFFFFFFFFFFFFFFF948C4A
:10DCF000880056A5FFFF7484880077ADFFFFFFFF03
:10DD0000FFFFFFFFFFFFFFFFFFFFFFFFFFFF2F5B97
:10DD10002700FCDEFFFFFFFF46008A21FFFFFFFF19
:10DD2000FFFFFFFFFFFFFFFF5AC62700B16BFFFF9A
:10DD3000FFFFFFFFFFFFFFFFFFFF337C8800D8B529
:10DD4000FFFFD5948800AE4A5384127C127C127C6B
:10DD5000127C127C127C127C137C948CB58C1CDFA0
:10DD6000FFFFF9BD8800D16BFFFFFFFFFFFFFFFF43
:10DD7000FFFFFFFFDEF754840A1177ADFFFFFFFFBF
:10DD8000FFFF5DE7CB29AB29BEF7FFFFFFFF3DE7B4
:10DD90006D422A19B16B137C127C127C127C127CAE
:10DDA000127C127C127C537C948C57A5FFFFB8B573
:10DDB0008700D273FFFFFFFFFFFFFFFFFFFFFFFFA3
:10DDC000FFFFFFFFFFFFD8B5C808B26BFFFFFFFFE3
:10DDD000FFFFFFFFFFFFFFFFFFFFFFFFFFFFFFFF53
:10DDE000FFFFFFFFFFFFFFFFFFFFFFFFFFFFFFFF43
:10DDF000FFFFFFFFFFFFFFFFFFFFFFFFFFFFFFFF33
:10DE0000FFFFFFFFFFFFFFFFFFFFFFFFFFFFFFFF22
:10E01000FFFFFFFFFFFFFFFF7D967C553EC7FFFF21
:10E02000FFFFFFFFFFFFFFFFDDAE7C55FEB6FFFFEA
:10E03000FFFFFFFFFFFFFFFF5D965C555ECFFFFF19
:10E04000FFFFFFFF5EDF5F6E7E8EDFF7FFFFFFFFEC
:10E05000FFFFFFFFFFFFFFFFFFFFFFFFFFFFFFFFD0
:10E06000FFFFFFFFFFFFFFFFFFFFDFEFBFEFFFFF40
:10E07000FFFFFFFFFFFFFFFF7484C908169DDFFF4E
:10E08000FFFFFFFFFFFFFFFFFFFFFFFFFFFFFFFFA0
:10E090006D4247005AC6FFFFFFFFFCDE0911AE4A82
:10E0A000DFF7FFFFFFFFFFFFFFFFFFFFFFFFF27341
:10E0B000880056A5FFFFD8B588007063FFFFFFFFFB
:10E0C000FFFFFFFFFFFFFFFFFFFFFFFFFFFF8A21B3
:10E0D0004700FCDEFFFFFFFF46008A21FFFFFFFF36
:10E0E000FFFFFFFFFFFFFFFF5AC62700B16BFFFFD7
:10E0F000FFFFFFFFFFFFFFFFFFFF337C8800D8B566
:10E10000FFFF39C64700B16BFFFFFFFFFFFFFFFFB7
:10E11000FFFFFFFFFFFFFFFFFFFF9BCEFCDEFFFFC8
:10E12000FFFFF9BD8800D16BFFFFFFFFFFFFFFFF7F
:10E13000FFFFFFFFDEF754840A1177ADFFFFFFFFFB
:10E14000FFFF5DE7CB29AB29BEF7FFFFFFFF7EEFA7
:10E1500091636B1939C6FFFFFFFFFFFFFFFFFFFF52
:10E16000FFFFFFFFFFFF9EF7BBD67DEFFFFF5AC605
:10E170000911CF4AFFFFFFFFFFFFFFFFFFFFFFFF78
:10E18000FFFFFFFFDFF7D594A800F273FFFFFFFF4B
:10E19000FFFFFFFFFFFFFFFFFFFFFFFFFFFFFFFF8F
:10E1A000FFFFFFFFFFFFFFFFFFFFFFFFFFFFFFFF7F
:10E1B000FFFFFFFFFFFFFFFFFFFFFFFFFFFFFFFF6F
:10E1C000FFFFFFFFFFFFFFFFFFFFFFFFFFFFFFFF5F
:10E3D000FFFFFFFFFFFFFFFF7D967C553EC7FFFF5E
:10E3E000FFFFFFFFFFFFFFFFDDAE7C55FEB6FFFF27
:10E3F000FFFFFFFFFFFFFFFF5D965C555ECFFFFF56
:10E40000FFFFFFFFFFFF5E86DD5D5ECFFFFFFFFFCB
:10E41000FFFFFFFFFFFFFFFFFFFF7EDFFEB67FDF97
:10E42000FFFFFFFFFFFFFFFF5ED7BE9E9F8E1EBF59
:10E43000DFF7FFFFFFFFFFFFBBD68B212C3A1CDF6E
:10E44000FFFFFFFFFFFFFFFFFFFFFFFFFFFFD8B54D
:10E450004A1946005AC6FFFFFFFFDFFF4A194A1953
:10E46000BEF7FFFFFFFFFFFFFFFFFFFFFFFF4D3A7C
:10E47000880056A5FFFFDFF76A190911DBD6FFFFF9
:10E48000FFFFFFFFFFFFFFFFFFFFFFFF57A5A800F4
:10E490004600FCDEFFFFFFFF46008A21FFFFFFFF73
:10E4A000FFFFFFFFFFFFFFFF5AC62700B16BFFFF13
:10E4B000FFFFFFFFFFFFFFFFFFFF337C8800D8B5A2
:10E4C000FFFFBEF74A194A191CDFFFFFFFFFFFFFDE
:10E4D000FFFFFFFFFFFFFFFF97ADEC29137CFFFF5E
:10E4E000FFFFF9BD8800D16BFFFFFFFFFFFFFFFFBC
:10E4F000FFFFFFFFDEF754840A1177ADFFFFFFFF38
:10E50000FFFF5DE7CB29AB29BEF7FFFFFFFFFFFF52
:10E5100098ADC908505BDFFFFFFFFFFFFFFFFFFF64
:10E52000FFFFFFFF5DE791638E4239C6FFFF3CE7C7
:10E530000F536B19B8B5FFFFFFFFFFFFFFFFFFFF92
:10E54000FFFFFFFFBBD66D42E908F273FFFFFFFF3D
:10E55000FFFFFFFFFFFFFFFFFFFFFFFFFFFFFFFFCB
:10E56000FFFFFFFFFFFFFFFFFFFFFFFFFFFFFFFFBB
:10E57000FFFFFFFFFFFFFFFFFFFFFFFFFFFFFFFFAB
:10E58000FFFFFFFFFFFFFFFFFFFFFFFFFFFFFFFF9B
:10E79000FFFFFFFFFFFFFFFF7D9E7C553ECFFFFF8A
:10E7A000FFFFFFFFFFFFFFFFDEB67C55FEBEFFFF52
:10E7B000FFFFFFFFFFFFFFFF7D967C555ED7FFFF4A
:10E7C000FFFFFFFFFFFF1EC7FE5D3E7E5ED7FFFF20
:10E7D000FFFFFFFFFFFFFFFF7EDF5E7EBD5D3ECFE1
:10E7E000FFFFFFFFFFFFBFF73E7E9D4D9E4DBD5DCE
:10E7F0005ED7FFFFFFFFFFFFFFFFF273A800B16BC3
:10E80000DBDEFFFFFFFFFFFFFFFFFFFF7ACE0C32D3
:10E81000091167005AC6FFFFFFFFFFFF0F53880073
:10E82000159DFFFFFFFFFFFFFFFFFFFF369DE9087C
:10E83000670056A5FFFFFFFFD5948800AE4ABBCE08
:10E84000FFFFFFFFFFFFFFFFFFFF5AC66A19091115
:10E850004600FCDEFFFFFFFF46008A21FFFFFFFFAF
:10E86000FFFFFFFFFFFFFFFF5AC62700B16BFFFF4F
:10E87000FFFFFFFFFFFFFFFFFFFF337C8800D8B5DE
:10E88000FFFFFFFF369D8800AE4ADBD6FFFFFFFF8C
:10E89000FFFFFFFFFFFF19BEAB296B1939C6FFFF52
:10E8A000FFFFF9BD8800D16BFFFFFFFFFFFFFFFFF8
:10E8B000FFFFFFFFDEF754840A1177ADFFFFFFFF74
:10E8C000FFFF5DE7CB29AB29BEF7FFFFFFFFFFFF8F
:10E8D0005DE7CE4AC90874847DEFFFFFFFFFFFFFAD
:10E8E000FFFF5DE75384E908305B9EEFFFFFFFFF0A
:10E8F000D8B54A194D3A7ACEFFFFFFFFFFFFFFFF61
:10E90000FFFFDBD67163A8000911F273FFFFFFFF61
:10E91000FFFFFFFFFFFFFFFFFFFFFFFFFFFFFFFF07
:10E92000FFFFFFFFFFFFFFFFFFFFFFFFFFFFFFFFF7
:10E93000FFFFFFFFFFFFFFFFFFFFFFFFFFFFFFFFE7
:10E94000FFFFFFFFFFFFFFFFFFFFFFFFFFFFFFFFD7
:10EB5000FFFFFFFF5ED71EC71D7E7C559D9E1EC713
:10EB60009FE7FFFF7EDF3EC75D8E7C4D7D96FEBE3C
:10EB70009FE7FFFF5ED71EC71D7E7C559EA61EBF6A
:10EB80009FE7FFFFFFFFFFFFDEAEBD555E7EFEB6D7
:10EB90005ED77EDF5ED7DEB63E763E66FEB6DFF738
:10EBA000FFFFFFFFFFFF7EDF1F667C4D7C557D452D
:10EBB0001EBFFFFFFFFFFFFFFFFF5DEF71638800D8
:10EBC000CF4A369D19BE5AC6F9BD948CAB294D3A31
:10EBD000EC3167003AC6FFFFFFFFFFFF9ACECC295A
:10EBE0004A19748419BE7ACE39C6948C0911CB297E
:10EBF0008800369DFFFFFFFFFFFFD27388006E4243
:10EC0000F59419BE7ACE19BE74848B212D3A4D3AF3
:10EC10002600FCDEFFFFFFFF26004919FFFFFFFF74
:10EC2000FFFFFFFFFFFFFFFF5AC627009163FFFFB3
:10EC3000FFFFFFFFFFFFFFFFFFFF127C8800B8B55B
:10EC4000FFFFFFFFFFFFB16BA8006E42F59439C6CE
:10EC50007ACEF8B55384CC296A19369DFFFFFFFFA1
:10EC6000FFFFF9B58800916BFFFFFFFFFFFFFFFF7C
:10EC7000FFFFFFFFBEF7537C0A0957A5FFFFFFFF09
:10EC8000FFFF3DE78A21AB29BEF7FFFFFFFFFFFF34
:10EC9000FFFF7ACE0C32C808B26B97AD5AC639C6A0
:10ECA00057A5505B2A11EF52DBD6FFFFFFFFFFFF96
:10ECB000BEF7B48C6B21EC29B58CF9BD7ACE39C680
:10ECC000369DAE4A4A194D3AE910B16BFFFFFFFF7E
:10ECD000FFFFFFFFFFFFFFFFFFFFFFFFFFFFFFFF44
:10ECE000FFFFFFFFFFFFFFFFFFFFFFFFFFFFFFFF34
:10ECF000FFFFFFFFFFFFFFFFFFFFFFFFFFFFFFFF24
:10ED0000FFFFFFFFFFFFFFFFFFFFFFFFFFFFFFFF13
:10EF1000FFFFDFF75D8E7C559C557C559D559C5DB4
:10EF20001EC7FFFFBDA6BD5D7C559C559C555C4D25
:10EF3000DEB6FFFF5D967C559C557C559D557C55F6
:10EF40001EC7FFFFFFFFFFFFDFF7FEB65E7EBD5D62
:10EF5000DD651E76BC659C555E76FEB6DFFFFFFF65
:10EF6000FFFFFFFFFFFFDFF75E869D4D7D4DBD6517
:10EF70007ED7FFFFFFFFFFFFFFFFFFFF1CE71274BD
:10EF8000EC310911AB290C326A19E9106E425AC6EC
:10EF9000B16BC9085AC6FFFFFFFFFFFFFFFF97AD28
:10EFA000AE4AC808AB294D3AAB29C808505BB48CAF
:10EFB000E90856A5FFFFFFFFFFFFFFFFB48C4D3AA6
:10EFC000C808AB292C326A21C8088E42BBD6305BF8
:10EFD00026003DE7FFFFFFFF87008A21FFFFFFFFBD
:10EFE000FFFFFFFFFFFFFFFF5AC68800B16BFFFF67
:10EFF000FFFFFFFFFFFFFFFFFFFF337CC900B8B536
:10F00000FFFFFFFFFFFFBEF753840D32C808AB2997
:10F010000C326A19E808CF4A77ADFFFFFFFFFFFF08
:10F02000FFFFF9BDC908D16BFFFFFFFFFFFFFFFF27
:10F03000FFFFFFFFBEF774844A1977ADFFFFFFFFA4
:10F04000FFFF3DE7CB29EC31BEF7FFFFFFFFFFFFDE
:10F05000FFFFFFFF5AC6305B8B210911EC31CB2932
:10F0600009118B21D26BBBD6FFFFFFFFFFFFFFFF14
:10F07000FFFFBEF7169D4D3A09116A212C32CB29AC
:10F0800029190C32D59456A50911D273FFFFFFFF41
:10F09000FFFFFFFFFFFFFFFFFFFFFFFFFFFFFFFF80
:10F0A000FFFFFFFFFFFFFFFFFFFFFFFFFFFFFFFF70
:10F0B000FFFFFFFFFFFFFFFFFFFFFFFFFFFFFFFF60
:10F0C000FFFFFFFFFFFFFFFFFFFFFFFFFFFFFFFF50
:10F2D000FFFFDFF71EC7BEA6DEAEDDB6DEAEDEAEDA
:10F2E0009EE7FFFF5ED7DEAEDEAEDDB6DEAEBEA6CB
:10F2F0007EDFFFFF3EC7BEAEDEAEDEB6DEAEBDA633
:10F300009EDFFFFFFFFFFFFFFFFFFFFF7EDFDEAEA1
:10F310009E969F8E7E96DEAE7EDFFFFFFFFFFFFF95
:10F32000FFFFFFFFFFFFFFFF5ED79E9E7E8E1EC783
:10F33000DFFFFFFFFFFFFFFFFFFFFFFFFFFFFFFFFD
:10F3400039BE7484916B7163916BF594DBD6FFFFCA
:10F3500019BEB48C3DE7FFFFFFFFFFFFFFFFFFFF7C
:10F36000BBD6D5949163505B7163D5949EF75DE7EE
:10F37000D58CDBD6FFFFFFFF948CB58CFFFF7ACED8
:10F38000B58C91637163916BF69CFCDEFFFF8B2162
:10F390006700FFFFFFFFFFFF948C369DFFFFFFFF1D
:10F3A000FFFFFFFFFFFFFFFF3DE7948419BEFFFF54
:10F3B000FFFFFFFFFFFFFFFFFFFF5AC6B58CFCDE1C
:10F3C000FFFFFFFFFFFFFFFFFFFF39BE948C71635C
:10F3D0005163B16B169DDCD6FFFFFFFFFFFFFFFF00
:10F3E000FFFF1CDFB58C19BEFFFFFFFFFFFFFFFF14
:10F3F000FFFFFFFFDFFF5AC6D594DBDEFFFFFFFFF5
:10F40000FFFFBEF7369D369DDFFFFFFFFFFFFFFFCB
:10F41000FFFFFFFFFFFF7DEF77A51274716371633C
:10F42000127CD8B59EEFFFFFFFFFFFFFFFFFFFFF3E
:10F43000FFFFFFFFFFFFBBD6D594916B5163916334
:10F4400094845AC6FFFF3DE7D59419BEFFFFFFFF26
:10F45000FFFFFFFFFFFFFFFFFFFFFFFFFFFFFFFFBC
:10F46000FFFFFFFFFFFFFFFFFFFFFFFFFFFFFFFFAC
:10F47000FFFFFFFFFFFFFFFFFFFFFFFFFFFFFFFF9C
:10F48000FFFFFFFFFFFFFFFFFFFFFFFFFFFFFFFF8C
:10F6D000FFFFDFF7FFFFFFFFFFFFFFFFFFFFFFFF62
:10F6E000FFFFFFFFFFFFFFFFFFFFDFF7DFF7FFFF7A
:10F6F000FFFFFFFFFFFFFFFFFFFFFFFFFFFFFFFF1A
:10F70000FFFFFFFFFFFFBEF7FFFFFFFFFFFFFFFF52
:10F71000FFFFFFFFFFFFFFFFFFFFFFFFFFFFFFFFF9
:10F72000FFFFFFFFDFFF9EEFDFFFFFFFFFFFFFFF9A
:10F73000FFFFFFFFFFFFFFFFCE4A4700F594FFFFEB
:10F74000FFFFFFFFBEF7FFFFFFFFFFFF5AC6680086
:10F750004D3AFFFFFFFFFFFFFFFFFFFFFFFFFFFF30
:10F76000FFFFFFFFFFFFFFFFFFFFFFFFFFFFFFFFA9
:10F77000FFFFFFFFFFFFFFFFFFFFFFFFFFFFFFFF99
:10F78000FFFFFFFFFFFFFFFFFFFFFFFFFFFFDFFFA9
:10F79000BEF7FFFFFFFFFFFFFFFFFFFFFFFFFFFFC2
:10F7A000FFFFFFFFFFFFFFFFFFFFFFFFFFFFFFFF69
:10F7B000FFFFFFFFFFFFFFFFFFFFFFFFFFFFFFFF59
:10F7C000FFFFFFFFFFFFFFFFFFFFFFFFFFFFFFFF49
:10F7D000FFFFFFFFFFFFFFFFFFFFFFFFBEF7DFF7AA
:10F7E000FFFFFFFFFFFFFFFFFFFFFFFFFFFFFFFF29
:10F7F000FFFFFFFFFFFFFFFFFFFFFFFFBEF7DFFF82
:10F80000FFFFFFFFFFFFFFFFFFFFFFFFFFFFFFFF08
:10F81000FFFFFFFFFFFFFFFFFFFFFFFFFFFFFFFFF8
:10F82000FFFFFFFFFFFFFFFFFFFFFFFFFFFFFFFFE8
:10F83000FFFFFFFFFFFFFFFFFFFFFFFFFFFFFFFFD8
:10FAF000FFFFFFFFFFFFFFFF9BD66A192A1177A5C3
:10FB00009EEFFFFFFFFFFFFFFFFF9ACE2D3A880019
:10FB1000F8B5FFFFFFFFFFFFFFFFFFFFFFFFFFFF46
:10FB2000FFFFFFFFFFFFFFFFFFFFFFFFFFFFFFFFE5
:10FB3000FFFFFFFFFFFFFFFFFFFFFFFFFFFFFFFFD5
:10FB4000FFFFFFFFFFFFFFFFFFFFFFFFFFFFFFFFC5
:10FB5000FFFFFFFFFFFFFFFFFFFFFFFFFFFFFFFFB5
:10FEB000FFFFFFFFFFFFFFFFFFFF369D8B210911B3
:10FEC0009163169D98AD77A5337C0D32C900F2730E
:10FED000FFFFFFFFFFFFFFFFFFFFFFFFFFFFFFFF32
:10FEE000FFFFFFFFFFFFFFFFFFFFFFFFFFFFFFFF22
:10FEF000FFFFFFFFFFFFFFFFFFFFFFFFFFFFFFFF12
:10FF0000FFFFFFFFFFFFFFFFFFFFFFFFFFFFFFFF01
:0200000490F377
:10027000FFFFFFFFFFFFFFFFFFFFFFFFB8B5305B92
:100280008B2109114919291109118E42D594DFF7E3
:10029000FFFFFFFFFFFFFFFFFFFFFFFFFFFFFFFF6E
:1002A000FFFFFFFFFFFFFFFFFFFFFFFFFFFFFFFF5E
:1002B000FFFFFFFFFFFFFFFFFFFFFFFFFFFFFFFF4E
:1002C000FFFFFFFFFFFFFFFFFFFFFFFFFFFFFFFF3E
:10063000FFFFFFFFFFFFFFFFFFFFFFFFFFFF5DE784
:10064000D8B5D594337C748477A5BBD6FFFFFFFF64
:10065000FFFFFFFFFFFFFFFFFFFFFFFFFFFFFFFFAA
:10066000FFFFFFFFFFFFFFFFFFFFFFFFFFFFFFFF9A
:10067000FFFFFFFFFFFFFFFFFFFFFFFFFFFFFFFF8A
:10068000FFFFFFFFFFFFFFFFFFFFFFFFFFFFFFFF7A
:0200000490F476
:100C20008A198A198A198A198A198A194A118A19F4
:100C30008A194A118A198A194A118A198A194A1174
:100C40008A198A194A118A198A194A118A198A191C
:100C50004A118A198A194A118A198A194A118A1954
:100C60008A194A118A198A194A118A198A194A1144
:100C70008A198A194A118A198A194A118A198A19EC
:100C80004A118A198A194A118A198A194A118A1924
:100C90008A194A118A198A194A118A198A194A1114
:100CA0008A198A194A118A198A194A118A198A19BC
:100CB0004A118A198A194A118A198A194A118A19F4
:100CC0008A194A118A198A194A118A198A194A11E4
:100CD0008A198A198A198A198A198A198A198A19FC
:100CE0008A198A198A198A198A198A198A198A19EC
:100CF0008A198A198A198A198A198A198A198A19DC
:100D00008A198A198A198A198A198A198A198A19CB
:100FE0008A198A196A118A198A198A198A198A1911
:100FF0008A198A198A198A198A198A198A198A19D9
:101000008A198A198A198A198A198A198A198A19C8
:101010008A198A198A198A198A198A198A198A19B8
:101020008A198A198A198A198A198A198A198A19A8
:101030008A198A198A198A198A198A198A198A1998
:101040008A198A198A198A198A198A198A198A1988
:101050008A198A198A198A198A198A198A198A1978
:101060008A198A198A198A198A198A198A198A1968
:101070008A198A198A198A198A198A198A198A1958
:101080008A198A198A198A198A198A198A198A1948
:101090008A196A118A198A198A198A198A198A1960
:1010A0008A198A198A198A198A198A198A198A1928
:1010B0008A198A198A198A198A198A198A198A1918
:1010C0008A198A198A198A198A198A198A198A1908
:1010D0008A198A198A198A198A198A198A198A19F8
:1013A0006A118A198A198A196A118A198A196A119D
:1013B0008A198A196A118A198A196A118A198A1965
:1013C0006A118A198A196A118A198A196A118A197D
:1013D0008A196A118A198A196A118A198A196A116D
:1013E0008A198A196A118A198A196A118A198A1935
:1013F0006A118A198A196A118A198A196A118A194D
:101400008A196A118A198A196A118A198A196A113C
:101410008A198A196A118A198A196A118A198A1904
:101420006A118A198A196A118A198A196A118A191C
:101430008A196A118A198A196A118A198A196A110C
:101440008A198A196A118A198A196A118A196A11FC
:101450008A198A198A198A196A118A196A118A19C4
:101460008A198A198A198A198A198A198A198A1964
:101470008A198A198A198A198A198A198A198A1954
:101480008A198A198A198A198A198A198A198A1944
:101490008A198A198A198A198A198A198A198A1934
:101750008A198A198A198A196A118A198A198A1999
:101760008A198A198A198A198A198A198A198A1961
:101770008A198A198A198A198A198A198A198A1951
:101780008A198A198A198A198A198A198A198A1941
:101790008A198A198A198A198A198A198A198A1931
:1017A0008A198A198A198A198A198A198A198A1921
:1017B0008A198A198A198A198A198A198A198A1911
:1017C0008A198A198A198A198A198A198A198A1901
:1017D0008A198A198A198A198A198A198A198A19F1
:1017E0008A198A198A198A198A198A198A198A19E1
:1017F0008A198A198A198A198A198A198A198A19D1
:101800008A198A198A198A198A198A198A198A19C0
:101810008A196A118A198A198A198A198A198A19D8
:101820006A118A198A198A198A198A198A198A19C8
:101830008A198A198A198A198A198A198A198A1990
:101840008A198A198A198A198A198A198A198A1980
:101850008A198A198A198A198A198A198A198A1970
:101860008A198A198A198A198A198A198A198A1960
:101B10006A118A196A118A198A198A198A196A1125
:101B20008A198A196A118A198A196A118A198A19ED
:101B30006A118A198A196A118A198A196A118A1905
:101B40008A196A118A198A196A118A198A196A11F5
:101B50008A198A196A118A198A196A118A198A19BD
:101B60006A118A198A196A118A198A196A118A19D5
:101B70008A196A118A198A196A118A198A196A11C5
:101B80008A198A196A118A198A196A118A198A198D
:101B90006A118A198A196A118A198A196A118A19A5
:101BA0008A196A118A198A196A118A198A196A1195
:101BB0008A198A196A118A198A196A118A198A195D
:101BC0006A118A198A196A118A198A196A118A1975
:101BD0008A198A198A198A198A196A118A198A1915
:101BE0008A198A198A198A196A118A198A198A1905
:101BF0008A198A198A198A198A198A198A198A19CD
:101C00008A198A198A198A198A198A198A198A19BC
:101C10008A198A198A198A198A198A198A198A19AC
:101C20008A198A198A198A198A198A198A198A199C
:101EC0008A198A198A198A198A198A196A118A1922
:101ED0008A198A198A198A196A118A198A198A1912
:101EE0008A198A198A198A198A198A198A198A19DA
:101EF0008A198A198A198A198A198A198A198A19CA
:101F00008A198A198A198A198A198A198A198A19B9
:101F10008A198A198A198A198A198A198A198A19A9
:101F20008A198A198A198A198A198A198A198A1999
:101F30008A198A198A198A198A198A198A198A1989
:101F40008A198A198A198A198A198A198A198A1979
:101F50008A198A198A198A198A198A198A198A1969
:101F60008A198A198A198A198A198A198A198A1959
:101F70008A198A198A198A198A198A198A198A1949
:101F80008A198A198A198A198A198A198A198A1939
:101F90006A118A198A196A118A198A198A196A11A1
:101FA0008A198A196A118A198A198A198A198A1941
:101FB0008A198A198A198A198A198A198A198A1909
:101FC0008A198A198A198A198A198A198A198A19F9
:101FD0008A198A198A198A198A198A198A198A19E9
:101FE0008A198A198A198A198A198A198A198A19D9
:101FF0008A198A198A198A198A198A198A198A19C9
:102000008A198A198A198A198A198A198A198A19B8
:102010008A198A198A198A198A198A198A198A19A8
:102020008A198A198A198A198A198A198A198A1998
:102030008A198A198A198A198A198A198A198A1988
:102040008A198A198A198A198A198A198A198A1978
:102050008A198A198A198A198A198A198A198A1968
:102060008A198A198A198A198A198A198A198A1958
:102070008A198A198A198A198A198A198A198A1948
:102080008A198A198A198A198A198A198A198A1938
:102090008A198A198A198A198A198A198A198A1928
:1020A0008A198A198A198A198A198A198A198A1918
:1020B0008A198A198A198A198A198A198A198A1908
:1020C0008A198A198A198A198A198A198A198A19F8
:1020D0008A198A198A198A198A198A198A198A19E8
:1020E0008A198A198A198A198A198A198A198A19D8
:1020F0008A198A198A198A198A198A198A198A19C8
:102100008A198A198A198A198A198A198A198A19B7
:102110008A198A198A198A198A198A198A198A19A7
:102120008A198A198A198A198A198A198A198A1997
:102130008A198A198A198A198A198A198A198A1987
:102140008A198A198A198A198A198A198A198A1977
:102150008A198A198A196A118A198A198A198A198F
:102160008A198A198A198A198A196A118A196A11A7
:102170008A196A118A198A198A198A198A198A196F
:102180008A198A198A198A198A198A198A198A1937
:102190008A198A198A198A198A198A198A198A1927
:1021A0008A198A198A198A198A198A198A198A1917
:1021B0008A198A198A198A198A198A198A198A1907
:1021C0008A198A198A198A198A198A198A198A19F7
:1021D0008A198A198A198A198A198A198A198A19E7
:1021E0008A198A198A198A198A198A198A198A19D7
:1021F0008A198A198A198A198A198A198A198A19C7
:102200008A198A198A198A198A198A198A198A19B6
:102210008A198A198A198A198A198A198A198A19A6
:102220008A198A198A198A198A198A198A198A1996
:102230008A198A198A198A198A198A198A198A1986
:102240008A198A198A198A198A198A198A198A1976
:102250008A198A198A198A198A198A198A198A1966
:102260008A198A198A198A198A198A198A198A1956
:102270008A198A198A198A198A198A198A198A1946
:102280008A198A198A198A196A118A198A198A195E
:102290008A198A198A198A198A198A198A198A1926
:1022A0006A118A198A196A118A198A196A118A198E
:1022B0008A196A118A198A196A118A198A196A117E
:1022C0008A198A196A118A198A196A118A198A1946
:1022D0006A118A198A196A118A198A196A118A195E
:1022E0008A196A118A198A196A118A198A196A114E
:1022F0008A198A196A118A198A196A118A198A1916
:102300006A118A198A196A118A198A196A118A192D
:102310008A196A118A198A196A118A198A196A111D
:102320008A198A196A118A198A196A118A198A19E5
:102330006A118A198A196A118A198A196A118A19FD
:102340008A196A118A198A196A118A196A118A19ED
:102350008A198A198A198A198A198A198A198A1965
:102360008A198A198A198A198A198A196A118A197D
:102370006A118A198A198A198A198A198A198A196D
:102380008A198A198A198A198A198A198A198A1935
:102390008A198A198A198A198A198A198A198A1925
:1023A0008A198A198A198A198A198A198A198A1915
:1023B0008A198A198A198A198A198A198A198A1905
:1023C0008A198A198A198A198A198A198A198A19F5
:1023D0008A198A198A198A198A198A198A198A19E5
:1023E0008A198A198A198A198A198A198A198A19D5
:1023F0008A198A198A198A198A198A198A198A19C5
:102400008A198A198A198A198A198A198A198A19B4
:102410008A198A198A198A198A198A198A198A19A4
:102420008A198A198A198A198A198A198A198A1994
:102430008A198A198A198A198A198A198A198A1984
:102440008A198A198A198A198A198A198A198A1974
:102450008A198A198A198A198A198A198A198A1964
:102460008A198A198A198A198A198A198A198A1954
:102470008A198A198A198A198A198A198A198A1944
:102480008A198A198A198A198A198A198A198A1934
:102490008A198A198A198A198A198A198A198A1924
:1024A0008A198A198A198A198A198A198A198A1914
:1024B0008A198A198A198A198A198A198A198A1904
:1024C0008A198A198A198A198A198A198A198A19F4
:1024D0008A198A198A198A198A198A198A198A19E4
:1024E0008A198A198A198A198A198A198A198A19D4
:1024F0008A198A198A198A198A198A198A198A19C4
:102500008A196A118A196A118A198A198A196A112B
:102510008A196A118A198A198A198A198A196A11F3
:102520008A196A118A196A118A198A198A198A19E3
:102530008A198A198A198A198A196A118A196A11D3
:102540008A198A198A198A198A198A198A198A1973
:102550008A198A198A198A198A198A198A198A1963
:102560008A198A198A198A198A198A198A198A1953
:102570008A198A198A198A198A198A198A198A1943
:102580008A198A198A198A198A198A198A198A1933
:102590008A198A198A198A198A198A198A198A1923
:1025A0008A198A198A198A198A198A198A198A1913
:1025B0008A198A198A198A198A198A198A198A1903
:1025C0008A198A198A198A198A198A198A198A19F3
:1025D0008A198A198A198A198A198A198A198A19E3
:1025E0008A198A198A198A198A198A198A198A19D3
:1025F0008A198A198A198A198A198A198A198A19C3
:102600008A198A198A198A198A198A198A198A19B2
:102610008A198A198A198A198A198A198A198A19A2
:102620008A198A198A198A198A198A198A198A1992
:102630008A198A198A198A198A198A198A198A1982
:102640008A198A196A118A198A198A196A118A19C2
:102650006A118A196A118A198A196A118A198A19DA
:102660008A198A198A198A198A198A198A198A1952
:102670008A198A198A198A198A198A198A198A1942
:102680008A198A198A198A198A198A198A198A1932
:102690008A198A198A198A198A198A198A198A1922
:1026A0008A198A198A198A198A198A198A198A1912
:1026B0008A198A198A198A198A198A198A198A1902
:1026C0008A198A198A198A198A198A198A198A19F2
:1026D0008A198A198A198A198A198A198A198A19E2
:1026E0008A198A198A198A198A198A198A198A19D2
:1026F0008A198A198A198A198A198A198A198A19C2
:102700008A198A198A198A198A198A198A198A19B1
:102710006A118A196A118A198A196A118A198A1919
:102720006A118A198A196A118A198A198A198A19E1
:102730008A198A196A118A198A198A198A198A19A9
:102740008A198A198A198A198A198A198A198A1971
:102750008A198A198A198A198A198A198A198A1961
:102760008A198A198A198A198A198A198A198A1951
:102770008A198A198A198A198A198A198A198A1941
:102780008A198A198A198A198A198A198A198A1931
:102790008A198A198A198A198A198A198A198A1921
:1027A0008A198A198A198A198A198A198A198A1911
:1027B0008A198A198A198A198A198A198A198A1901
:1027C0008A198A198A198A198A198A198A198A19F1
:1027D0008A198A198A198A198A198A198A198A19E1
:1027E0008A198A198A198A198A198A198A198A19D1
:1027F0008A198A198A198A198A198A198A198A19C1
:102800008A198A198A198A198A198A198A198A19B0
:102810008A198A198A198A198A198A198A198A19A0
:102820008A198A198A198A198A198A198A198A1990
:102830008A198A198A198A198A198A198A198A1980
:102840008A198A198A198A198A198A198A198A1970
:102850008A198A198A198A198A198A198A198A1960
:102860008A198A198A198A198A198A198A198A1950
:102870008A198A198A198A198A198A198A198A1940
:102880008A198A198A198A198A198A198A198A1930
:102890008A198A198A198A198A198A198A198A1920
:1028A0008A198A198A198A198A198A198A196A1138
:1028B0008A196A118A196A118A196A118A198A1978
:1028C0008A198A198A198A198A196A118A198A1918
:1028D0008A198A198A196A118A198A198A198A1908
:1028E0008A198A198A198A198A198A198A198A19D0
:1028F0006A118A198A196A118A198A198A198A1910
:102900008A198A198A198A198A198A198A198A19AF
:102910008A198A198A198A198A198A198A198A199F
:102920008A198A198A198A198A198A198A198A198F
:102930008A198A198A198A198A198A198A198A197F
:102940008A198A198A198A198A198A198A198A196F
:102950008A198A198A198A198A198A198A198A195F
:102960008A198A198A198A198A198A198A198A194F
:102970008A198A198A198A198A198A198A198A193F
:102980008A198A198A198A198A198A198A198A192F
:102990008A198A198A198A198A198A198A198A191F
:1029A0008A198A198A198A198A198A198A198A190F
:1029B0008A198A198A198A198A198A198A198A19FF
:1029C0008A198A198A198A198A198A198A198A19EF
:1029D0008A198A198A198A198A198A198A198A19DF
:1029E0008A198A198A198A198A198A198A198A19CF
:1029F0008A198A198A198A198A198A198A198A19BF
:102A00006A118A198A198A198A198A198A198A19D6
:102A10008A198A198A198A198A198A198A198A199E
:102A20008A196A118A198A196A118A198A196A1106
:102A30008A198A196A118A198A196A118A198A19CE
:102A40006A118A198A196A118A198A196A118A19E6
:102A50008A196A118A198A196A118A198A196A11D6
:102A60008A198A196A118A198A196A118A198A199E
:102A70006A118A198A196A118A198A196A118A19B6
:102A80008A196A118A198A196A118A198A196A11A6
:102A90008A198A196A118A198A196A118A198A196E
:102AA0006A118A198A196A118A198A196A118A1986
:102AB0008A196A118A198A196A118A198A196A1176
:102AC0008A198A196A118A198A196A118A198A193E
:102AD0008A198A198A198A198A198A198A198A19DE
:102AE0008A198A198A198A198A198A198A196A11F6
:102AF0008A198A198A198A198A196A118A198A19E6
:102B00008A198A198A198A198A198A198A198A19AD
:102B10008A198A198A198A198A198A198A198A199D
:102B20008A198A198A198A198A198A198A198A198D
:102B30008A198A198A198A198A198A198A198A197D
:102B40008A198A198A198A198A198A198A198A196D
:102B50008A198A198A198A198A198A198A198A195D
:102B60008A198A198A198A198A198A198A198A194D
:102B70008A198A198A198A198A198A198A198A193D
:102B80008A198A198A198A198A198A198A198A192D
:102B90008A198A198A198A198A198A198A198A191D
:102BA0008A198A198A198A198A198A198A198A190D
:102BB0008A198A198A198A198A198A198A198A19FD
:102BC0008A198A198A198A198A198A198A198A19ED
:102BD0008A198A198A198A198A198A198A198A19DD
:102BE0008A198A198A198A198A198A198A198A19CD
:102BF0008A198A198A198A198A198A198A198A19BD
:102C00008A198A198A198A198A198A198A198A19AC
:102C10008A198A198A198A198A198A198A198A199C
:102C20008A198A198A198A198A198A198A198A198C
:102C30008A198A198A198A198A198A198A198A197C
:102C40008A198A198A198A198A198A198A198A196C
:102C50008A198A198A198A198A198A198A198A195C
:102C60008A198A198A196A118A196A118A198A199C
:102C70008A198A198A198A198A198A198A196A1164
:102C80008A198A196A118A198A198A198A198A1954
:102C90008A198A198A198A198A198A198A196A1144
:102CA0008A198A198A196A118A198A196A118A195C
:102CB0008A198A198A198A198A198A198A198A19FC
:102CC0008A198A198A198A198A198A198A198A19EC
:102CD0008A198A198A198A198A198A198A198A19DC
:102CE0008A198A198A198A198A198A198A198A19CC
:102CF0008A198A198A198A198A198A198A198A19BC
:102D00008A198A198A198A198A198A198A198A19AB
:102D10008A198A198A198A198A198A198A198A199B
:102D20008A198A198A198A198A198A198A198A198B
:102D30008A198A198A198A198A198A198A198A197B
:102D40008A198A198A198A198A198A198A198A196B
:102D50008A198A198A198A198A198A198A198A195B
:102D60008A198A198A198A198A198A198A198A194B
:102D70008A198A198A198A198A198A198A198A193B
:102D80008A198A198A198A198A198A198A198A192B
:102D90008A198A198A198A198A198A198A198A191B
:102DA0008A198A198A198A198A198A198A198A190B
:102DB0008A198A198A198A198A196A118A198A1923
:102DC0008A198A196A118A196A118A198A198A193B
:102DD0008A196A118A198A196A118A198A196A1153
:102DE0008A198A198A198A198A198A198A198A19CB
:102DF0008A198A198A198A198A198A198A198A19BB
:102E00008A198A198A198A198A198A198A198A19AA
:102E10008A198A198A198A198A198A198A198A199A
:102E20008A198A198A198A198A198A198A198A198A
:102E30008A198A198A198A198A198A198A198A197A
:102E40008A198A198A198A198A198A198A198A196A
:102E50008A198A198A198A198A198A198A198A195A
:102E60008A198A198A198A198A198A198A198A194A
:102E70008A198A198A198A198A198A198A198A193A
:102E80008A198A198A198A198A198A198A196A1152
:102E90008A198A196A118A196A118A198A196A1192
:102EA0008A198A196A118A198A196A118A198A195A
:102EB0008A196A118A198A198A198A198A196A114A
:102EC0008A198A198A198A198A198A198A198A19EA
:102ED0008A198A198A198A198A198A198A198A19DA
:102EE0008A198A198A198A198A198A198A198A19CA
:102EF0008A198A198A198A198A198A198A198A19BA
:102F00008A198A198A198A198A198A198A198A19A9
:102F10008A198A198A198A198A198A198A198A1999
:102F20008A198A198A198A198A198A198A198A1989
:102F30008A198A198A198A198A198A198A198A1979
:102F40008A198A198A198A198A198A198A198A1969
:102F50008A198A198A198A198A198A198A198A1959
:102F60008A198A198A198A198A198A198A198A1949
:102F70008A198A198A198A198A198A198A198A1939
:102F80008A198A198A198A198A198A198A198A1929
:102F90008A198A198A198A198A198A198A198A1919
:102FA0008A198A198A198A198A198A198A198A1909
:102FB0008A198A198A198A198A198A198A198A19F9
:102FC0008A198A198A198A198A198A198A198A19E9
:102FD0008A198A198A198A198A198A198A198A19D9
:102FE0008A198A198A198A198A198A198A198A19C9
:102FF0008A198A198A198A198A198A198A198A19B9
:103000008A198A198A198A198A198A198A198A19A8
:103010008A198A198A198A196A118A198A196A11E8
:103020008A198A198A198A198A198A198A198A1988
:103030008A198A198A198A198A198A198A198A1978
:103040008A198A198A198A196A118A198A196A11B8
:103050008A196A118A198A196A118A198A198A19A8
:103060008A196A118A198A198A198A198A198A1970
:103070006A118A196A118A198A196A118A196A11D8
:103080004A118A198A198A198A198A198A198A1970
:103090008A198A198A198A198A198A198A198A1918
:1030A0008A198A198A198A198A198A198A198A1908
:1030B0008A198A198A198A198A198A198A198A19F8
:1030C0008A198A198A198A198A198A198A198A19E8
:1030D0008A198A198A198A198A198A198A198A19D8
:1030E0008A198A198A198A198A198A198A198A19C8
:1030F0008A198A198A198A198A198A198A198A19B8
:103100008A198A198A198A198A198A198A198A19A7
:103110008A198A198A198A198A198A198A198A1997
:103120008A198A198A198A198A198A198A198A1987
:103130008A198A198A198A198A198A198A198A1977
:103140008A198A198A198A198A198A198A198A1967
:103150008A198A198A198A198A198A198A198A1957
:103160008A198A198A198A198A198A198A198A1947
:103170008A198A198A196A118A198A198A198A195F
:103180006A118A198A198A198A198A198A196A1177
:103190008A198A198A198A198A198A198A198A1917
:1031A0008A198A198A196A198A196A198A196A1967
:1031B0008A196A198A196A198A196A198A196A1977
:1031C0008A196A198A196A198A196A198A196A1967
:1031D0008A196A198A196A198A196A198A196A1957
:1031E0008A196A198A196A198A196A198A196A1947
:1031F0008A196A198A196A198A196A198A196A1937
:103200008A196A198A196A198A196A198A196A1926
:103210008A196A198A196A198A196A198A196A1916
:103220008A196A198A196A198A196A198A196A1906
:103230008A196A198A196A198A196A198A196A19F6
:103240008A196A198A196A198A196A198A198A19C6
:103250008A198A198A198A198A198A198A198A1956
:103260008A198A198A198A198A198A198A198A1946
:103270008A198A198A198A198A196A118A198A195E
:103280008A196A118A198A198A198A198A198A194E
:103290008A198A198A198A198A198A198A198A1916
:1032A0008A198A198A198A198A198A198A198A1906
:1032B0008A198A198A198A198A198A198A198A19F6
:1032C0008A198A198A198A198A198A198A198A19E6
:1032D0008A198A198A198A198A198A198A198A19D6
:1032E0008A198A198A198A198A198A198A198A19C6
:1032F0008A198A198A198A198A198A198A198A19B6
:103300008A198A198A198A198A198A198A198A19A5
:103310008A198A198A198A198A198A198A198A1995
:103320008A198A198A198A198A198A198A198A1985
:103330008A198A198A198A198A198A198A198A1975
:103340008A198A198A198A198A198A198A198A1965
:103350008A198A198A198A198A198A198A198A1955
:103360008A198A198A198A198A198A198A198A1945
:103370008A198A198A198A198A198A198A198A1935
:103380008A198A198A198A198A198A198A198A1925
:103390008A198A198A198A198A198A198A198A1915
:1033A0008A198A198A198A198A198A198A198A1905
:1033B0008A198A198A198A198A198A198A198A19F5
:1033C0008A198A198A198A198A198A196A118A190D
:1033D0006A118A196A118A198A198A198A198A1925
:1033E0008A196A118A198A196A118A198A196A113D
:1033F0008A196A118A196A118A196A118A198A192D
:103400006A118A196A118A198A198A198A198A19F4
:103410008A198A198A198A198A198A198A196A11BC
:103420008A198A198A198A198A198A196A118A19AC
:103430008A198A198A198A198A198A198A198A1974
:103440008A198A198A198A198A198A198A198A1964
:103450008A198A198A198A198A198A198A198A1954
:103460008A198A198A198A198A198A198A198A1944
:103470008A198A198A198A198A198A198A198A1934
:103480008A198A198A198A198A198A198A198A1924
:103490008A198A198A198A198A198A198A198A1914
:1034A0008A198A198A198A198A198A198A198A1904
:1034B0008A198A198A198A198A198A198A198A19F4
:1034C0008A198A198A198A198A198A198A198A19E4
:1034D0008A198A198A198A198A198A198A198A19D4
:1034E0008A198A198A198A198A198A198A198A19C4
:1034F0008A198A198A198A198A198A198A198A19B4
:103500008A198A198A198A198A198A198A198A19A3
:103510008A198A198A198A198A198A198A198A1993
:103520008A198A198A198A198A198A198A198A1983
:103530008A196A118A198A198A196A118A198A19C3
:103540008A198A198A196A118A198A198A198A198B
:103550008A196A118A196A118A198A196A118A19CB
:103560008A196A198A198A198A198A198A198A1963
:103570008A198A198A198A198A198A198A198A1933
:103580008A198A198A198A198A198A198A198A1923
:103590008A198A198A198A198A198A198A198A1913
:1035A0008A198A198A198A198A198A198A198A1903
:1035B0008A198A198A198A198A198A198A198A19F3
:1035C0008A198A198A198A198A198A198A198A19E3
:1035D0008A198A198A198A198A198A198A198A19D3
:1035E0008A198A198A198A198A198A198A198A19C3
:1035F0008A198A198A198A198A198A198A198A19B3
:103600008A198A198A198A198A198A198A196A19C2
:103610008A196A198A198A196A198A196A198A19F2
:103620006A118A198A196A118A198A196A118A19FA
:103630008A196A118A198A198A198A198A198A199A
:103640008A198A198A196A118A198A198A198A198A
:103650008A198A198A198A198A198A198A198A1952
:103660008A198A198A198A198A198A198A198A1942
:103670008A198A198A198A198A198A198A198A1932
:103680008A198A198A198A198A198A198A198A1922
:103690008A198A198A198A198A198A198A198A1912
:1036A0008A198A198A198A198A198A198A198A1902
:1036B0008A198A198A198A198A198A198A198A19F2
:1036C0008A198A198A198A198A198A198A198A19E2
:1036D0008A198A198A198A198A198A198A198A19D2
:1036E0008A198A198A198A198A198A198A198A19C2
:1036F0008A198A198A198A198A198A198A198A19B2
:103700008A198A198A198A198A198A198A198A19A1
:103710008A198A198A198A198A198A198A198A1991
:103720008A198A198A198A198A198A198A198A1981
:103730008A198A198A198A198A198A198A198A1971
:103740008A198A198A198A198A198A198A198A1961
:103750008A198A198A198A198A198A198A198A1951
:103760008A198A198A198A198A198A198A198A1941
:103770008A198A198A198A198A198A198A198A1931
:103780008A198A198A196A118A198A198A198A1949
:103790008A198A198A198A196A118A198A198A1939
:1037A0008A198A198A198A198A198A198A198A1901
:1037B0008A198A198A198A198A198A198A198A19F1
:1037C0008A198A198A198A196A118A198A196A1131
:1037D0008A198A196A118A198A196A118A198A1921
:1037E0008A196A118A196A118A198A198A198A1911
:1037F0008A196A118A198A196A118A198A196A1129
:103800008A196A118A196A118A198A198A198A19F0
:103810008A198A198A198A198A198A198A198A1990
:103820008A198A198A198A198A198A198A198A1980
:103830008A198A198A198A198A198A198A198A1970
:103840008A198A198A198A198A198A198A198A1960
:103850008A198A198A198A198A198A198A198A1950
:103860008A198A198A198A198A198A198A198A1940
:103870008A198A198A198A198A198A198A198A1930
:103880008A198A198A198A198A198A198A198A1920
:103890008A198A198A198A198A198A198A198A1910
:1038A0008A198A198A198A198A198A198A198A1900
:1038B0008A198A198A198A198A198A198A198A19F0
:1038C0008A198A198A198A198A198A198A198A19E0
:1038D0008A198A198A198A198A198A198A198A19D0
:1038E0008A198A198A198A198A198A198A196A11E8
:1038F0008A198A198A198A198A198A198A198A19B0
:103900008A196A118A198A198A198A198A196A11EF
:103910008A198A198A198A198A198A198A198A198F
:103920008A198A198A198A196A198A198A196A19BF
:103930008A198A196A198A198A196A198A198A19AF
:103940006A198A198A196A198A198A196A198A19BF
:103950008A196A198A198A196A198A198A196A19AF
:103960008A198A196A198A198A196A198A198A197F
:103970006A198A198A196A198A198A196A198A198F
:103980008A196A198A198A196A198A198A196A197F
:103990008A198A196A198A198A196A198A198A194F
:1039A0006A198A198A196A198A198A196A198A195F
:1039B0008A196A198A198A196A198A198A196A194F
:1039C0008A198A196A198A198A196A198A198A191F
:1039D0008A198A196A198A198A198A198A198A19EF
:1039E0008A198A198A198A198A198A198A198A19BF
:1039F0008A198A198A198A196A118A198A196A11FF
:103A00008A196A118A198A198A198A198A198A19C6
:103A10008A198A198A198A198A198A198A198A198E
:103A20008A198A198A198A198A198A198A198A197E
:103A30008A198A198A198A198A198A198A198A196E
:103A40008A198A198A198A198A198A198A198A195E
:103A50008A198A198A198A198A198A198A198A194E
:103A60008A198A198A198A198A198A198A198A193E
:103A70008A198A198A198A198A198A198A198A192E
:103A80008A198A198A198A198A198A198A198A191E
:103A90008A198A198A198A198A198A198A198A190E
:103AA0008A198A198A198A198A198A198A198A19FE
:103AB0008A198A198A198A198A198A198A198A19EE
:103AC0008A198A198A198A198A198A198A198A19DE
:103AD0008A198A198A198A198A198A198A198A19CE
:103AE0008A198A198A198A198A198A198A198A19BE
:103AF0008A198A198A198A198A198A198A198A19AE
:103B00008A198A198A198A198A198A198A198A199D
:103B10008A198A198A198A198A198A198A198A198D
:103B20008A198A198A198A198A198A198A198A197D
:103B30008A198A198A198A198A198A198A198A196D
:103B40008A196A118A198A198A196A118A198A19AD
:103B50008A198A198A198A198A198A198A196A1175
:103B60008A198A196A118A198A196A118A198A198D
:103B70006A118A198A198A198A198A196A118A197D
:103B80008A196A118A198A198A198A198A198A1945
:103B90008A198A198A198A198A198A198A198A190D
:103BA0008A198A198A198A198A198A198A196A1125
:103BB0008A198A198A198A198A198A198A198A19ED
:103BC0008A198A198A198A198A196A118A198A1905
:103BD0008A198A198A198A198A198A198A198A19CD
:103BE0008A198A198A198A198A198A198A198A19BD
:103BF0008A198A198A198A198A198A198A198A19AD
:103C00008A198A198A198A198A198A198A198A199C
:103C10008A198A198A198A198A198A198A198A198C
:103C20008A198A198A198A198A198A198A198A197C
:103C30008A198A198A198A198A198A198A198A196C
:103C40008A198A198A198A198A198A198A198A195C
:103C50008A198A198A198A198A198A198A198A194C
:103C60008A198A198A198A198A198A198A198A193C
:103C70008A198A198A198A198A198A198A198A192C
:103C80008A198A198A198A198A198A198A198A191C
:103C90008A198A198A198A198A198A198A198A190C
:103CA0008A198A198A198A198A196A118A198A1924
:103CB0008A196A118A196A118A198A196A118A1964
:103CC0008A198A198A196A118A198A198A198A1904
:103CD0008A198A196A198A196A198A196A198A192C
:103CE0006A198A196A198A198A198A198A198A19FC
:103CF0008A198A198A198A198A198A198A198A19AC
:103D00008A198A198A198A198A198A198A198A199B
:103D10008A198A198A198A198A198A198A198A198B
:103D20008A198A198A198A198A198A198A198A197B
:103D30008A198A198A198A198A198A198A198A196B
:103D40008A198A198A198A198A198A198A198A195B
:103D50008A198A198A198A198A198A198A198A194B
:103D60008A198A198A198A198A198A198A198A193B
:103D70008A198A198A198A198A198A198A198A192B
:103D80008A198A198A198A198A198A198A198A191B
:103D90008A198A198A198A196A198A198A196A194B
:103DA0008A196A198A196A118A196A118A198A196B
:103DB0006A118A198A198A198A198A198A198A1913
:103DC0008A198A198A196A118A196A118A196A1153
:103DD0008A198A198A198A198A198A198A198A19CB
:103DE0008A198A198A198A198A198A198A198A19BB
:103DF0008A198A198A198A198A198A198A198A19AB
:103E00008A198A198A198A198A198A198A198A199A
:103E10008A198A198A198A198A198A198A198A198A
:103E20008A198A198A198A198A198A198A198A197A
:103E30008A198A198A198A198A198A198A198A196A
:103E40008A198A198A198A198A198A198A198A195A
:103E50008A198A198A198A198A198A198A198A194A
:103E60008A198A198A198A198A198A198A198A193A
:103E70008A198A198A198A198A198A198A198A192A
:103E80008A198A198A198A198A198A198A198A191A
:103E90008A198A198A198A198A198A198A198A190A
:103EA0008A198A198A198A198A198A198A198A19FA
:103EB0008A198A198A198A198A198A198A198A19EA
:103EC0008A198A198A198A198A198A198A198A19DA
:103ED0008A198A198A198A198A198A198A198A19CA
:103EE0008A198A198A198A198A198A198A198A19BA
:103EF0008A198A198A198A196A118A196A118A19FA
:103F00008A198A198A198A198A198A198A196A11C1
:103F10008A196A118A198A196A118A198A198A19D9
:103F20008A198A198A198A198A198A198A198A1979
:103F30008A198A196A118A198A198A198A198A1991
:103F40008A198A198A196A118A198A196A118A19A9
:103F50008A196A118A198A196A118A198A196A11C1
:103F60008A198A196A118A198A196A118A198A1989
:103F70008A196A118A196A118A198A196A118A19A1
:103F80008A198A196A118A198A198A198A198A1941
:103F90006A118A198A198A198A198A198A198A1931
:103FA0008A198A198A198A198A198A198A198A19F9
:103FB0008A198A198A198A198A198A198A198A19E9
:103FC0008A198A198A198A198A198A198A198A19D9
:103FD0008A198A198A198A198A198A198A198A19C9
:103FE0008A198A198A198A198A198A198A198A19B9
:103FF0008A198A198A198A198A198A198A198A19A9
:104000008A198A198A198A198A198A198A198A1998
:104010008A198A198A198A198A198A198A198A1988
:104020008A198A198A198A198A198A198A198A1978
:104030008A198A198A198A198A198A198A198A1968
:104040008A198A198A198A198A198A198A198A1958
:104050008A198A198A198A198A198A198A198A1948
:104060008A198A198A196A118A198A198A198A1960
:104070008A198A198A198A198A198A198A198A1928
:104080008A196A118A198A198A198A196A118A1968
:104090006A198A198A198A198A198A198A198A1928
:1040A0008A198A198A198A198A198A198A198A19F8
:1040B0008A198A198A198A198A198A198A198A19E8
:1040C0008A198A198A198A198A198A198A198A19D8
:1040D0008A198A198A198A198A198A198A198A19C8
:1040E0008A198A198A198A198A198A198A198A19B8
:1040F0008A198A198A198A198A198A198A198A19A8
:104100008A198A198A198A198A198A198A198A1997
:104110008A198A198A198A198A198A198A198A1987
:104120008A198A198A198A198A198A198A198A1977
:104130008A198A198A198A198A198A198A198A1967
:104140008A198A198A198A198A198A198A198A1957
:104150008A198A198A198A198A198A198A198A1947
:104160008A198A198A198A198A198A198A198A1937
:104170008A198A196A118A198A196A118A198A1977
:104180006A118A198A198A198A198A198A198A193F
:104190008A196A118A198A198A198A198A198A192F
:1041A0008A198A198A198A198A198A198A198A19F7
:1041B0008A198A198A198A198A198A198A198A19E7
:1041C0008A198A198A198A198A198A198A198A19D7
:1041D0008A198A198A198A198A198A198A198A19C7
:1041E0008A198A198A198A198A198A198A198A19B7
:1041F0008A198A198A198A198A198A198A198A19A7
:104200008A198A198A198A198A198A198A198A1996
:104210008A198A198A198A198A198A198A198A1986
:104220008A198A198A198A198A198A198A198A1976
:104230008A198A198A198A198A198A198A198A1966
:104240008A198A198A198A198A198A198A198A1956
:104250008A198A198A198A198A198A198A198A1946
:104260008A198A198A198A198A198A198A198A1936
:104270008A198A198A198A198A198A198A198A1926
:104280008A198A198A198A198A198A198A198A1916
:104290008A198A198A198A198A198A198A198A1906
:1042A0008A198A198A198A198A198A198A198A19F6
:1042B0008A198A196A118A198A198A198A198A190E
:1042C0006A118A198A196A118A196A118A198A194E
:1042D0008A198A198A198A198A198A198A198A19C6
:1042E0006A118A198A196A118A198A196A118A192E
:1042F0006A118A198A198A196A118A198A196A111E
:104300008A196A118A198A198A198A198A198A19BD
:104310008A198A198A198A198A198A198A198A1985
:104320008A198A198A198A198A198A198A198A1975
:104330008A198A198A198A198A198A198A198A1965
:104340006A118A198A198A196A118A198A198A19A5
:104350008A198A196A118A196A118A198A198A1995
:104360008A198A198A198A198A198A198A198A1935
:104370008A198A198A198A198A198A198A198A1925
:104380008A198A198A198A198A198A198A198A1915
:104390008A198A198A198A198A198A198A198A1905
:1043A0008A198A198A198A198A198A198A198A19F5
:1043B0008A198A198A198A198A198A198A198A19E5
:1043C0008A198A198A198A198A198A198A198A19D5
:1043D0008A198A198A198A198A198A198A198A19C5
:1043E0008A198A198A198A198A198A198A198A19B5
:1043F0008A198A198A198A198A198A198A198A19A5
:104400008A198A198A198A198A198A198A198A1994
:104410008A198A198A198A198A198A198A196A11AC
:104420008A198A198A198A198A196A118A196A11C4
:104430008A198A196A118A198A196A118A198A19B4
:104440008A198A198A196A198A198A198A198A1974
:104450008A198A196A198A198A198A198A198A1964
:104460008A198A198A198A198A198A198A198A1934
:104470008A198A198A198A198A198A198A198A1924
:104480008A198A198A198A198A198A198A198A1914
:104490008A198A198A198A198A198A198A198A1904
:1044A0008A198A198A198A198A198A198A198A19F4
:1044B0008A198A198A198A198A198A198A198A19E4
:1044C0008A198A198A198A198A198A198A198A19D4
:1044D0008A198A198A198A198A198A198A198A19C4
:1044E0008A198A198A198A198A198A198A198A19B4
:1044F0008A198A198A198A198A198A198A198A19A4
:104500008A198A198A198A198A198A198A198A1993
:104510008A198A196A198A198A198A198A198A19A3
:104520008A198A198A198A198A196A198A196A19B3
:104530008A198A198A198A198A198A198A198A1963
:104540008A198A196A118A198A198A198A198A197B
:104550008A198A198A196A118A198A198A198A196B
:104560008A198A198A198A198A198A198A198A1933
:104570008A198A198A198A198A198A198A198A1923
:104580008A198A198A198A198A198A198A198A1913
:104590008A198A198A198A198A198A198A198A1903
:1045A0008A198A198A198A198A198A198A198A19F3
:1045B0008A198A198A198A198A198A198A198A19E3
:1045C0008A198A198A198A198A198A198A198A19D3
:1045D0008A198A198A198A198A198A198A198A19C3
:1045E0008A198A198A198A198A198A198A198A19B3
:1045F0008A198A198A198A198A198A198A198A19A3
:104600008A198A198A198A198A198A198A198A1992
:104610008A198A198A198A198A198A198A198A1982
:104620008A198A198A198A198A198A198A198A1972
:104630008A198A198A198A198A198A198A198A1962
:104640008A198A198A198A198A198A198A198A1952
:104650008A198A198A198A198A198A198A198A1942
:104660008A198A198A198A198A198A198A196A115A
:104670008A198A198A198A198A198A198A198A1922
:104680008A198A198A198A198A198A198A198A1912
:104690006A118A198A196A118A198A196A118A197A
:1046A0008A198A198A198A198A198A198A198A19F2
:1046B0008A198A198A198A198A198A198A198A19E2
:1046C0008A198A198A196A118A196A118A198A1922
:1046D0006A118A198A196A118A198A196A118A193A
:1046E0008A196A198A196A198A196A198A196A1932
:1046F0008A198A196A198A196A118A198A196A1112
:104700008A198A198A198A198A198A198A198A1991
:104710006A118A198A198A198A198A198A198A19A9
:104720006A118A198A198A198A198A198A198A1999
:104730008A198A198A198A198A198A198A198A1961
:104740008A198A198A198A198A198A198A198A1951
:104750008A198A198A198A198A198A198A198A1941
:104760008A198A198A198A198A198A198A198A1931
:104770008A198A198A198A198A198A198A198A1921
:104780008A198A198A198A198A198A198A198A1911
:104790008A198A198A198A198A198A198A198A1901
:1047A0008A198A198A198A198A198A198A198A19F1
:1047B0008A198A198A198A198A198A198A198A19E1
:1047C0008A198A198A198A198A198A198A198A19D1
:1047D0008A198A198A198A198A196A118A198A19E9
:1047E0008A198A198A196A118A198A198A198A19D9
:1047F0008A198A198A198A198A198A198A198A19A1
:104800008A196A118A198A198A198A196A198A19D8
:104810008A198A198A198A198A198A196A198A19A0
:104820008A196A198A198A198A198A198A198A1990
:104830008A198A198A198A198A198A198A198A1960
:104840008A198A198A198A198A198A198A198A1950
:104850008A198A198A198A198A198A198A198A1940
:104860008A198A198A198A198A198A198A198A1930
:104870008A198A198A198A198A198A198A198A1920
:104880008A198A198A198A198A198A198A198A1910
:104890008A198A198A198A198A198A198A198A1900
:1048A0008A198A198A198A198A198A198A198A19F0
:1048B0008A198A198A198A198A198A198A198A19E0
:1048C0008A198A198A198A198A198A198A198A19D0
:1048D0008A198A198A198A198A198A198A198A19C0
:1048E0006A198A198A196A198A198A198A198A19F0
:1048F0008A198A198A196A118A198A196A118A19F0
:104900006A118A198A198A198A196A118A196A1107
:104910008A196A118A198A198A198A198A196A11CF
:104920008A198A198A198A198A198A198A198A196F
:104930008A198A198A198A198A198A198A198A195F
:104940008A198A198A198A198A198A198A198A194F
:104950008A198A198A198A198A198A198A198A193F
:104960008A198A198A198A198A198A198A198A192F
:104970008A198A198A198A198A198A198A198A191F
:104980008A198A198A198A198A198A198A198A190F
:104990008A198A198A198A198A198A198A198A19FF
:1049A0008A198A198A198A198A198A198A198A19EF
:1049B0008A198A198A198A198A198A198A198A19DF
:1049C0008A198A198A198A198A198A198A198A19CF
:1049D0008A198A198A198A198A198A198A198A19BF
:1049E0008A198A198A198A198A198A198A198A19AF
:1049F0008A198A198A198A198A198A198A198A199F
:104A00008A198A198A198A198A198A198A198A198E
:104A10008A198A198A198A198A198A198A198A197E
:104A20008A198A198A198A198A196A118A198A1996
:104A30008A196A118A198A196A118A196A118A19D6
:104A40008A196A118A196A118A198A196A118A19C6
:104A50008A198A198A198A198A198A198A198A193E
:104A60008A198A196A118A198A196A118A198A197E
:104A70006A118A198A196A118A198A196A118A1996
:104A80006A198A198A198A198A198A198A198A192E
:104A90008A198A198A198A198A198A198A198A19FE
:104AA0008A198A198A198A198A198A198A198A19EE
:104AB0006A198A198A198A198A198A198A198A19FE
:104AC0006A118A196A118A198A196A118A198A1946
:104AD0008A198A198A196A118A198A196A118A190E
:104AE0008A198A198A198A198A198A198A198A19AE
:104AF0008A198A198A198A198A198A198A198A199E
:104B00008A198A198A198A198A198A198A198A198D
:104B10008A198A198A198A198A198A198A198A197D
:104B20008A198A198A198A198A198A198A198A196D
:104B30008A198A198A198A198A198A198A198A195D
:104B40008A198A198A198A198A198A198A198A194D
:104B50008A198A198A198A198A198A198A198A193D
:104B60008A198A198A198A198A198A198A198A192D
:104B70008A198A198A198A198A198A198A198A191D
:104B80008A198A198A198A198A198A198A198A190D
:104B90008A196A118A198A198A198A198A196A114D
:104BA0008A198A198A198A198A198A196A118A1915
:104BB0008A196A118A198A196A118A198A196A194D
:104BC0008A198A198A196A198A198A198A198A19ED
:104BD0006A198A198A198A198A198A198A198A19DD
:104BE0008A198A198A198A198A198A198A198A19AD
:104BF0008A198A198A198A198A198A198A198A199D
:104C00008A198A198A198A198A198A198A198A198C
:104C10008A198A198A198A198A198A198A198A197C
:104C20008A198A198A198A198A198A198A198A196C
:104C30008A198A198A198A198A198A198A198A195C
:104C40008A198A198A198A198A198A198A198A194C
:104C50008A198A198A198A198A198A198A198A193C
:104C60008A198A198A198A198A198A198A198A192C
:104C70008A198A198A198A198A198A198A198A191C
:104C80008A198A198A198A198A198A198A198A190C
:104C90008A198A198A198A196A198A198A198A191C
:104CA0008A198A198A198A198A198A198A196A190C
:104CB0008A196A198A198A198A198A198A198A19FC
:104CC0008A198A198A196A118A198A198A198A19F4
:104CD0008A198A198A196A118A198A198A198A19E4
:104CE0008A196A118A198A198A198A198A198A19D4
:104CF0008A198A198A198A198A198A198A198A199C
:104D00008A198A198A198A198A198A198A198A198B
:104D10008A198A198A198A198A198A198A198A197B
:104D20008A198A198A198A198A198A198A198A196B
:104D30008A198A198A198A198A198A198A198A195B
:104D40008A198A198A198A198A198A198A198A194B
:104D50008A198A198A198A198A198A198A198A193B
:104D60008A198A198A198A198A198A198A198A192B
:104D70008A198A198A198A198A198A198A198A191B
:104D80008A198A198A198A198A198A198A198A190B
:104D90008A198A198A198A198A198A198A198A19FB
:104DA0008A198A198A198A198A198A198A198A19EB
:104DB0008A198A198A198A198A198A198A198A19DB
:104DC0008A198A198A198A198A198A198A198A19CB
:104DD0008A198A198A198A198A198A198A198A19BB
:104DE0008A196A118A198A198A198A198A198A19D3
:104DF0008A198A198A198A198A198A198A198A199B
:104E00008A198A198A198A198A198A198A198A198A
:104E10006A118A196A118A198A196A118A198A19F2
:104E20006A118A198A198A198A198A198A198A1992
:104E30008A198A198A198A198A198A198A198A195A
:104E40008A198A196A198A198A196A198A196A19AA
:104E50008A198A198A196A198A196A198A198A197A
:104E60008A196A198A198A198A198A198A198A194A
:104E70008A198A196A198A196A118A196A118A198A
:104E80008A198A198A198A198A198A198A198A190A
:104E90008A196A118A198A198A198A198A198A1922
:104EA0008A198A198A196A118A196A118A198A193A
:104EB0008A198A198A198A198A198A198A198A19DA
:104EC0008A198A198A198A198A198A198A198A19CA
:104ED0008A198A198A198A198A198A198A198A19BA
:104EE0008A198A198A198A198A198A198A198A19AA
:104EF0008A198A198A198A198A198A198A198A199A
:104F00008A198A198A198A198A198A198A198A1989
:104F10008A198A198A198A198A198A198A198A1979
:104F20008A198A198A198A198A198A198A198A1969
:104F30008A198A198A198A198A198A198A198A1959
:104F40008A198A198A198A198A198A196A118A1971
:104F50008A198A198A198A198A196A118A198A1961
:104F60008A196A118A198A196A118A198A198A1979
:104F70008A198A198A198A198A198A198A198A1919
:104F80008A196A198A198A198A198A198A198A1929
:104F90008A198A198A198A198A198A198A198A19F9
:104FA0008A198A198A198A198A198A198A198A19E9
:104FB0008A198A198A198A198A198A198A198A19D9
:104FC0008A198A198A198A198A198A198A198A19C9
:104FD0008A198A198A198A198A198A198A198A19B9
:104FE0008A198A198A198A198A198A198A198A19A9
:104FF0008A198A198A198A198A198A198A198A1999
:105000008A198A198A198A198A198A198A198A1988
:105010008A198A198A198A198A198A198A198A1978
:105020008A198A198A198A198A198A198A198A1968
:105030008A198A198A198A198A198A198A198A1958
:105040008A198A198A198A198A198A198A198A1948
:105050008A196A198A198A198A198A198A198A1958
:105060008A198A198A198A198A196A198A198A1948
:105070008A198A198A198A196A198A196A198A1958
:105080008A196A198A198A198A198A198A198A1928
:105090008A198A198A198A198A198A198A196A1120
:1050A0008A198A198A198A198A198A198A198A19E8
:1050B0008A198A198A198A198A198A198A198A19D8
:1050C0008A198A198A198A198A198A198A198A19C8
:1050D0008A198A198A198A198A198A198A198A19B8
:1050E0008A198A198A198A198A198A198A198A19A8
:1050F0008A198A198A198A198A198A198A198A1998
:105100008A198A198A198A198A198A198A198A1987
:105110008A198A198A198A198A198A198A198A1977
:105120008A198A198A198A198A198A198A198A1967
:105130008A198A198A198A198A198A198A198A1957
:105140008A198A198A198A198A198A198A198A1947
:105150008A198A198A198A198A198A198A198A1937
:105160008A198A198A198A198A198A198A198A1927
:105170008A198A198A198A198A198A198A198A1917
:105180008A198A198A198A198A198A198A198A1907
:105190008A198A198A198A198A198A198A196A111F
:1051A0008A198A198A198A196A118A198A196A1137
:1051B0008A198A196A118A198A196A118A198A1927
:1051C0006A118A198A196A118A198A196A118A193F
:1051D0008A198A198A198A198A198A198A198A19B7
:1051E0008A198A198A198A196A198A196A198A19E7
:1051F0006A198A198A198A196A198A198A198A19D7
:105200006A198A198A196A198A198A198A198A19C6
:105210008A198A198A198A198A198A198A198A1976
:105220008A198A198A198A198A196A198A198A1986
:105230008A198A198A198A198A198A198A198A1956
:105240008A196A118A198A196A118A198A196A11BE
:105250008A198A198A196A118A196A118A198A1986
:105260006A118A198A198A198A198A198A196A1176
:105270008A198A198A198A198A198A198A198A1916
:105280008A198A198A198A198A198A198A198A1906
:105290008A198A198A198A198A198A198A198A19F6
:1052A0008A198A198A198A198A198A198A198A19E6
:1052B0008A198A198A198A198A198A198A198A19D6
:1052C0008A198A198A198A198A198A198A198A19C6
:1052D0008A198A198A198A198A198A198A198A19B6
:1052E0008A198A198A198A198A198A198A198A19A6
:1052F0008A198A198A198A198A198A198A198A1996
:105300008A198A196A118A198A198A198A198A19AD
:105310006A118A198A196A118A198A198A198A19C5
:105320008A198A198A198A198A198A196A118A198D
:105330006A118A198A196A198A196A198A196A19DD
:105340008A198A198A198A198A196A198A198A1965
:105350008A198A196A198A198A198A198A198A1955
:105360008A198A198A198A198A198A198A198A1925
:105370008A198A198A198A198A198A198A198A1915
:105380008A198A198A198A198A198A198A198A1905
:105390008A198A198A198A198A198A198A198A19F5
:1053A0008A198A198A198A198A198A198A198A19E5
:1053B0008A198A198A198A198A198A198A198A19D5
:1053C0008A198A198A198A198A198A198A198A19C5
:1053D0008A198A198A198A198A198A198A198A19B5
:1053E0008A198A198A198A198A198A198A198A19A5
:1053F0008A198A198A198A198A198A198A198A1995
:105400008A198A198A198A198A198A198A198A1984
:105410008A196A198A198A198A198A196A198A19B4
:105420008A198A198A198A198A198A198A198A1964
:105430008A198A198A198A198A198A198A198A1954
:105440006A198A198A196A118A196A118A196A11DC
:105450008A196A118A198A196A118A198A198A1984
:105460008A196A118A196A118A198A198A198A1974
:105470008A198A198A198A198A198A198A198A1914
:105480008A198A198A198A198A198A198A198A1904
:105490008A198A198A198A198A198A198A198A19F4
:1054A0008A198A198A198A198A198A198A198A19E4
:1054B0008A198A198A198A198A198A198A198A19D4
:1054C0008A198A198A198A198A198A198A198A19C4
:1054D0008A198A198A198A198A198A198A198A19B4
:1054E0008A198A198A198A198A198A198A198A19A4
:1054F0008A198A198A198A198A198A198A198A1994
:105500008A198A198A198A198A198A198A198A1983
:105510008A198A198A198A198A198A198A198A1973
:105520008A198A198A198A198A198A198A198A1963
:105530008A198A198A198A198A198A198A198A1953
:105540008A198A198A198A198A198A198A198A1943
:105550008A198A198A196A118A198A198A198A195B
:105560008A196A118A198A198A198A198A198A194B
:105570008A198A198A198A198A198A198A198A1913
:105580008A198A198A198A198A198A198A198A1903
:105590008A196A198A196A198A196A198A196A1973
:1055A0008A198A198A196A196A198A198A198A1923
:1055B0008A198A198A198A198A198A198A198A19D3
:1055C0008A198A198A198A198A198A198A198A19C3
:1055D0008A198A198A198A198A198A198A198A19B3
:1055E0008A198A198A198A198A198A198A198A19A3
:1055F0008A198A198A198A198A198A196A118A19BB
:105600008A196A198A198A196A198A198A196A19E2
:105610008A198A198A196A198A196A198A198A19B2
:105620006A198A198A198A196A118A198A196A19CA
:105630008A198A198A196A118A196A118A196A11CA
:105640008A198A198A198A198A198A198A198A1942
:105650008A198A198A198A198A198A198A198A1932
:105660008A198A198A198A198A198A198A198A1922
:105670008A198A198A198A198A198A198A198A1912
:105680008A198A198A198A198A198A198A198A1902
:105690008A198A198A198A198A198A198A198A19F2
:1056A0008A198A198A198A198A198A198A198A19E2
:1056B0008A198A198A198A198A198A196A118A19FA
:1056C0006A118A198A198A198A198A196A118A1912
:1056D0008A198A198A196A198A198A198A196A11FA
:1056E0008A198A196A118A196A118A196A198A1912
:1056F0006A198A198A198A198A198A198A198A19B2
:105700008A198A198A196A198A198A198A198A19A1
:105710006A198A198A196A198A198A198A198A19B1
:105720008A198A198A198A198A198A198A198A1961
:105730008A198A198A198A198A198A198A198A1951
:105740008A198A198A198A198A198A198A198A1941
:105750008A198A198A198A198A198A198A198A1931
:105760008A198A198A198A198A198A198A198A1921
:105770008A198A198A198A198A198A198A198A1911
:105780008A198A198A198A198A198A198A198A1901
:105790008A198A198A198A198A198A198A198A19F1
:1057A0008A198A198A198A198A198A198A198A19E1
:1057B0008A198A198A198A198A198A198A198A19D1
:1057C0008A198A198A198A198A198A198A198A19C1
:1057D0008A198A198A198A198A198A196A198A19D1
:1057E0008A198A198A198A198A198A196A198A19C1
:1057F0008A196A198A198A198A198A198A198A19B1
:105800008A198A198A196A198A198A198A198A19A0
:105810008A196A198A198A196A198A198A196A11D8
:105820008A196A198A196A198A196A118A198A19C8
:105830006A118A198A198A198A198A198A198A1978
:105840008A198A198A198A198A198A198A198A1940
:105850008A198A198A198A198A198A198A198A1930
:105860008A198A198A198A198A198A198A198A1920
:105870008A198A198A198A198A198A198A198A1910
:105880008A198A198A198A198A198A198A198A1900
:105890008A198A198A198A198A198A198A198A19F0
:1058A0008A198A198A198A198A198A198A198A19E0
:1058B0008A198A198A198A198A198A198A198A19D0
:1058C0008A198A198A198A198A198A198A198A19C0
:1058D0008A198A198A198A198A198A198A198A19B0
:1058E0008A198A198A198A198A198A198A198A19A0
:1058F0008A198A198A198A198A198A198A198A1990
:105900008A198A198A198A198A198A198A198A197F
:105910008A196A118A198A198A198A198A196A11BF
:105920008A198A198A198A198A196A118A198A1987
:105930006A118A198A196A118A198A196A118A19C7
:105940008A196A118A196A198A196A198A196A19C7
:105950008A198A198A198A198A198A198A198A192F
:105960008A198A198A198A198A198A198A198A191F
:105970008A198A198A198A198A198A198A198A190F
:105980008A198A198A198A198A198A196A198A191F
:105990008A196A198A198A196A198A198A196A194F
:1059A0008A198A198A198A198A198A196A198A19FF
:1059B0008A198A198A198A196A118A198A198A19F7
:1059C0006A118A198A196A118A198A196A118A1937
:1059D0008A196A118A198A196A118A198A196A1127
:1059E0008A198A196A118A196A198A196A118A190F
:1059F0008A196A118A196A198A198A198A196A19F7
:105A00008A196A118A196A118A198A198A198A19CE
:105A10008A198A198A198A198A198A198A198A196E
:105A20008A198A198A198A198A198A198A198A195E
:105A30008A198A198A198A198A198A198A198A194E
:105A40008A198A198A198A198A198A198A198A193E
:105A50008A198A198A198A198A198A198A198A192E
:105A60008A198A198A198A198A198A198A198A191E
:105A70008A198A198A198A196A118A196A198A1956
:105A80006A198A196A118A198A198A198A198A1946
:105A90006A118A196A118A198A196A118A196A1986
:105AA0008A198A198A198A196A198A198A196A191E
:105AB0008A196A198A196A198A198A198A198A190E
:105AC0008A198A198A196A198A198A198A198A19DE
:105AD0006A198A198A198A198A198A198A198A19CE
:105AE0008A198A198A198A198A198A198A198A199E
:105AF0008A198A198A198A198A198A198A198A198E
:105B00008A198A198A198A198A198A198A198A197D
:105B10008A198A198A198A198A198A198A198A196D
:105B20008A198A198A198A198A198A198A198A195D
:105B30008A198A198A198A198A198A198A198A194D
:105B40008A198A198A198A198A198A198A198A193D
:105B50008A198A198A198A198A198A198A198A192D
:105B60008A198A198A198A198A198A198A198A191D
:105B70008A198A198A198A198A198A198A198A190D
:105B80008A198A198A198A198A198A198A198A19FD
:105B90008A198A198A198A198A198A198A198A19ED
:105BA0008A198A198A198A198A198A196A198A19FD
:105BB0008A198A198A198A198A198A196A198A19ED
:105BC0006A198A196A198A198A198A198A198A19FD
:105BD0006A118A198A196A118A198A198A196A191D
:105BE0008A198A198A198A198A196A198A198A19BD
:105BF0006A198A198A198A198A198A198A198A19AD
:105C00008A198A198A198A198A198A198A198A197C
:105C10008A198A198A198A198A198A198A198A196C
:105C20008A198A198A198A198A198A198A198A195C
:105C30008A198A198A198A198A198A198A198A194C
:105C40008A198A198A198A198A198A198A198A193C
:105C50008A198A198A198A198A198A198A198A192C
:105C60008A198A198A198A198A198A198A198A191C
:105C70008A198A198A198A198A198A198A198A190C
:105C80008A198A198A198A198A198A198A198A19FC
:105C90008A198A198A198A198A198A198A198A19EC
:105CA0008A198A198A198A198A198A198A198A19DC
:105CB0008A198A198A198A198A198A198A198A19CC
:105CC0008A198A198A198A198A198A198A196A11E4
:105CD0008A196A198A196A118A198A198A198A19F4
:105CE0008A196A118A198A198A196A198A198A19E4
:105CF0006A198A198A198A198A198A196A198A19CC
:105D00008A198A198A198A198A198A198A198A197B
:105D10008A196A198A198A198A198A198A198A198B
:105D20008A198A198A198A198A198A196A198A197B
:105D30008A196A198A198A196A198A198A196A19AB
:105D40008A198A196A198A198A198A198A198A195B
:105D50008A198A198A198A198A198A198A198A192B
:105D60008A196A198A198A198A198A196A198A195B
:105D70008A198A198A198A198A198A196A118A1933
:105D80006A198A198A196A198A198A196A198A195B
:105D90008A196A198A198A196A198A198A196A194B
:105DA0008A198A196A198A198A198A198A198A19FB
:105DB0008A196A198A198A198A198A198A198A19EB
:105DC0008A196A198A196A198A198A198A196A1123
:105DD0008A198A196A118A196A118A198A198A19FB
:105DE0008A198A198A198A198A198A198A198A199B
:105DF0008A198A198A198A198A198A198A198A198B
:105E00008A198A198A198A198A198A198A198A197A
:105E10008A198A198A198A198A198A198A198A196A
:105E20008A198A198A198A196A118A196A118A19AA
:105E30006A118A196A118A198A198A198A198A199A
:105E40008A198A196A198A198A198A196A118A1982
:105E50006A198A196A198A198A196A198A198A198A
:105E60008A198A196A118A198A196A198A198A1962
:105E70008A198A198A198A198A198A196A198A192A
:105E80008A198A198A196A198A198A198A198A191A
:105E90006A198A198A198A198A198A198A198A190A
:105EA0008A198A198A198A198A198A198A198A19DA
:105EB0008A198A198A198A198A198A198A198A19CA
:105EC0008A198A198A198A198A198A198A198A19BA
:105ED0008A198A198A198A198A198A198A198A19AA
:105EE0008A198A198A198A198A198A198A198A199A
:105EF0008A198A198A198A198A198A198A198A198A
:105F00008A198A198A198A198A198A198A198A1979
:105F10008A198A198A198A198A198A198A198A1969
:105F20008A198A198A198A198A198A198A198A1959
:105F30008A198A198A198A198A198A198A198A1949
:105F40008A198A198A198A198A198A198A198A1939
:105F50008A198A198A198A198A198A198A198A1929
:105F60008A198A198A198A198A198A196A198A1939
:105F70008A198A198A198A198A198A196A198A1929
:105F80008A198A198A198A196A198A196A198A1939
:105F90008A198A198A196A198A198A196A118A1931
:105FA0008A196A118A196A118A198A196A118A1951
:105FB0008A196A118A196A118A198A198A198A1919
:105FC0008A198A198A198A198A198A198A198A19B9
:105FD0008A198A198A198A198A198A198A198A19A9
:105FE0008A198A198A198A198A198A198A198A1999
:105FF0008A198A198A198A198A198A198A198A1989
:106000008A198A198A198A198A198A198A198A1978
:106010008A198A198A198A198A198A198A198A1968
:106020008A198A198A198A198A198A198A198A1958
:106030008A198A198A198A198A198A198A198A1948
:106040008A198A198A198A198A198A198A198A1938
:106050008A198A198A198A198A198A198A198A1928
:106060008A198A198A198A198A198A198A198A1918
:106070008A198A198A198A198A198A198A198A1908
:106080008A198A198A198A198A196A118A198A1920
:106090008A198A198A196A198A198A198A196A1130
:1060A0008A196A198A196A118A198A196A118A1948
:1060B0008A196A118A196A118A196A198A196A1958
:1060C0008A196A198A198A196A198A198A196A1918
:1060D0008A198A198A198A198A198A196A198A19C8
:1060E0008A196A198A198A198A198A198A198A19B8
:1060F0008A198A198A198A198A198A198A198A1988
:106100008A198A198A198A198A198A198A198A1977
:106110008A198A198A198A198A198A198A198A1967
:106120008A196A198A198A198A198A198A198A1977
:106130008A196A198A198A196A198A198A198A1987
:106140006A118A196A118A198A196A198A196A11CF
:106150008A198A196A118A198A196A118A198A1977
:106160006A118A198A196A118A198A196A118A198F
:106170006A118A198A196A118A196A118A196A11A7
:106180008A198A196A118A198A196A118A196A1967
:106190008A198A196A198A196A198A196A118A194F
:1061A0008A196A118A198A198A196A118A198A1927
:1061B0006A118A198A198A198A198A198A198A19EF
:1061C0008A198A198A196A118A198A198A198A19DF
:1061D0008A198A198A198A198A196A118A196A11F7
:1061E0008A196A118A198A196A198A198A198A19DF
:1061F0008A198A196A198A196A118A196A118A19F7
:106200006A118A198A196A118A198A196A198A19E6
:106210008A196A118A198A196A118A198A196A11DE
:106220008A198A196A198A196A198A198A196A19B6
:106230008A198A198A198A198A196A198A198A1966
:106240008A198A198A196A198A198A198A198A1956
:106250006A198A198A198A198A198A198A198A1946
:106260008A198A198A198A198A198A198A198A1916
:106270008A198A198A198A198A198A198A198A1906
:106280008A198A198A198A198A198A198A198A19F6
:106290008A198A198A198A198A198A198A198A19E6
:1062A0008A198A198A198A198A198A198A198A19D6
:1062B0008A198A198A198A198A198A198A198A19C6
:1062C0008A198A198A198A198A198A198A198A19B6
:1062D0008A198A198A198A198A198A198A198A19A6
:1062E0008A198A198A198A198A198A198A198A1996
:1062F0008A198A198A198A198A198A198A198A1986
:106300008A198A198A198A198A198A198A198A1975
:106310008A198A198A198A198A198A198A198A1965
:106320008A198A198A198A198A198A196A198A1975
:106330008A198A198A198A198A198A196A198A1965
:106340008A198A198A198A198A198A198A198A1935
:106350006A198A196A118A198A198A196A198A198D
:106360008A198A198A196A198A198A196A198A1955
:106370008A196A198A196A198A196A118A196A1195
:106380008A198A198A198A198A198A198A198A19F5
:106390008A198A198A198A198A198A198A198A19E5
:1063A0008A198A198A198A198A198A198A198A19D5
:1063B0008A198A198A198A198A198A198A198A19C5
:1063C0008A198A198A198A198A198A198A198A19B5
:1063D0008A198A198A198A198A198A198A198A19A5
:1063E0008A198A198A198A198A198A198A198A1995
:1063F0008A198A198A198A198A198A198A198A1985
:106400008A198A198A198A198A198A198A198A1974
:106410008A198A198A198A198A198A198A198A1964
:106420008A198A198A198A198A198A198A198A1954
:106430008A198A198A198A198A198A198A198A1944
:106440008A196A118A198A198A198A198A196A1184
:106450008A196A118A198A196A118A198A198A1974
:106460008A198A198A196A198A198A196A198A1954
:106470008A196A198A196A198A198A198A198A1944
:106480008A198A198A196A198A198A198A198A1914
:106490008A198A198A198A198A198A198A198A19E4
:1064A0008A198A198A198A198A198A198A198A19D4
:1064B0008A198A198A198A198A198A198A198A19C4
:1064C0008A198A198A198A198A198A198A198A19B4
:1064D0008A198A198A198A198A198A198A198A19A4
:1064E0008A196A198A198A198A198A198A198A19B4
:1064F0008A196A198A198A198A198A196A118A19CC
:106500006A198A196A198A198A198A198A196A19D3
:106510008A198A196A198A198A196A198A198A19A3
:106520006A198A198A196A198A198A196A198A19B3
:106530006A198A198A196A198A196A198A196A19C3
:106540008A198A196A198A198A196A198A198A1973
:106550006A118A198A196A118A198A196A198A1993
:106560008A196A198A196A118A196A198A198A197B
:106570006A198A198A196A118A196A118A196A119B
:106580008A196A118A196A198A198A198A196A1163
:106590008A196A118A196A118A196A198A196A1973
:1065A0008A196A198A196A118A198A198A198A191B
:1065B0008A198A198A198A196A198A196A198A1903
:1065C0006A198A198A196A198A198A198A196A111B
:1065D0008A196A198A198A196A118A198A196A190B
:1065E0008A198A196A198A198A198A198A198A19B3
:1065F0008A198A198A198A198A198A198A198A1983
:106600008A198A198A196A198A198A198A198A1992
:106610006A198A198A198A198A198A198A198A1982
:106620008A198A198A198A198A198A198A198A1952
:106630008A198A198A198A198A198A198A198A1942
:106640008A198A198A198A198A198A198A198A1932
:106650008A198A198A198A198A198A198A198A1922
:106660008A198A198A198A198A198A198A198A1912
:106670008A198A198A198A198A198A198A198A1902
:106680008A198A198A198A198A198A198A198A19F2
:106690008A198A198A198A198A198A198A198A19E2
:1066A0008A198A198A198A198A198A198A198A19D2
:1066B0008A198A198A198A198A198A198A198A19C2
:1066C0008A198A198A198A198A198A198A198A19B2
:1066D0008A198A198A198A198A198A198A198A19A2
:1066E0008A198A198A198A198A198A198A196A19B2
:1066F0008A198A198A198A198A198A198A198A1982
:106700006A198A198A198A198A198A196A198A19B1
:106710008A198A196A198A196A118A198A196A11D1
:106720008A196A118A198A196A118A198A196A11C9
:106730008A198A196A118A198A196A198A196A19A9
:106740008A198A196A118A198A198A198A198A1959
:106750008A198A198A198A198A198A198A198A1921
:106760008A198A198A198A198A198A198A198A1911
:106770008A198A198A198A198A198A198A198A1901
:106780008A198A198A198A198A198A198A198A19F1
:106790008A198A198A198A198A198A198A198A19E1
:1067A0008A198A198A198A198A198A198A198A19D1
:1067B0008A198A198A198A198A198A198A198A19C1
:1067C0008A198A198A198A198A198A198A198A19B1
:1067D0008A198A198A198A198A198A198A198A19A1
:1067E0008A198A198A198A198A198A198A198A1991
:1067F0008A198A198A198A198A198A198A196A11A9
:106800008A196A198A198A198A196A118A196A19D8
:106810008A196A198A198A196A198A198A196A11C8
:106820008A198A196A118A198A196A118A196A19C0
:106830008A196A198A196A198A198A196A198A19A0
:106840008A196A198A198A198A198A198A198A1950
:106850008A198A198A196A198A198A198A198A1940
:106860008A198A198A198A198A198A198A198A1910
:106870008A198A198A198A198A198A198A198A1900
:106880008A198A198A198A198A198A198A198A19F0
:106890008A198A198A198A198A198A198A198A19E0
:1068A0008A198A196A198A198A198A198A198A19F0
:1068B0008A198A198A198A196A198A196A198A1900
:1068C0008A196A118A198A196A198A198A196A1918
:1068D0008A196A198A196A198A196A118A196A1130
:1068E0008A198A196A118A198A196A118A198A19E0
:1068F0006A118A198A196A118A198A198A196A11F8
:106900008A196A118A198A196A118A198A198A19BF
:106910006A198A198A196A198A196A118A198A19C7
:106920008A198A198A196A198A196A118A198A1997
:106930006A118A198A196A198A196A198A196A19C7
:106940008A196A198A196A118A198A198A196A1997
:106950008A196A198A196A198A198A198A198A195F
:106960008A198A198A196A198A196A118A196A117F
:106970008A196A118A198A196A118A198A198A194F
:106980006A118A196A118A198A196A118A196A1987
:106990008A196A118A196A118A198A196A198A194F
:1069A0006A198A198A198A198A198A198A198A19EF
:1069B0008A198A198A198A198A198A198A198A19BF
:1069C0008A198A196A198A198A198A198A198A19CF
:1069D0006A198A198A198A198A198A198A198A19BF
:1069E0008A198A198A198A198A198A198A198A198F
:1069F0008A198A198A198A198A198A198A198A197F
:106A00008A198A198A198A198A198A198A198A196E
:106A10008A198A198A198A198A198A198A198A195E
:106A20008A198A198A198A198A198A198A198A194E
:106A30008A198A198A198A198A198A198A198A193E
:106A40008A198A198A198A198A198A198A198A192E
:106A50008A198A198A198A198A198A198A198A191E
:106A60008A198A198A198A198A198A198A198A190E
:106A70008A198A198A198A198A198A198A198A19FE
:106A80008A198A198A198A198A198A198A198A19EE
:106A90008A198A198A198A198A198A198A198A19DE
:106AA0008A198A198A198A198A198A198A198A19CE
:106AB0008A198A198A198A198A198A198A198A19BE
:106AC0008A198A198A198A198A198A198A198A19AE
:106AD0008A198A198A198A196A198A198A196A11E6
:106AE0008A196A118A198A196A198A198A196A19F6
:106AF0008A198A196A198A196A118A198A196A11EE
:106B00008A198A196A198A196A118A198A198A19B5
:106B10008A198A198A198A198A198A198A198A195D
:106B20008A198A198A198A198A198A198A198A194D
:106B30008A198A198A198A198A198A198A198A193D
:106B40008A198A198A198A198A198A198A198A192D
:106B50008A198A198A198A198A198A198A198A191D
:106B60008A198A198A198A198A198A198A198A190D
:106B70008A198A198A198A198A198A198A198A19FD
:106B80008A198A198A198A198A198A198A198A19ED
:106B90008A198A198A198A198A198A198A198A19DD
:106BA0008A198A198A198A198A198A198A198A19CD
:106BB0008A198A196A118A196A118A198A196A192D
:106BC0008A196A118A198A198A196A198A198A19F5
:106BD0006A118A198A196A118A198A198A196A190D
:106BE0008A198A196A118A198A196A198A198A19D5
:106BF0008A198A198A198A198A198A198A198A197D
:106C00008A198A198A198A198A198A198A198A196C
:106C10008A198A198A198A198A198A198A198A195C
:106C20008A198A198A198A198A198A198A198A194C
:106C30008A198A198A198A198A198A198A198A193C
:106C40008A198A198A198A198A198A198A198A192C
:106C50008A198A198A198A198A198A198A198A191C
:106C60008A198A198A198A198A196A198A198A192C
:106C70008A198A198A198A196A198A196A118A1944
:106C80008A196A198A198A196A196A198A198A194C
:106C90008A198A198A198A198A196A198A196A191C
:106CA0008A198A196A198A198A196A118A198A1914
:106CB0006A118A198A196A198A196A118A196A194C
:106CC0008A196A198A198A196A198A198A198A19EC
:106CD0006A118A198A196A118A196A198A198A190C
:106CE0008A196A118A196A118A196A198A198A19FC
:106CF0006A198A196A118A198A198A198A198A19C4
:106D00008A198A198A196A198A196A118A198A19B3
:106D10006A118A198A198A198A196A118A196A11D3
:106D20008A196A118A196A118A196A198A196A19DB
:106D30008A196A198A198A196A198A196A118A19A3
:106D40006A198A196A198A198A196A198A198A198B
:106D50008A196A198A196A198A198A198A198A195B
:106D60008A198A198A198A196A198A198A198A192B
:106D70008A198A198A198A198A198A198A198A19FB
:106D80008A198A198A198A198A198A198A198A19EB
:106D90006A198A198A198A198A198A198A198A19FB
:106DA0008A198A198A198A198A198A198A198A19CB
:106DB0008A198A198A198A198A198A198A198A19BB
:106DC0008A198A198A198A198A198A198A198A19AB
:106DD0008A198A198A198A198A198A198A198A199B
:106DE0008A198A198A198A198A198A198A198A198B
:106DF0008A198A198A198A198A198A198A198A197B
:106E00008A198A198A198A198A198A198A198A196A
:106E10008A198A198A198A198A198A198A198A195A
:106E20008A198A198A198A198A198A198A198A194A
:106E30008A198A198A198A198A198A198A198A193A
:106E40008A198A198A198A198A198A198A198A192A
:106E50008A198A198A198A198A198A198A198A191A
:106E60008A198A198A198A198A198A198A198A190A
:106E70008A198A198A198A198A198A198A198A19FA
:106E80008A198A198A198A198A198A198A198A19EA
:106E90008A198A198A198A198A196A198A196A191A
:106EA0008A198A196A118A198A196A118A198A191A
:106EB0006A118A196A118A196A198A198A196A194A
:106EC0008A198A196A118A196A198A198A198A19F2
:106ED0006A118A198A198A198A198A198A198A19C2
:106EE0008A198A198A198A198A198A198A198A198A
:106EF0008A198A198A198A198A198A198A198A197A
:106F00008A198A198A198A198A198A198A198A1969
:106F10008A198A198A198A198A198A198A198A1959
:106F20008A198A198A198A198A198A198A198A1949
:106F30008A198A198A198A198A198A198A198A1939
:106F40008A198A198A198A198A198A198A198A1929
:106F50008A198A198A198A198A198A198A198A1919
:106F60008A198A198A198A198A198A198A198A1909
:106F70006A118A196A198A196A198A196A118A1989
:106F80008A196A198A196A118A198A196A118A1959
:106F90006A198A198A196A198A196A118A198A1941
:106FA0006A118A196A198A196A198A196A198A1951
:106FB0008A196A198A198A198A198A198A198A19D9
:106FC0008A198A198A198A198A198A198A198A19A9
:106FD0008A198A198A198A198A198A198A198A1999
:106FE0008A198A198A198A198A198A198A198A1989
:106FF0008A198A198A198A198A198A198A198A1979
:107000008A198A198A198A198A198A198A198A1968
:107010008A198A198A198A198A198A198A198A1958
:107020006A198A198A198A198A196A198A198A1988
:107030008A198A198A198A198A198A196A198A1958
:107040006A118A198A196A118A198A198A198A1978
:107050008A198A198A198A198A198A198A198A1918
:107060008A196A198A196A198A196A198A196A1190
:107070008A198A196A118A198A196A198A198A1940
:107080006A118A198A196A118A198A196A118A1960
:107090006A198A198A196A198A196A118A198A1940
:1070A0008A196A198A196A198A196A118A198A1930
:1070B0008A198A196A198A196A118A196A118A1928
:1070C0006A118A198A198A198A196A198A198A19F0
:1070D0006A198A196A118A198A196A198A196A1920
:1070E0008A196A198A196A198A198A198A198A19C8
